:020000040800F2
:1000000000800020FDC500085DD300085FD3000814
:1000100000000000000000000000000000000000E0
:1000200000000000000000000000000061D3000894
:10003000000000000000000063D30008799B000866
:1000400031C6000833C6000835C6000837C60008A8
:1000500039C600083BC600083DC6000843DE00085C
:1000600041C60008C99B000845C6000847C60008ED
:1000700049C600084BC600084DC600084FC6000818
:1000800051C6000853C6000855C6000857C60008E8
:1000900059C60008E99B00085DC600085FC6000855
:1000A00061C6000863C6000865C60008D99B000841
:1000B00069C600086BC600086DC600086FC6000858
:1000C000EDAF16204A62304029BD56B31544E9BF52
:1000D00077900D9CFE0B88C07E2615FA83807340B6
:0800E0000FCE674B80D541C033
:1000E800000000000000244000000000000059400B
:1000F800000000000088C3400000000084D797413A
:100108000080E03779C34143176E05B5B5B893460B
:10011800F5F93FE9034F384D321D30F94877825AD7
:080128003CBF737FDD4F15752C
:1001300001000000000000000A00000000000000B4
:100140006400000000000000E80300000000000060
:100150001027000000000000A08601000000000041
:1001600040420F0000000000809698000000000050
:1001700000E1F5050000000000CA9A3B0000000005
:1001800000E40B540200000000E87648170000006D
:100190000010A5D4E800000000A0724E180900006D
:1001A00000407A10F35A00000080C6A47E8D030040
:1001B0000000C16FF286230000008A5D784563016C
:1001C000000064A7B3B6E00D0000E8890423C78AE5
:1001D00000B581B06946002008700A4A1168012004
:1001E00003021943116000F00FF8002803D069469C
:1001F0000120087001E009F0A5FC6846007801B014
:0802000000BDC04600200240D1
:1002080000B583B0029001A9002008701748007853
:10021800002824D0164800680090144801787D20F2
:10022800C0000BF0C5F8014600980BF0C1F80DF0BE
:1002380056FB00280FD10298032808D802990022FB
:10024800D0430DF03EFB02980A49086002E001A97C
:100258000120087002E001A90120087002E001A94C
:100268000120087001A8007803B000BD9C000020A0
:0802780098000020880000201E
:100280000348027803490868801808607047C04630
:080290009C000020AC0F0020CF
:0C029800014800687047C046AC0F002011
:1002A40000B583B00290FFF7F5FF0190029800902B
:1002B4000098401C002804D0074801780098401892
:1002C4000090FFF7E7FF0199401A0099884200D295
:0C02D400F7E703B000BDC0469C0000200E
:1002E00000B589B0079006A9002008700590049019
:1002F00002900798002803D108A90120087066E140
:1003000007983C21405C0128FFD10798006900282C
:1003100005D007980069012149058842FFD1079857
:10032000806D002808D1079805F054FB079900203C
:10033000C865079954228854079800680DF0C3F9DE
:10034000002812D10798006800F052F9A24800680E
:10035000A2490BF031F84000801C0290029800285E
:1003600003D00298401E0290F8E7079800680DF04D
:10037000AAF900280BD10799886D102210438865CF
:10038000079AD16D01200143D16506A9087007982D
:1003900000680CF0F8F903900798806DC0060028FB
:1003A00000D509E10398002800D005E10798806D89
:1003B00002210843012109028843079988650798AB
:1003C00000680DF08AF9002800D0A1E00798816844
:1003D000027E92031143427ED2031143827E520376
:1003E0001143026B531E9A4112031143C268114319
:1003F0000191C07C0006002806D5079800690121FC
:10040000C9078843009002E001204005009001994F
:100410000098014307982C22805C40000143059816
:100420000843059007982021405C012813D10798C4
:10043000807E002805D10598012109040843059014
:1004400009E00799886D2022104388650799C86DD7
:1004500001221043C8650798406A002809D0079810
:10046000416A072292011140806A014305980843BE
:10047000059007980068C0685949084005990843E5
:1004800007990968C86007984168032292071140DC
:10049000C06C014304980843049007983C21405CD9
:1004A00001280FD1079948680322920710400A6C6F
:1004B00010434A6C1043896C084304990843012196
:1004C0000843049007980068006946490840049969
:1004D000084307990968086107984068032189075C
:1004E000884215D0079840680121890788420FD0BB
:1004F000079840680121C907884209D03A4908682D
:100500000F2293049843079A52681A408018086093
:10051000079908684A6B00210CF07DF90799086873
:100520008A6B32490CF077F907980069002807D1E7
:1005300007980168886A0F22D2431043886216E048
:100540000798006901214905884210D10798006881
:10055000806A0799C8698000021F1C2002400F2092
:10056000C04390400A6E104309688862FFE707980D
:10057000006800210DF0B9F80799496B88420BD14A
:1005800007990020C8650798806D01210843022162
:100590008843079988650EE00798806D102108430D
:1005A0000221884307998865079AD16D012001438C
:1005B000D16506A9087007E00799886D10221043DD
:1005C000886506A901200870069808A9087008A87F
:1005D000007809B000BDC04698000020400D03001F
:1005E0000102DEFF02FCFF1F0827014004FFFF0796
:1005F00081B00090009880680121090708430349F1
:1006000008400099886001B07047C046E8FFFF7F4E
:1006100000B585B0039000200190039800680DF0AC
:100620005CF800285BD10398006880682F49084275
:100630000CD00399886D102210438865039AD16D00
:1006400001200143D16504A908704BE003980068BC
:1006500000F00CFB26480CF033F9000200280DD501
:100660002448006824490AF0A7FE401C0190019824
:10067000002803D00198401E0190F8E70398407EBF
:1006800001282CD0FFF708FE02900398006800684C
:10069000C007002823D1039800680DF01EF8002839
:1006A00003D10398006800F0E1FAFFF7F5FD029925
:1006B000401A032812D3039800680068C007002876
:1006C0000CD10399886D102210438865039AD16D6F
:1006D00001200143D16504A9087003E0D5E704A90E
:1006E0000020087004A8007805B000BD1700008045
:0C06F0000827014098000020400D030086
:1006FC0081B000900098806803490840001D009963
:0C070C00886001B07047C046E8FFFF7F26
:1007180000B585B0039002910192039800680CF02F
:100728002EF8002860D103985421405C012803D199
:1007380004A9022008705DE003995422012088541E
:1007480003980068C068C00700280FD103980068A4
:100758000CF0BFFF002803D00398006800F056F89B
:1007680003980168C86801221043C8600398FFF71E
:100778004BFF0146684601700078002833D1039882
:10078800806D0121090208431C49084003998865C6
:1007980003990020C8650398016D1948C862039839
:1007A800016D184808630398016D1748486303985A
:1007B80001681C200860039954220020885403987B
:1007C800016848681022104348600399086D096859
:1007D8004031029A019B0CF031F969460870039880
:1007E8000068FFF787FF02E069460220087000985A
:1007F80004A9087004A8007805B000BDFEF1FFFF49
:0C080800B7D7000853C8000869C80008F2
:1008140081B000900098806803490840801C0099CA
:0C082400886001B07047C046E8FFFF7F0D
:1008300000B59DB01B901A9119A90020087017905F
:100840001B9800690121C907884204D01B980069E0
:10085000E649884200D1FFE71B985421405C0128FB
:1008600003D11CA902200870BCE11B99542201206D
:1008700088541B9800680BF086FF002800D0A2E186
:100880001A984068022800D15BE11B980069012199
:10089000C907884204D01B980069D449884206D110
:1008A0001B9800681A99096800F0AEF9F1E01B98EE
:1008B000016E1A9843681F2213400F229A409143F9
:1008C000169100684003002807D11A9800681F217C
:1008D00089060840800E1590C2E01A980078C0077B
:1008E000002802D000201490B8E01A980078800701
:1008F000002802D501201390AEE01A980078400736
:10090000002802D502201290A4E01A98007800076F
:10091000002802D5032011909AE01A980078C006AA
:10092000002802D50420109090E01A9800788006E4
:10093000002802D505200F9086E01A98007840061E
:10094000002802D506200E907CE01A980078000658
:10095000002802D507200D9072E01A984078C00751
:10096000002802D008200C9068E01A984078800790
:10097000002802D509200B905EE01A9840784007C5
:10098000002802D50A200A9054E01A9840780007FF
:10099000002802D50B2009904AE01A984078C0063A
:1009A000002802D50C20089040E01A984078800674
:1009B000002802D50D20079036E01A9840784006AE
:1009C000002802D50E2006902CE01A9840780006E8
:1009D000002802D50F20059022E01A988078C007E1
:1009E000002802D01020049018E01A988078800720
:1009F000002802D5112003900EE01A98016801200A
:100A0000820411401220002301939142029001D0F0
:100A1000019802900298039003980490049805901E
:100A200005980690069807900798089008980990EE
:100A300009980A900A980B900B980C900C980D90BE
:100A40000D980E900E980F900F981090109811908E
:100A5000119812901298139013981490149815905E
:100A6000169815991A9A52681F231A409140084304
:100A70001B9908661A9840688008401C1B99C96930
:100A8000884206D81B9800681A9A516812680BF0C1
:100A900000FF1B9800681A9A1168926800F0C2F86B
:100AA0001A98C078000600284AD551480BF008FF74
:100AB00018901A9800684F4988421DD118A880786C
:100AC0000006002818D418990120C00501434848A1
:100AD0000CF0CDFE4A4800684A490AF06DFC014618
:100AE0000C2048430C3017901798002803D0179813
:100AF000401E1790F8E723E01A9800683E498842A4
:100B00000CD118A8C078C007002807D11899012077
:100B10000006014336480CF0AAFE11E01A9800685E
:100B2000364988420CD118A880784006002807D49E
:100B300018990120800501432D480CF098FEFFE72D
:100B400040E01B9800690121C907884204D01B9826
:100B500000692649884205D11B9800681A990968DE
:100B600000F074F81A98C078000600282AD52048AA
:100B70000BF0A6FE18901A9800681E49884207D10B
:100B800018990120C005814319480CF070FE19E046
:100B90001A9800681849884207D118990120000660
:100BA000814313480CF063FE0CE01A980068134967
:100BB000884207D118990120800581430C480CF028
:100BC00056FEFFE707E01B99886D202210438865D9
:100BD00019A9012008701B995422002088541998E3
:100BE0001CA908701CA800781DB000BD040000807E
:100BF00008270140001000B0004000B8002000B4F9
:080C000098000020400D0300E4
:100C080082B001900091009A034802400199886AD5
:0C0C18001043886202B07047FFFF070025
:100C240083B00290019100920298406901990A02EE
:100C3400904300991140034A1140084302994861C6
:080C440003B0704700FFFF0739
:100C4C0082B0019000910098C2430448024301997C
:100C5C00886A1040886202B07047C0460000F8FFF6
:100C6C0081B000900098806803490840401C0099AE
:0C0C7C00886001B07047C046E8FFFF7FB1
:100C880000B58BB009900020079004900998542172
:100C9800405C012803D10AA902200870C5E009991F
:100CA80054220120885409980CF029FD08A90870DD
:100CB800099800680CF0E5FD002800D0A9E0099823
:100CC800806D02210843012109028843099988653A
:100CD80009980068C0685749084006900998016853
:100CE800C868554A1040C860002005900598072834
:100CF8002DD8099800680BF0F1FD099800680CF0F0
:100D0800C8FD002817D00798401C079007984C4941
:100D180088420FD30998806D102108430221884327
:100D28000999886509995422002088540AA9012044
:100D380008707AE0E1E7099800680BF0DCFD0146ED
:100D48000498401804900598401C0590CEE7059932
:100D580004980AF02DFB04900998006800F072F8D6
:100D6800099800680BF0D0FD002817D133480BF024
:100D7800D4FD02900298800C07280FD30298800CAB
:100D8800C11E0120884001900198400801900198F7
:100D9800002803D00198401E0190F8E709980068E0
:100DA80004990CF080FD0998006800F059F8FFF7E5
:100DB8006FFA0390099800680CF063FD002819D0B9
:100DC800FFF766FA0399401A032812D309980068B6
:100DD8000CF057FD00280CD00999886D102210439B
:100DE8008865099AD16D01200143D1650AA9087067
:100DF8001BE0DFE7069A09980168C8681043C860D5
:100E08000998806D01210843022188430999886562
:100E180004E00999886D10221043886509995422C5
:100E28000020885408980AA908700AA800780BB00E
:100E380000BDC04603800000FC7FFFFF082701407B
:040E480000F20200B2
:100E4C0081B000900098806803490840401C0099CC
:0C0E5C00886001B07047C046E8FFFF7FCF
:100E680081B000900098806803490840801C009970
:0C0E7800886001B07047C046E8FFFF7FB3
:100E840070B582B0024601A802700091002140565C
:100E9400002815D4002401A908570322D34318407D
:100EA400164A805809578C07E50EFF24AC40A0432E
:100EB400009CA401E4B2AC4020431940885019E0DE
:100EC40001A908780F24204008380322D34318408E
:100ED400094A8058002549578D07EE0EFF25B54075
:100EE400A843009DAD01EDB2B54028432140083927
:100EF4001940885002B070BD1CED00E000E400E031
:100F040081B001466846017000214056002807D48C
:100F1400684601781F20014001208840014908608B
:080F240001B0704700E100E09C
:100F2C0081B00146684601700021405600280BD460
:100F3C00684601781F200140012088400349086061
:100F4C00BFF34F8FBFF36F8F01B0704780E100E0AC
:100F5C0000B583B001900198401E000E002802D00D
:100F6C000120029010E00198401E09490860002001
:100F7C000090C0430321FFF77FFF009805490860EC
:100F8C00054A072111600290029803B000BDC046CB
:0C0F9C0014E000E018E000E010E000E0CD
:100FA80000B583B001900198002803D102A901205F
:100FB800087050E00198407F002805D10199002071
:100FC800087701980CF093FC019902204877019862
:100FD800007900280CD101980168214848610198DE
:100FE80000688068182188430199096888600AE0C8
:100FF80001988168C2680BF039FB002803D002A968
:101008000120087027E001984079002805D101984F
:1010180001680020C043086103E001990869096874
:1010280008610198006880686021884301994A69CD
:1010380010430968886001980068806880218843A7
:1010480001998A69104309688860019901204877E5
:1010580002A90020087002A8007803B000BDC046AD
:04106800B71DC104EB
:10106C0000B585B003900398002803D104A9012092
:10107C00087066E003980190006834494018142108
:10108C000AF094F901998000086403992522022042
:10109C0088540398016808682D4A1040086003982A
:1010AC0002908268C1680A4301690A4341690A4394
:1010BC0081690A43C1690A43016A0A4301680868E5
:1010CC0010430860039800F045F8039880680121EC
:1010DC008903884202D1039900204860039948682B
:1010EC003F221040496C08600399C86C896C4860B9
:1010FC000398406800280FD00398406804280BD848
:10110C00039800F049F80398016D002008600399DA
:10111C00886D496D486006E00399002008650399C5
:10112C0048650399886503990020C86303992522B3
:10113C0001208854039924220020885404A90020FB
:10114C00087004A8007805B000BDC046F8FFFDBFCC
:04115C000F80FFFF02
:1011600000B583B002900299086C032290430B4AA9
:101170008018486402980078083814210AF01CF995
:10118000019002990648886401991F2001400120BE
:1011900088400299C86403B000BDC0460008024000
:0411A0008008024081
:1011A40082B00190019840683F2108400090009867
:1011B4008000084940180199086501990648486566
:1011C4000098411E03200140012088400199886550
:0C11D40002B07047FC08024040090240D5
:1011E00084B003900291019200930399C86C896CBA
:1011F00048600398006D002803D00399886D496DFD
:1012000048600398006C1C210840012282400F496D
:1012100008681043086000980399096848600398BB
:101220008068102808D1019803990968886002989D
:1012300003990968C86007E0029803990968886003
:10124000019803990968C86004B07047040002401F
:1012500000B583B002904C48006801900298006885
:101260000068009001980299096C1C221140C84046
:101270004007002822D568460078400700281DD581
:101280000298006800688006002805D4029801686A
:1012900008680422904308600298006C1C210840F2
:1012A0000422824039490868104308600298006BA4
:1012B000002802D00298016B884763E001980299E8
:1012C000096C1C221140C840800700282AD56846B6
:1012D00000788007002825D50298006800688006FD
:1012E000002809D40298016808680A22904308601F
:1012F00002992522012088540298006C1C21084084
:101300000222824021490868104308600299242281
:10131000002088540298C06A002802D00298C16A4E
:1013200088472FE001980299096C1C221140C8409F
:101330000007002826D5684600780007002821D538
:101340000298016808680E22904308600298016CB8
:101350001C200140012003468B400C4A11681943B0
:1013600011600299C86302992522885402992422A7
:10137000002088540298406B002802D00298416BEC
:101380008847FFE703B000BD0000024004000240B0
:1013900010B588B006900591039302921C4800781E
:1013A000012803D107A9022008702DE01849012067
:1013B00008701749002048607D20C00000F034F814
:1013C000014601A801700078002817D1069801286D
:1013D00005D10598039B029A00F07AF803E005987E
:1013E000029900F019F87D20C00000F01DF801A955
:1013F0000870069A0749086890430860044900206D
:101400000870019807A9087007A8007808B010BDF7
:10141000800F00201420024008B4024B9C4608BCF8
:081420006047C04601000020F6
:1014280000B585B00390FEF733FF0190012000045A
:10143800029021480068029908420FD00398401C86
:1014480000280AD0FEF724FF0199401A0399884220
:1014580003D304A90320087029E0EAE716490868BD
:10146800164A10400290164808600298002806D0D4
:1014780002981449486004A90120087017E00E4832
:101488000068400300280FD50398401C00280AD0A4
:10149800FEF7FEFE0199401A0399884203D304A976
:1014A8000320087003E0EAE704A90020087004A8F4
:1014B800007805B000BDC04610200240FA83000045
:0814C800FB830000800F0020EF
:1014D00084B00390019300920749086801221043E9
:1014E0000860009803990860BFF36F8F0198039913
:0C14F000486004B07047C0461420024061
:1014FC0081B06946002008700A480068C00F0028B7
:10150C000CD009490948086009480860054800687A
:10151C00C00F002802D06946012008706846007888
:10152C0001B0704714200240082002402301674597
:04153C00AB89EFCDBB
:1015400000B583B002A90120019008707D20C00081
:10155000FFF76AFF019A08480168D207114301604A
:101560000068C00F002802D002A90020087002A85D
:0C157000007803B000BDC046142002400B
:10157C0081B06946012008700A48006840000028C4
:10158C000CD50949094808600948086005480068F5
:10159C004000002802D46946002008706846007894
:1015AC0001B07047142002400C2002403B2A19085D
:0415BC007F6E5D4C95
:1015C00000B583B002A90120019008707D20C00001
:1015D000FFF72AFF019A084801689207114301604A
:1015E00000684000002802D502A90020087002A867
:0C15F000007803B000BDC046142002408B
:1015FC0000B585B0039002912E480078012803D1E4
:10160C0004A90220087051E02A49012008702949D8
:10161C00002048607D20C000FFF700FF014601A8B4
:10162C000170007800283BD103990420486003988E
:10163C00006804280AD10398406800F03FF87D2028
:10164C00C000FFF7EBFE01A9087029E00299002009
:10165C00C04308600398806800900098039A9168D2
:10166C00D2688918884216D203984068009900F015
:10167C0033F87D20C000FFF7D1FE014601A80170B0
:10168C000078002803D000980299086003E00098C5
:10169C00401C0090E1E7084908680222904308606A
:1016AC00044900200870019804A9087004A8007867
:0C16BC0005B000BD800F0020142002408B
:1016C80081B00090009804490A681043012212046E
:0C16D8001043086001B07047142002406D
:1016E40083B00290019107490868074A10400090AE
:1016F400009A0198C0001043044A1043086003B0E4
:101704007047C0461420024007E0FFFF02000100BA
:1017140000B587B0059035480078012803D106A9A3
:10172400022008705EE03149012008702F49002032
:10173400486005980078C007002805D0059A5068CD
:101744009168D26800F056F80598006806210840B0
:10175400062806D1059A50699169126900F064F867
:101764001DE0059800788007002809D500F074F87A
:101774000490049905980269084600F055F80EE0B3
:10178400059800784007002809D500F073F8049004
:10179400059948698969049A00F046F8FFE77D20B5
:1017A400C000FFF73FFE014603A80170007800283F
:1017B40012D10F4902910868012252040192104388
:1017C40008607D20C000FFF72DFE019A029903AB4B
:1017D4001870086890430860044900200870039852
:1017E40006A9087006A8007807B000BD800F002085
:0417F400142002407B
:1017F80083B00290019100920298012806D10098C6
:101808000004019908430649086005E000980004AF
:10181800019908430149086003B07047302002402D
:041828002C2002402E
:10182C0084B0039002910192084908680090039AD1
:10183C0000989043FF22904300900098029A104326
:10184C00019A1043086004B07047C0462020024043
:10185C0081B004480068044908400090009801B029
:0C186C007047C0462020024000604F077B
:1018780082B009480068C0B200900098AA2805D034
:101888000098CC2802D0BB20019001E0009801907C
:0C189800019802B07047C04620200240BA
:1018A40000B581B00090009907200860009A506844
:1018B400114608310C3200F00FF8FFF7DBFF0099F6
:1018C4000861FFF7C9FF00998861009901484861E0
:0818D40001B000BD00604F07E8
:1018DC0083B0029001910092029801280CD10E481D
:1018EC0002683F210A40019B1A6000680904084005
:1018FC00000C009908600BE0064802683F210A4082
:10190C00019B1A60006809040840000C00990860EB
:0C191C0003B07047302002402C20024035
:101928008AB00990089100200790089800680799E4
:10193800C840002800D130E108980068079A0121C2
:101948009140084006900698002800D121E10898A7
:10195800406803210840012805D008984068032101
:10196800084002282AD10998806805900798400005
:10197800032181400598884305900898C168079815
:1019880040008140059808430590059809998860AA
:101998000998406805900798012181400598884377
:1019A800059008984068102108400109079881406F
:1019B8000598084305900598099948600898406873
:1019C80003210840032814D00998C0680590079897
:1019D8004000032181400598884305900898816854
:1019E8000798400081400598084305900598099993
:1019F800C860089840680321084002281ED1099849
:101A08000799C90889004018006A05900798400797
:101A1800C00E0F21814005988843059008980169F8
:101A280007984007C00E814005980843059005981F
:101A38000999079AD20892008918086209980068DB
:101A4800059007984100032002468A400599914372
:101A58000591089949680140079840008140059818
:101A680008430590059809990860089880798007C7
:101A7800002800D18DE00798032188434849405841
:101A8800059007988007C00E0F218140059888436C
:101A98000590099805210907884202D10020049081
:101AA8001DE009983F49884202D10120039014E0C3
:101AB80009983D49884202D1022002900BE0099919
:101AC8003A4A0320052300939142019001D00098DF
:101AD8000190019802900298039003980490049949
:101AE80007988007C00E814005980843059005981F
:101AF8000799032291432A4A88502D480068059087
:101B0800069905988843059008988079C0060028AA
:101B180003D5069905980843059005982449086057
:101B28002448006805900699059888430590089808
:101B380080798006002803D5069905980843059002
:101B480005981C4908601C48006805900699059886
:101B580088430590089880798007002803D506995E
:101B680005980843059005981349086013480068CC
:101B78000590069905988843059008988079C007CC
:101B8800002803D0069905980843059005980B4945
:101B980008600798401C0790C7E60AB07047C0461F
:101BA800601802400004005000080050000C00506B
:101BB80000180240041802408418024080180240AD
:101BC80000B581B0694608800D4800680988084258
:101BD80006D0684601880A4A116000880AF0BAFFF0
:101BE8000848006869460988084206D0684601889E
:101BF800044A1160008806F08FFE01B000BDC0469F
:081C08000C1802401018024004
:101C10000349086801221202104308607047C04659
:041C20000070004010
:101C24000349086801221202904308607047C046C5
:041C340000700040FC
:101C380000B583B001901749086803225202904307
:101C4800019A10430860019801214902884219D17C
:101C58001148016806204843104909F0A9FB401CB7
:101C680000900F480068400500280BD50098002810
:101C780003D00098401E009003E002A903200870DA
:101C880003E0EEE702A90020087002A8007803B07C
:101C980000BDC046007000409800002040420F0080
:041CA8001470004074
:101CAC0010B588B006900698002803D107A901202A
:101CBC000870C0E206980078C007002873D0FA4874
:101CCC000068382108400490F84800680321084057
:101CDC0003900498102802D10398032802D004988A
:101CEC0008280DD1F24800688003002807D5069813
:101CFC004068002803D107A9012008709BE252E03C
:101D0C000698406801210904884206D1E849086810
:101D1C0001221204104308601AE00698406805215D
:101D2C00090488420AD1E249086801229304184345
:101D3C000860086812041043086009E0DC49086870
:101D4C0001221304984308600868920490430860C9
:101D5C0006984068002813D0FEF798FA0590D448EE
:101D6C000068800300280AD4FEF790FA0599401AFF
:101D7C00652803D307A9032008705CE2EFE712E0A3
:101D8C00FEF784FA0590CA480068800300280AD53B
:101D9C00FEF77CFA0599401A652803D307A903209E
:101DAC00087048E2EFE7069800788007002800D416
:101DBC0090E0BD480068382108400490BB4800689A
:101DCC000321084003900498102802D1039802289C
:101DDC0002D00498002834D1B5480068400500288A
:101DEC0007D50698C068002803D107A90120087000
:101DFC0021E2B04908687F2212029043069A526988
:101E0C00120210430860049800280FD1A8480268F9
:101E1C000721C9028A43069B1B691A4302600068AA
:101E2C000840C10AA448C840A4490860A4480068F6
:101E3C00FEF7E4F9002803D007A901200870FAE1A5
:101E4C0048E00698C06800282BD0994908680722FA
:101E5C00D2029043069A1269104308600868012266
:101E6C00120210430860FEF711FA0590F64800685C
:101E7C00400500280AD4FEF709FA0599401A0328F0
:101E8C0003D307A903200870D5E1EFE7EF490868F1
:101E9C007F2212029043069A526912021043086084
:101EAC0018E0E94908680122120290430860FEF725
:101EBC00EDF90590E4480068400500280AD5FEF7C6
:101ECC00E5F90599401A032803D307A903200870E4
:101EDC00B1E1EFE7069800780007002848D5D8480C
:101EEC0000683821084018280DD1D94800688007AF
:101EFC00002807D506988069002803D107A901207E
:101F0C00087098E134E006988069002818D0D04910
:101F1C000868012210430860FEF7B8F90590CC4818
:101F2C000068800700280AD4FEF7B0F90599401A1A
:101F3C00032803D307A9032008707CE1EFE717E01F
:101F4C00C3490868012290430860FEF79FF9059089
:101F5C00BF480068800700280AD5FEF797F9059955
:101F6C00401A032803D307A90320087063E1EFE7A5
:101F7C00069800784007002800D4ADE002A90020A4
:101F8C000870AF4800683821084020280DD1B348AC
:101F9C0000688007002807D506988068002803D1C0
:101FAC0007A90120087046E196E0AA480068C00025
:101FBC0000280CD4A7480268012109070A430260D3
:101FCC00006808400190019802A901200870A248FD
:101FDC000068C005002818D49F4908680122120225
:101FEC0010430860FEF752F905909B480068C00545
:101FFC0000280AD4FEF74AF90599401A032803D39E
:10200C0007A90320087016E1EFE7069880680128FD
:10201C0005D19249086801221043086016E0069821
:10202C008068052809D18D4908680422104308608E
:10203C00086801221043086008E0884908680122FA
:10204C0090430860086804229043086006988068F2
:10205C00002814D0FEF71AF9059080480068800714
:10206C0000280BD4FEF712F90599401A7C498842D6
:10207C0003D307A903200870DDE0EEE722E0FEF7AA
:10208C0005F9059075480068800700281AD5FEF7F9
:10209C00FDF80599401A7249884203D307A9032019
:1020AC000870C8E0EEE7C046081002400C10024071
:1020BC0000100240041002400024F400980000209C
:1020CC008800002002A80078012805D16149086821
:1020DC0001221207904308600698C069002800D1BD
:1020EC00A6E0574800683821084010286AD00698A6
:1020FC00C069022847D1544908680122120690434E
:10210C000860FEF7C3F805904F480068800100286E
:10211C000AD5FEF7BBF80599401A032803D307A983
:10212C000320087087E0EFE7464908684E4A1040E4
:10213C00069B1A6A5C6A22439C6A24022243DC6A6C
:10214C0022431B6B1A43104308603F4B1868012253
:10215C001406204318600868120710430860FEF745
:10216C0095F8059038480068800100280AD4FEF7DD
:10217C008DF80599401A032803D307A9032008708A
:10218C0059E0EFE71DE03049086801221206904340
:10219C000860FEF77BF805902B480068800100284A
:1021AC000AD5FEF773F80599401A032803D307A93B
:1021BC00032008703FE0EFE722490868294A1040E5
:1021CC00086035E00698C069012803D107A90120F1
:1021DC00087030E01B480068039003980321084006
:1021EC000699096A88421FD1039870210840069904
:1021FC00496A884218D103987F2109020840069940
:10220C00896A090288420FD103981F2149040840AA
:10221C000699C96A884207D10398072149070840E3
:10222C000699096B884203D007A90120087002E0C7
:10223C0007A90020087007A8007808B010BDC04698
:10224C00081002400C100240001002400410024022
:10225C00601002403C100240007000405C100240D4
:0C226C0089130000FCFFFEEF8C80C11FF6
:1022780000B585B0039002910398002803D104A902
:1022880001200870E9E002987649096807221140A0
:1022980088421CD97349086807229043029A104360
:1022A8000860FDF7F5FF01906E48006807210840B7
:1022B800029988420BD0FDF7EBFF0199401A71494A
:1022C800884203D304A903200870C6E0ECE703980A
:1022D80000788007002813D5039800784007002865
:1022E80005D56149086807221203104308605E4952
:1022F80008680F2212029043039A926810430860FC
:1023080003980078C007002860D003984068012827
:1023180009D1584800688003002803D404A9012083
:1023280008709AE032E003984068022809D15148C1
:1023380000688001002803D404A9012008708CE0FB
:1023480024E003984068002809D14A4800684005FD
:10235800002803D404A9012008707EE016E0039841
:102368004068032809D1424800688007002803D440
:1023780004A90120087070E008E03C480068800764
:10238800002803D404A90120087066E036490868CB
:1023980007229043039A526810430860FDF778FFBC
:1023A8000190314800683821084003994968C900FC
:1023B80088420BD0FDF76CFF0199401A31498842D9
:1023C80003D304A90320087047E0EAE702982549E7
:1023D80009680722114088421CD22249086807224E
:1023E8009043029A10430860FDF752FF01901D4880
:1023F800006807210840029988420BD0FDF748FF82
:102408000199401A1F49884203D304A90320087080
:1024180023E0ECE7039800784007002808D5124924
:102428000868072212039043039AD2681043086091
:1024380000F02AF80C4909680F22120211408A0993
:102448000D4989581F221140C8400C4908600C48A2
:102458000068FDF7D5FE04A9087004A8007805B047
:1024680000BDC04600200240081002405C10024037
:10247800601002400010024004C5000898000020C7
:08248800880000208913000008
:1024900000B587B03A4800688006400F00280ED18A
:1024A0003B4800680721C9020840C10A0120884052
:1024B00002900299354808F07FFF01905CE03048B7
:1024C000006838210840082802D12F48019053E0C5
:1024D0002B48006838210840102837D12948016866
:1024E0000322114005910068702108400009401C3A
:1024F000039005980090022810D0009803280DD171
:102500000399214808F058FF01461E4800687F22C1
:1025100012021040000A484306900CE003991B4841
:1025200008F04AFF0146174800687F221202104057
:10253000000A4843069013480068400F401C04906E
:102540000698049908F038FF019015E00C480068DF
:1025500038210840202803D10120C00301900BE05E
:102560000748006838210840182803D17D20000260
:10257000019001E000200190019807B000BDC04625
:10258000081002400C10024000127A000024F400EF
:0425900000100240F5
:0C259400014800687047C0469800002015
:1025A00000B581B0FFF7F6FF009000F00DF801468E
:1025B0000098090B8A00034989581F221140C8401E
:0825C00001B000BD44C5000894
:1025C80002480068072109030840704708100240C4
:1025D80000B587B0069003A90020087002A908700A
:1025E800069880788007002800D487E001A9002099
:1025F800087072480068C00000280CD46F48026850
:10260800012109070A430260006808400090009809
:1026180001A9012008706A490868012212021043C2
:102628000860FDF735FE049065480068C00500287D
:102638000AD4FDF72DFE0499401A032803D303A9F1
:102648000320087000E0EFE703A80078002848D1CD
:102658005C48006803210902084005900598002895
:1026680014D005980699896988420FD05549086899
:1026780003221202904305900868012212041043B5
:1026880008600868904308600598086005A8007805
:10269800C007002813D0FDF7FBFD049049480068E7
:1026A800800700280BD4FDF7F3FD0499401A46492A
:1026B800884203D303A90320087000E0EEE703A8CB
:1026C8000078002809D13F49086803221202904384
:1026D800069A92691043086002E0039802A90870FC
:1026E80002E0039802A9087001A80078012805D122
:1026F800324908680122120790430860069800785A
:10270800C007002807D03149086803229043069A79
:10271800526810430860069800788007002807D59B
:102728002A4908680C229043069A92681043086068
:10273800069800788006002808D5244908680322EE
:1027480012039043069AD2681043086006984078AE
:102758004006002814D51D490868032292079043B3
:10276800069A526910430860069840690121890752
:10277800884205D1164908680122120410430860EE
:10278800069840780007002814D5104908680322E5
:1027980092039043069A12691043086006980069EC
:1027A80001218903884205D10949086801221204D8
:1027B8001043086002A8007807B000BD3C10024032
:1027C800007000405C100240891300005410024061
:0427D8000C1002409F
:1027DC0000B583B0029001A901200870029800286E
:1027EC0065D002982921405C00280AD10299282240
:1027FC000020885402991120C0024860029806F00B
:10280C00CBFF029929220220885402980168CA2021
:10281C0048620298016853204862029800F04EF812
:10282C00014601A801700078002834D10298016893
:10283C008869214A104088610298826841690A437C
:10284C00C1690A4301688869104388610299086963
:10285C00096808610298C1680A0401680869104394
:10286C000861029800F066F8014601A80170007832
:10287C00002810D1029801688869072252079043FA
:10288C0088610298426A016A0A4381690A430168B5
:10289C0088691043886102980168FF20486201A88A
:1028AC000078002803D1029929220120885401A81C
:0C28BC00007803B000BDC046BFFF8FFBDA
:1028C80000B585B0049002A900200870049800683B
:1028D800C0684006002828D404980168C868802287
:1028E8001043C860FDF7D4FC039004980068C168E1
:1028F800002049060029019005D402A80078C01ECE
:10290800411E884101900198C00700280DD0FDF7AD
:10291800BFFC0399401A0749884205D302A903203E
:102928000870049929228854DFE702A8007805B0C6
:0829380000BDC046E9030000E8
:1029400000B583B0029001A90020087017490868FB
:1029500080229043086016480068800600280BD447
:10296000029800F045F9002805D002992922032099
:10297000885401A9087014E00D490868202290438A
:102980000860029800F034F9002805D00299292245
:102990000320885401A908700549086820221043C3
:1029A000086001A8007803B000BDC0460C280040B4
:0429B00018280040A3
:1029B40000B589B007900691059207982821405CDC
:1029C400012803D108A90220087085E0079928226C
:1029D4000120885407992922022088540798016805
:1029E400CA20486207980168532048620798FFF795
:1029F40069FF014603A801700078002859D10598A1
:102A0400002825D10798006880694006002800D571
:102A140002E006990020C870069800780AF0FBFFCF
:102A240000040190069840780AF0F5FF01460198E9
:102A3400090240180290069880780AF0ECFF0146DB
:102A4400029840180699C97889050843049015E04E
:102A54000798006880694006002800D502E00699BE
:102A64000020C8700699087800044A781202801879
:102A74008A788018C978890508430490049818490D
:102A84000840079909680860079801688869012265
:102A94009204904388610698C268006902430798CB
:102AA40001688869104388610798FFF747FF03A905
:102AB400087007980168FF20486203A8007800287E
:102AC40003D107992922012088540799282200203C
:102AD4008854039808A9087008A8007809B000BDB4
:042AE4007F7F7F0071
:102AE80000B589B007900691059207982821405CA7
:102AF800012803D108A9022008706FE0079928224D
:102B08000120885407992922022088540598002812
:102B18000AD106984078C006002805D50699487855
:102B2800EF2210400A304870059800281BD10698FB
:102B3800C0780AF06EFF00040190069840780AF009
:102B480068FF0146019809024018029006988078AB
:102B58000AF05FFF01460298401806990978490370
:102B6800084304900BE00699C87800044A781202DA
:102B780080188A78801809784903084304900798D0
:102B88000168CA204862079801685320486207987C
:102B9800FFF796FE014603A80170007800280AD1C5
:102BA8000498104908400799096848600798FFF792
:102BB800C3FE03A9087007980168FF20486203A8AC
:102BC8000078002803D10799292201208854079901
:102BD800282200208854039808A9087008A80078BB
:082BE80009B000BD3FFFFF0032
:102BF00000B583B0019001980168C868A022904395
:102C0000C860FDF749FB009001980068C068800625
:102C100000280BD4FDF740FB0099401A0749884271
:102C200003D302A90320087003E0EDE702A9002006
:102C3000087002A8007803B000BDC046E903000098
:102C400010B584B002900298002803D103A9012096
:102C5000087090E00298406A00280AD10298406803
:102C600041218900884200D102E002990020C86118
:102C700004E002990020086102994861029900204D
:102C8000886202985D21405C002806D102995C228E
:102C900000208854029806F007FF02995D22022066
:102CA000885402980168086840229043086002989E
:102CB000C0683349884202D30020019002E001201D
:102CC000000301900298C0680F210902884208D0D1
:102CD0000298C06807210902884202D002990020A8
:102CE0008862029A009250684121890008409168E8
:102CF00021239B02194040181169022319404018F2
:102D0000536901210B40C01893694C022340C0183D
:102D1000D36938242340C018136A80242340C01884
:102D2000936A4C032340184312681060029A508B38
:102D300004231840536A10242340C018536B0824FE
:102D40002340C018D3680F2424022340C018019BDD
:102D50000C032340C0181268506002980268D069C2
:102D6000CB029843D061029A00201066029A5D233C
:102D7000D15403A9087003A8007804B010BDC04660
:042D80000107000047
:102D840010B58EB0109C0C900B910A9209A8038088
:102D94000120049003A9002008700C985C21405C79
:102DA400012803D10DA90220087083E10C995C224B
:102DB40001208854FDF76EFA05900C985D21415C62
:102DC40006A801700C9949680791099908AA11800D
:102DD4000078012810D0079841218900884207D142
:102DE4000C988068002803D106A80078042803D032
:102DF40003A90220087056E10B98002806D00A980F
:102E0400002803D009A80088002803D103A90120C1
:102E1400087048E10C985D21405C042803D00C99AB
:102E24005D22052088540C99002008660A990C9AA2
:102E3400116409990C9A4623D15209990C9A442396
:102E4400D1520B990C9A916309990C9AD1870999DB
:102E54000C9A91870C99C8640C9908650C98C06801
:102E64009649884207D30C980168486801221203E6
:102E74009043486006E00C980168486801221203F8
:102E8400104348600C9800680068402108404028BE
:102E940005D00C98016808684022104308600C981B
:102EA400C0688649884271D30C984068002803D0D2
:102EB40008A8008801280CD10C99886B008809683F
:102EC400C8600C99886B801C88630C99C88F401E5D
:102ED400C8870C98C18F01200029029005D10C9855
:102EE4004621405A411E884102900298C00700289A
:102EF4004BD00C98006880688007002815D50C9882
:102F0400C08F002811D0049801280ED10C99886B29
:102F140000880968C8600C99886B801C88630C99C8
:102F2400C88F401EC887002004900C9800688068F1
:102F3400C007002815D00C984621405A002810D00C
:102F44000C980068C0680C99096C08800C99086C8E
:102F5400801C08640C994622885A401E885201201D
:102F64000490FDF797F90599401A109988420BD3FC
:102F74001098401C002807D003A9032008700C995E
:102F84005D22012088548EE0A3E773E00C9840682A
:102F9400002803D008A8008801280CD10C99886B5C
:102FA4000078096808730C99886B401C88630C9935
:102FB400C88F401EC8870C98C18F0120002901903A
:102FC40005D10C984621405A411E88410190019830
:102FD400C00700284ED00C9800688068800700283D
:102FE40015D50C98C08F002811D0049801280ED153
:102FF4000C99886B0078096808730C99886B401CDD
:1030040088630C99C88F401EC887002004900C98D0
:1030140000688068C007002815D00C984621405AE3
:10302400002810D00C980068007B0C99096C08707B
:103034000C99086C401C08640C994622885A401E5E
:10304400885201200490FDF725F90599401A10993A
:10305400884203D31098401C002802D110980028FD
:1030640007D103A9032008700C995D22012088541C
:1030740019E0A0E70C981099059A09F072FD002850
:1030840005D003A9012008700C99202008660C982B
:10309400006E002803D003A90120087003E00C99F6
:1030A4005D22012088540C995C22002088540398E6
:1030B4000DA908700DA800780EB010BD010700001E
:1030C40010B58CB00E9C0A9009910892079302A93E
:1030D4000020087007980190FDF7DCF8024601987B
:1030E4000E99891A40180590FDF7D4F804900A98AF
:1030F40000680C30039005993A4802682320504335
:10310400000D484306900A980068806809990840B1
:10311400089988425FD0099803214902884207D15F
:103124000898002804D10398007802A9087002982E
:103134000798401C00284DD0FDF7ACF80499401ABC
:103144000599884202D2059800283BD10A98016863
:103154004868E022904348600A9840684121890009
:10316400884211D10A9880680121C903884205D098
:103174000A98806801218902884205D10A98016869
:1031840008684022904308600A98806A0121490334
:1031940088420BD10A9801680868012252039043BF
:1031A40008600A9801680868104308600A995D225B
:1031B400012088540A995C22002088540BA903201A
:1031C40008700BE00698002801D1002005900698AD
:1031D400401E069097E70BA9002008700BA8007802
:0831E4000CB010BD98000020A2
:1031EC0010B58AB00C9C0890079106A80270059344
:1031FC0005980190FDF74AF8024601980C99891A36
:10320C0040180390FDF742F8029003993548006886
:10321C004001000D484304900898006880680799A5
:10322C000840401A4142484106A90978884252D0C8
:10323C000598401C00284DD0FDF728F80299401A3B
:10324C000399884202D2039800283BD10898016860
:10325C004868E02290434860089840684121890002
:10326C00884211D1089880680121C903884205D091
:10327C000898806801218902884205D10898016864
:10328C0008684022904308600898806A012149032D
:10329C0088420BD1089801680868012252039043B8
:1032AC0008600898016808681043086008995D2256
:1032BC000120885408995C220020885409A9032015
:1032CC0008700BE00498002801D1002003900498AA
:1032DC00401E0490A0E709A90020087009A80078F6
:0832EC000AB010BD980000209B
:1032F40083B00290019102980068009002983349CB
:10330400884203D002983249884208D1009870213B
:1033140088430090019841680098084300900298FF
:103324002A49884213D00298294988420FD002982A
:10333400284988420BD002982749884207D002982E
:103344002649884203D002982549884209D1009829
:1033540003210902884300900198C168009808433A
:10336400009000988021884301994969084300909E
:10337400009802990860019880680299C8620198CF
:103384000068029988620298104988420BD002981A
:103394001149884207D002981049884203D0029804
:1033A4000F49884203D10198006902990863029980
:1033B4000120486102980069C007002804D00299DE
:1033C400086901229043086103B07047002C014052
:1033D400000400400020004000400140004401403F
:0433E400004801405C
:1033E80000B581B0009000993D22022088540098D1
:1033F8000068006A204908420BD100980068006AFA
:103408001E49084205D100980168086801229043C6
:10341800086000980AF01DFB009948220020885493
:1034280000993E220020885400993F228854009930
:103438004022885400994122885400994222885495
:103448000099432288540099442200208854009906
:103458004522885400994622885400994722885466
:1034680000993D220020885400993C22002088546D
:10347800002001B000BDC046111100004404000046
:1034880000B597B01590149113A9002008701498EE
:10349800002804D115983E21405C0F902BE0149829
:1034A800042804D115983F21405C0E9021E014981F
:1034B800082804D115984021405C0D9017E0149815
:1034C8000C2804D115984121405C0C900DE014980B
:1034D800102804D115984221405C0B9003E0159800
:1034E8004321405C0B900B980C900C980D900D9814
:1034F8000E900E980F900F9811A908701498002834
:1035080004D115984421405C0A9017E014980428C7
:1035180004D115984521405C09900DE014980828BD
:1035280004D115984621405C089003E0159847217E
:10353800405C08900898099009980A900A9810A980
:10354800087011A80078012803D110A80078012874
:1035580003D016A901200870D2E01498002804D1DD
:1035680015993E22022088542FE01498042805D18A
:1035780015993F2202208854079025E014980828BE
:1035880005D1159940220220885406901AE0149813
:103598000C2805D1159941220220885405900FE086
:1035A8001498102805D115994222022088540490B5
:1035B80004E0159943220220885404900498059049
:1035C800059806900698079007981498002804D143
:1035D800159944220220885419E01498042805D12A
:1035E800159945220220885403900FE01498082862
:1035F80005D11599462202208854029004E01599B5
:103608004722022088540290029803900398149845
:1036180001900C283AD80198810001A040588746AB
:103628005D3600089536000895360008953600087E
:103638006B36000895360008953600089536000860
:103648007936000895360008953600089536000842
:103658008736000815980168C86802221043C860B8
:1036680017E015980168C86804221043C86010E084
:1036780015980168C86808221043C86009E01598C1
:103688000168C86810221043C86002E013A901202D
:10369800087013A8007800282FD11598006814998D
:1036A800012209F0A3FA159800681749884209D041
:1036B800159800681549884204D01598006814497F
:1036C800884214D115980068806812490840129001
:1036D800129806280AD0129801210904884205D0B8
:1036E80015980168086801221043086005E01598DC
:1036F80001680868012210430860139816A9087029
:1037080016A8007817B000BD002C01400004004046
:08371800004001400700010020
:1037200000B58BB00A90099108A90020087009988B
:1037300007900C283AD80798810001A04058874686
:1037400075370008AD370008AD370008AD37000801
:1037500083370008AD370008AD370008AD370008E3
:1037600091370008AD370008AD370008AD370008C5
:103770009F3700080A980168C86802229043C86011
:1037800017E00A980168C86804229043C86010E0F6
:103790000A980168C86808229043C86009E00A983E
:1037A0000168C86810229043C86002E008A901209F
:1037B000087008A80078002871D10A980068099953
:1037C000002209F017FA0A980068006A3649084290
:1037D0000BD10A980068006A3449084205D10A985A
:1037E000016808680122904308600998002804D104
:1037F0000A993E22012088542FE00998042805D117
:103800000A993F2201208854069025E0099808284B
:1038100005D10A9940220120885405901AE00998A0
:103820000C2805D10A9941220120885404900FE008
:103830000998102805D10A99422201208854039042
:1038400004E00A99432201208854039003980490CD
:10385000049805900598069006980998002804D1C8
:103860000A9944220120885419E00998042805D1B6
:103870000A9945220120885402900FE009980828EF
:1038800005D10A99462201208854019004E00A9942
:10389000472201208854019001980290029808A8BC
:1038A00000780BB000BDC0461111000044040000B8
:1038B00000B583B0029002980068C0680190029839
:1038C00000680069009068460078800700281FD5CE
:1038D00001A80078800700281AD502980168022004
:1038E000C043086102990120087702980068806946
:1038F0008007002803D0029801F002FB05E002983F
:103900000AF0AFF802980AF0B0F8029900200877A0
:10391000684600784007002820D501A800784007B5
:1039200000281BD5029801680420C0430861029951
:10393000022008770298006880698005800F0028BF
:1039400003D0029801F0DCFA05E002980AF089F849
:1039500002980AF08AF802990020087768460078F1
:10396000000700281FD501A80078000700281AD5F5
:10397000029801680820C043086102990420087772
:1039800002980068C0698007002803D0029801F0FF
:10399000B7FA05E002980AF064F802980AF065F8B0
:1039A00002990020087768460078C006002820D5D4
:1039B00001A80078C00600281BD5029801681020D5
:1039C000C043086102990820087702980068C0691E
:1039D0008005800F002803D0029801F091FA05E0DD
:1039E00002980AF03EF802980AF03FF80299002087
:1039F000087768460078C00700280CD001A8007836
:103A0000C007002807D0029801680120C043086160
:103A100002980AF02EF8009880210840802804D0EF
:103A200068464078800600280BD501A8007800067B
:103A3000002806D5029801681D48086102980AF01E
:103A4000AAF868464078C00700280BD001A8007883
:103A50000006002806D502980168164808610298F9
:103A60000AF09DF868460078400600280CD501A8A9
:103A700000784006002807D5029801684020C0431E
:103A80000861029809F0F9FF68460078800600286E
:103A90000CD501A800788006002807D50298016897
:103AA0002020C043086102980AF071F803B000BDFD
:083AB0007FDFFFFFFFFEFFFFB7
:103AB80087B006900591049203930698006A0190D6
:103AC800069A116A01208143116206998969029157
:103AD80006991E4A914200900BD0069901201C4A73
:103AE8009142009005D006981A4940184142484131
:103AF80000900098C007002808D002980321884346
:103B08000290049902980843029003E00298012168
:103B1800084302900298F02188430290039800011C
:103B2800C1B202980843029001990A208143019189
:103B38000599014001980843019002980699886107
:103B480001980699086207B07047C046002C0140EA
:083B58000004004000C0FEBFA4
:103B600000B5F7B076900020729071A9087070903F
:103B7000769988680A6910434A691043C9690843FD
:103B800075907698416E75980843759076980068A0
:103B900000686A4908407599084376990968086081
:103BA0007698006840680321090388437699CA68BB
:103BB0001043096848607698806975907698016A24
:103BC0007598084375907698006880685C4908404D
:103BD0007599084376990968886076980068C06A84
:103BE0000F21884376994A6A10430968C86276981B
:103BF00000685449884227D153480068032108408F
:103C00006F9003281CD86F98810001A04058874608
:103C1000213C0008313C0008293C0008393C0008E0
:103C200073A9002008700EE073A9022008700AE052
:103C300073A90420087006E073A90820087002E048
:103C400073A91020087054E0769800683F498842B4
:103C50003AD13D4800680C2108406E900C282FD8BE
:103C60006E98810001A040588746C046A13C0008DC
:103C7000C13C0008C13C0008C13C0008B13C000840
:103C8000C13C0008C13C0008C13C0008A93C000838
:103C9000C13C0008C13C0008C13C0008B93C000818
:103CA00073A9002008700EE073A9022008700AE0D2
:103CB00073A90420087006E073A90820087002E0C8
:103CC00073A91020087014E0769800682049884293
:103CD00003D173A9002008700BE0769800681D4995
:103CE000884203D173A90020087002E073A9102054
:103CF00008707698C0690121C903884200D03DE26E
:103D000073A800786D90082800D918E26D9881009A
:103D100001A040588746C046593D00083F41000871
:103D2000553E00083F4100084B3F00083F41000856
:103D30003F4100083F41000847400008F369FFCFBA
:103D4000FFF4FF11003801405410024000440040CD
:103D500000480040004C0040FEF722FC6C90769832
:103D6000406A002802D101206B9065E07698406A95
:103D7000012802D102206A905CE07698406A02280D
:103D800002D10420699053E07698406A032802D15A
:103D9000062068904AE07698406A042802D10820FC
:103DA000679041E07698406A052802D10A20669023
:103DB00038E07698406A062802D10C2065902FE002
:103DC0007698406A072802D11020649026E0769801
:103DD000406A082802D1202063901DE07698406A4E
:103DE000092802D14020629014E07698406A0A289F
:103DF00002D1802061900BE07698416A01205F90AB
:103E000000020B29609001D05F98609060986190EB
:103E100061986290629863906398649064986590EA
:103E200065986690669867906798689068986990BA
:103E300069986A906A986B906C986B9907F0BCFAD5
:103E40004000769949684A08801807F0B5FA80B2B0
:103E5000729077E17698406A002802D101205E9046
:103E600065E07698406A012802D102205D905CE00E
:103E70007698406A022802D104205C9053E076983C
:103E8000406A032802D106205B904AE07698406A97
:103E9000042802D108205A9041E07698406A05280B
:103EA00002D10A20599038E07698406A062802D15B
:103EB0000C2058902FE07698406A072802D11020F5
:103EC000579026E07698406A082802D12020569024
:103ED0001DE07698406A092802D14020559014E0F0
:103EE0007698406A0A2802D1802054900BE0769898
:103EF000416A0120529000020B29539001D0529840
:103F0000539053985490549855905598569056986D
:103F10005790579858905898599059985A905A983D
:103F20005B905B985C905C985D905D985E905E990C
:103F3000A14807F041FA4000769949684A0880187C
:103F400007F03AFA80B27290FCE0FEF7A1FA5190C5
:103F50007698406A002802D10120509065E076985A
:103F6000406A012802D102204F905CE07698406AB6
:103F7000022802D104204E9053E07698406A03282C
:103F800002D106204D904AE07698406A042802D17A
:103F900008204C9041E07698406A052802D10A201A
:103FA0004B9038E07698406A062802D10C204A905F
:103FB0002FE07698406A072802D11020499026E029
:103FC0007698406A082802D1202048901DE0769813
:103FD000406A092802D14020479014E07698406A50
:103FE0000A2802D1802046900BE07698416A012091
:103FF000449000020B29459001D044984590459883
:1040000046904698479047984890489849904998D4
:104010004A904A984B904B984C904C984D904D98A4
:104020004E904E984F904F9850905198509907F05D
:10403000C3F94000769949684A08801807F0BCF92E
:1040400080B272907EE07698406A002802D101200A
:10405000439065E07698406A012802D102204290A0
:104060005CE07698406A022802D10420419053E037
:104070007698406A032802D1062040904AE076985C
:10408000406A042802D108203F9041E07698406AB7
:10409000052802D10A203E9038E07698406A06282A
:1040A00002D10C203D902FE07698406A072802D17B
:1040B00010203C9026E07698406A082802D1202003
:1040C0003B901DE07698406A092802D140203A9042
:1040D00014E07698406A0A2802D1802039900BE0DB
:1040E0007698416A0120379000020B29389001D060
:1040F000379838903898399039983A903A983B9058
:104100003B983C903C983D903D983E903E983F9027
:104110003F984090409841904198429042984390F7
:1041200043990120C00307F047F940007699496898
:104130004A08801807F040F980B2729002E071A935
:10414000012008707298102814D372A840880028A3
:1041500010D172990F20814374A8018072990E22A8
:1041600011404A08749911430180008876990968C2
:10417000C86002E071A90120087020E273A80078ED
:104180003690082800D908E23698810001A04058EE
:104190008746C046BD4100089B450008B74200085D
:1041A0009B450008AB4300089B4500089B45000861
:1041B0009B450008A54400080024F400FEF7F0F930
:1041C00035907698406A002802D10120349065E04D
:1041D0007698406A012802D1022033905CE07698FC
:1041E000406A022802D10420329053E07698406A57
:1041F000032802D1062031904AE07698406A0428CC
:1042000002D10820309041E07698406A052802D11A
:104210000A202F9038E07698406A062802D10C20B8
:104220002E902FE07698406A072802D110202D901A
:1042300026E07698406A082802D120202C901DE0C4
:104240007698406A092802D140202B9014E0769895
:10425000406A0A2802D180202A900BE07698416AB1
:104260000120289000020B29299001D0289829903C
:1042700029982A902A982B902B982C902C982D9046
:104280002D982E902E982F902F9830903098319016
:1042900031983290329833903398349035983499DD
:1042A00007F08AF8769949684A08801807F084F878
:1042B00080B2729074E17698406A002802D10120A1
:1042C000279065E07698406A012802D10220269066
:1042D0005CE07698406A022802D10420259053E0E1
:1042E0007698406A032802D1062024904AE0769806
:1042F000406A042802D10820239041E07698406A61
:10430000052802D10A20229038E07698406A0628D3
:1043100002D10C2021902FE07698406A072802D124
:104320001020209026E07698406A082802D12020AC
:104330001F901DE07698406A092802D140201E9007
:1043400014E07698406A0A2802D180201D900BE084
:104350007698416A01201B9000020B291C9001D025
:104360001B981C901C981D901D981E901E981F90C5
:104370001F98209020982190219822902298239095
:104380002398249024982590259826902698279065
:104390002799934807F010F8769949684A088018D9
:1043A00007F00AF880B27290FAE0FEF771F81A90FE
:1043B0007698406A002802D10120199065E076982D
:1043C000406A012802D1022018905CE07698406A89
:1043D000022802D10420179053E07698406A0328FF
:1043E00002D1062016904AE07698406A042802D14D
:1043F0000820159041E07698406A052802D10A20ED
:10440000149038E07698406A062802D10C20139068
:104410002FE07698406A072802D11020129026E0FB
:104420007698406A082802D1202011901DE07698E5
:10443000406A092802D14020109014E07698406A22
:104440000A2802D180200F900BE07698416A012063
:104450000D9000020B290E9001D00D980E900E9831
:104460000F900F9810901098119011981290129828
:1044700013901398149014981590159816901698F8
:10448000179017981890189819901A98199906F07B
:1044900093FF769949684A08801806F08DFF80B22C
:1044A00072907DE07698406A002802D101200C903D
:1044B00065E07698406A012802D102200B905CE00A
:1044C0007698406A022802D104200A9053E0769838
:1044D000406A032802D1062009904AE07698406A93
:1044E000042802D10820089041E07698406A052807
:1044F00002D10A20079038E07698406A062802D157
:104500000C2006902FE07698406A072802D11020F0
:10451000059026E07698406A082802D12020049071
:104520001DE07698406A092802D14020039014E0EB
:104530007698406A0A2802D1802002900BE0769893
:10454000416A0120009000020B29019001D00098DF
:1045500001900198029002980390039804900498A7
:104560000590059806900698079007980890089877
:10457000099009980A900A980B900B980C900C9946
:104580000120C00306F018FF769949684A08801890
:1045900006F012FF80B2729002E071A9012008704B
:1045A0007298102808D372A84088002804D1729805
:1045B00076990968C86002E071A9012008707699AF
:1045C0006A220120885276996822885276990020C2
:1045D000C8667699086771A8007877B000BDC046B4
:0445E0000024F400BF
:1045E40000B585B003900399882200208850FBF71A
:1045F40051FE0290039800680068000700280ED559
:104604000398029B1949009101214905002209F0F0
:10461400C8FA002803D004A90320087022E00398F4
:1046240000680068400700280ED50398029B0F49D4
:10463400009101218905002209F0B3FA002803D072
:1046440004A9032008700DE00399802220208850DB
:1046540003998422885003997C220020885404A959
:104664000020087004A8007805B000BDFFFFFF011A
:1046740084B00290019168460280029880214058DB
:10468400202800D081E00198002803D068460088E3
:10469400002803D103A90120087079E002988068FA
:1046A4000121090388420CD102980069002808D12D
:1046B40001A80078C007002803D003A901200870CE
:1046C40066E002987C21405C012803D103A9022002
:1046D40008705DE002997C220120885401980299B7
:1046E400086500980299542288520098029956222B
:1046F40088520299002008670299882288500299FA
:104704008022212088500298406E01214907884266
:104714001CD10298806801210903884207D10298BC
:104724000069002803D102991E48086702E0029933
:104734001B48086702997C2200208854029801686B
:1047440088680122D205104388601AE002988068C4
:1047540001210903884207D102980069002803D186
:1047640002990E48086702E002990B48086702990B
:104774007C22002088540298016808688022104333
:10478400086003A90020087002E003A90220087051
:1047940003A8007804B070476BD0000839480008BB
:0847A400EDCF0008AD4700084D
:1047AC0083B0029002988021405821283AD1029877
:1047BC006A21405A6946088068460088002831D032
:1047CC0002985621405A00280DD102980168886839
:1047DC000122D20590438860029801680868402243
:1047EC00104308601EE002980068C06900060028AB
:1047FC0013D50298006D0190019800880A49084071
:10480C000299096888620299086D801C08650299F2
:10481C005622885A401E8852FFE70098401E69466F
:0C482C000880C9E703B07047FF010000DE
:1048380082B00190019880214058212824D1019804
:104848005621405A00280CD1019801680868802236
:104858009043086001980168086840221043086086
:1048680012E00198006D0090009800880749084000
:104878000199096888620199086D801C0865019989
:104888005622885A401E885202B07047FF01000025
:1048980084B00290019168460280029884214058B1
:1048A800202800D0D3E00198002803D0684600886B
:1048B800002803D103A901200870CBE00298806882
:1048C8000121090388420CD102980069002808D107
:1048D80001A80078C007002803D003A901200870A8
:1048E800B8E002987C21405C012803D103A902208A
:1048F8000870AFE002997C2201208854019802993F
:104908008865009802995C228852009802995E2274
:10491800885202990020C86602988068012109031C
:1049280088420DD102980069002804D102996022BA
:104938004A48885203E002996022FF20885229E001
:104948000298806800280DD102980069002804D1D7
:1049580002996022FF20885203E0029960227F209A
:10496800885217E0029880680121090788420DD112
:1049780002980069002804D1029960227F20885299
:1049880003E0029960223F20885203E002996022E6
:104998000020885202998822002088500299842297
:1049A800222088500298026890680121084390608C
:1049B8000298406E4907884229D1684600880299C2
:1049C8006822895A884222DB0298806801210903FB
:1049D800884207D102980069002803D10299234828
:1049E800C86602E002992048C86602997C22002025
:1049F8008854029801680868012213021843086065
:104A08000298016888681207104388601BE00298C2
:104A1800806801210903884207D1029800690028AB
:104A280003D102990F48C86602E002990C48C8668B
:104A380002997C220020885402980168086809229B
:104A480052011043086003A90020087002E003A97E
:104A58000220087003A8007804B07047FF01000026
:104A68004BD10008BDD00008694B0008794A0008FE
:104A780000B587B0069006986021405A04A90880BE
:104A880006988421405822285ED106986821405A09
:104A980002A9088002A80088002835D00698006876
:104AA800406A03A908800698806D059003980499C8
:104AB8000840059908800699886D801C8865069AC3
:104AC8005E21505A401E50520698405A002816D16E
:104AD8000698016808680122120290430860069847
:104AE800016888681D4A1040886006998422202041
:104AF800885006990020C866069809F09AF8029826
:104B0800401E02A90880C5E706985E21415A01A8FF
:104B180001800088002816D001A80088069968221C
:104B2800895A88420FDA06980168886801221207B4
:104B38009043886006990848C8660698016808681E
:104B480020221043086005E0069801688869082259
:104B58001043886107B000BDBDD00008FEFFFFEF1D
:104B680000B585B0049004986021405A03A90880D4
:104B780004988421405822285CD104986821405A1E
:104B880001A9088001A80088002833D0049800688B
:104B9800406A02A908800298039908400499896D1F
:104BA80008700499886D401C8865049A5E21505AE3
:104BB800401E50520498405A002816D104980168A3
:104BC8000868012212029043086004980168886806
:104BD8001D4A104088600499842220208850049936
:104BE8000020C866049809F024F80198401E01A91D
:104BF8000880C7E704985E21415A6846018000880A
:104C0800002816D06846008804996822895A884284
:104C18000FDA0498016888680122120790438860B7
:104C280004990848C8660498016808682022104357
:104C3800086005E0049801688869082210438861C3
:0C4C480005B000BD4BD10008FEFFFFEFDF
:104C540000B585B000200190049004987F282DD8D9
:104C6400049881002348405800900020029003904B
:104C740003987F280DD8009803998A001D49895804
:104C8400884202DD0298401C02900398401C039065
:104C9400EEE70499029A164881540299405C002870
:104CA40008D10198012803D1134806F04FFCFEE710
:104CB400012001900498401C0490CEE70B49402049
:104CC40008700020049004987F280DD807480078C5
:104CD400049A0749895C884202D104980349087000
:104CE4000498401C0490EEE705B000BD9D00002030
:0C4CF4002E1400206C08002086DF000851
:104D000080B500F0B5F802490420086080BDC046B7
:044D1000101000205F
:104D140000B585B02D48006804280CD12B4901202A
:104D240008602B480021FEF7ADFB152007F000FEBC
:104D34000220049046E025480068032802D002209F
:104D440004903FE021480068032839D1152007F07A
:104D5400FAFD1F480021FEF7E1FC1C49042008600D
:104D64001C480068002806D01B48006802031B4941
:104D740008688018086017480068092806D815498B
:104D84000868401C0860022004901BE00020029088
:104D94000390104908600E480068806A401C009027
:104DA4000E48019000680A2106F004FB009B01995B
:104DB400024602985A43039208600398049001E063
:104DC40000200490049805B000BDC04610100020D7
:104DD400C40E0020BC0F002014100020D00F0020AF
:104DE40000B587B0002000900490FFF787FF00987B
:104DF400802102911B4909687F2212021140090A8D
:104E04000391049004980299884220D215490868B5
:104E14007F2212029043049A120210430860022077
:104E240006900698022803D1FFF772FF0690F8E770
:104E34000020059006990598401805900598049956
:104E44008A00094988500498401C0490DAE705490F
:104E540008687F2212029043039A120210430860EA
:0C4E640007B000BD041002406C080020E4
:104E700000B587B01E480268012149040A43026058
:104E800000680840029002981A4801901A4901608F
:104E9000FEF7AAFA01981949C16000214160016139
:104EA000816007F0C0FE002800D0FEE700220392D8
:104EB000012004900C20059006920E4803A907F0EB
:104EC000FFFE002800D0FEE70A480221002208F079
:104ED0000EFE002800D0FEE71520009000221146AB
:104EE00008F0F3FC009807F030FD07B000BDC046A5
:104EF00040100240C40E002000440140FFFF0000AB
:104F000000B583B002900298007F012863D1334836
:104F10000068012809D10298002107F03DFC3249C0
:104F200008602E490220086055E02C4800680228DD
:104F300051D102980021009107F02EFC28490191DF
:104F40000860152007F001FD00992648FEF7E8FBF0
:104F5000019802990A680221C94311610068224937
:104F60000968884215D91E4800681F490968411A16
:104F70001F480160006800031E49884208D81E4887
:104F800006F0E6FA1A48006801031C4806F0E0FA49
:104F90001EE01348006814490968884217D2124875
:104FA00001680F480068401A104941181048016014
:104FB000006800030F49884208D80F4806F0C8FA75
:104FC0000B48006801030D4806F0C2FA00E0FEE756
:104FD00002490320086003B000BDC0461010002045
:104FE000FC0F0020C40E002000100020FFFF000076
:104FF000141000203F5DC60019E400082AE40008F0
:1050000010B588B00B9C0A9C0790069105920493FA
:10501000069807990860079801684548086007984E
:1050200001684B20000248600798026801210803CC
:105030009060079802680020D060079A1268890281
:10504000116107990A680C21516107990968886103
:1050500007990968C861079909680862079909688A
:105060004862079909688862059807990968486045
:105070000498002809D10798026801208102116173
:10508000079909680003886014E0049801280AD190
:105090000798016803204002086107980168012011
:1050A0000003886006E007980168002008610799FE
:1050B000096888600A98012804D1079801680020CF
:1050C000C86004E00798016801204003C8600798A1
:1050D000006803900B9806F0E5F800220292154B49
:1050E00008F05DF906F066F8029B0146039800910E
:1050F00019461A4600F022F8002801D008F02DF9D0
:105100000798006808F09DFD002801D008F025F9F7
:1051100007990868273101221202FFF7BDFB00281A
:1051200003D0054806F014FAFEE708B010BDC046EB
:0C5130000038014000000C4089E100083C
:10513C0010B588B00A9C06900591049203930698CA
:10514C00002803D107A90120087063E0069880218C
:10515C004058002806D106997C22002088540698D5
:10516C0004F03AFE069980222420885006980168A3
:10517C0008680122904308600698FEF7EBFC0128B2
:10518C0003D107A90120087044E00698806A002822
:10519C0002D0069807F089FE06980168486801223B
:1051AC00D3051843486006980168086892061043B6
:1051BC000860069840684B21090288420BD8069873
:1051CC0000684069FF21090608400A9908430699BE
:1051DC000968486113E00698416810484843104933
:1051EC0006F0E4F8401C0190069800684069FF2125
:1051FC000906084001990843069909684861069810
:10520C00016808680122104308600698FFF7E4F96A
:10521C0007A9087007A8007808B010BDD6060000D2
:04522C0040420F00ED
:1052300010B58AB0099009980068C069089009986B
:10524000006800680790099800684068069009980F
:1052500000688068059008980F2108400490049821
:1052600000285BD005988F49084205D107A800881F
:1052700009214901084251D008A80078C007002838
:105280000DD007A84078C007002808D0099800680A
:10529000012303620999882288581843885008A876
:1052A0000078800700280ED505A80078C0070028E0
:1052B00009D0099801680220086209998822885853
:1052C00004231843885008A80078400700280ED50A
:1052D00005A80078C007002809D0099801680420B3
:1052E000086209998822885802231843885008A820
:1052F00000780007002811D507A80078800600284C
:1053000003D405986749084208D009980068082323
:1053100003620999882288581843885008A8407861
:105320000007002819D507A8C0784007002804D432
:1053300005A88078000600280FD50998026801208A
:10534000C1021162099A84232021D150099A802335
:10535000D15055490875554A885408A800788006E8
:1053600000282BD507A800788006002804D405A8BB
:10537000C078C006002821D50998842140582228E9
:1053800016D149484521C9004058FF2810D809982E
:105390000068406A44494522D2008B58CB18272424
:1053A00018558858401C8850404A0120885405E010
:1053B00009980168886908221043886108A8007864
:1053C0000006002813D507A800780006002804D49A
:1053D00005A880780006002809D5334802900068A7
:1053E00008F065FC0299232002010120885408A8D6
:1053F0000078400600280FD507A80078400600284E
:105400000AD52949262200208854099807F01FFF51
:105410000999842222208850099888214058002820
:105420003DD0099984222220885008A8007880065F
:10543000002814D507A800788006002804D405A801
:10544000C078C00600280AD5099801688869082232
:105450001043886109998822002088501FE008A81D
:105460000078000600281AD507A800780006002852
:1054700004D405A880780006002810D50A490191B7
:10548000262200208854099807F0E1FE0199099A24
:1054900084232220D05023200201012088540AB006
:1054A00010BDC04601000010380600203102000087
:1054B00085B00490039102A918480880002001904B
:1054C00001980399884225D204980199415C029879
:1054D000484002A90880082000900098002815D0B4
:1054E00002A80088C007002808D002A90888400840
:1054F000088002980A4A5040088003E002A9088800
:10550000400808800098401E0090E6E70198401C83
:105510000190D5E702A8008805B07047FFFF0000A2
:0455200001A00000E6
:1055240000B585B003900398273001900398452176
:10553400C90040580290019800780090029804280D
:1055440005D8039807F0B2FE002004901FE00198EC
:10555400029908F0E0FB401C002805D1039807F0ED
:10556400A5FE0020049012E00098002802D1022039
:1055740004900CE000980749098B884202D102206C
:10558400049004E0039807F091FE0020049004982E
:0855940005B000BDA0000020DD
:10559C0010B588B006900591049203A803700078AA
:1055AC003649098B88420BD003A80078002807D015
:1055BC000698049B06210B2207F0B0FE079059E0D9
:1055CC00059988780002C9784018029005990879E5
:1055DC0000024979401800900098002802D00098E9
:1055EC007E2807D30698049B0322114607F096FEEB
:1055FC0007903FE0029800994018401E80087728D9
:10560C0007D30698049B0321022207F087FE07901C
:10561C0030E00699049A032088540498401C0490A6
:10562C00009840000699049A88540498401C0490F1
:10563C000298019001980299009A8918884217D211
:10564C00019841000D4841184978069A049BD154A1
:10565C000499491C049101994900405C0699049AEB
:10566C0088540498401C04900198401C0190E1E778
:10567C0004980790079808B010BDC046A000002001
:10568C0000B587B0059004910392029302982C49BF
:10569C00098B88420AD00298002807D00598039BF2
:1056AC0006210B2207F03AFE069045E00499887813
:1056BC000002C9784018019001988008772807D318
:1056CC000598039B0621022207F028FE069033E082
:1056DC000498007901994A0019498A185070049865
:1056EC004079019A520088540599039A06208854EF
:1056FC000398401C03900198000A0599039A88545A
:10570C000398401C039001980599039A88540398B8
:10571C00401C0390049800790599039A88540398C7
:10572C00401C0390049840790599039A8854039877
:10573C00401C039003980690069807B000BDC04625
:04574C00A000002099
:1057500000B589B0079006910592049304984149D9
:10576000098B88420AD00498002807D00798059B27
:1057700006210B2207F0D8FD08906FE00699887883
:105780000002C97840180390069908790002497907
:1057900040180290072000900298002802D002983A
:1057A0007C2807D30798059B1021032207F0BCFD36
:1057B000089053E0039802994018401E800877280B
:1057C00007D30798059B1021022207F0ADFD089032
:1057D00044E00398019001980399029A891888423D
:1057E00015D206980099405C01994A001D498A1813
:1057F0005070069A009880184078019A5200885498
:105800000098801C00900198401C0190E3E70799E4
:10581000059A102088540598401C05900398000AAA
:105820000799059A88540598401C05900398079994
:10583000059A88540598401C05900298000A07991B
:10584000059A88540598401C059002980799059A76
:1058500088540598401C059005980890089809B050
:0858600000BDC046A0000020BD
:1058680010B586B0002101910591049103914D482E
:1058780002904D4A02600122D3074360031D8160F4
:10588800C16054050461082444610176417682763A
:10589800C4611977416281622C23C25413030363E4
:1058A8000723436383633C23C254102202642022EB
:1058B80042648164C164FAF70FFD002801D007F043
:1058C80048FD01200390002004900590354803A965
:1058D800FAF7AAFF002801D007F03BFD33480390F0
:1058E80004200490002005902E4803A9FAF79CFF95
:1058F800002801D007F02DFD2D48039008200490C2
:1059080000200590274803A9FAF78EFF002801D048
:1059180007F01FFD274803900C20049000200590F5
:10592800204803A9FAF780FF002801D007F011FDED
:10593800214803901020049000200590194803A9DD
:10594800FAF772FF002801D007F003FD1B48039007
:10595800142004901A480590124803A9FAF764FF26
:10596800002801D007F0F5FC164803901820049091
:10597800134805900B4803A9FAF756FF002801D0F1
:1059880007F0E7FC104803901C20049000200590C5
:10599800044803A9FAF748FF002801D007F0D9FC0A
:1059A80006B010BD040E00200024014002000004CF
:1059B800040000080800000C10000010000100207E
:0C59C80004FFFF07000200240004002878
:1059D40030B593B012900020119010900F900E905B
:1059E4000D90129800684F49884200D098E04E48C4
:1059F4000268012109050A430260006808400C900E
:105A04000C984A48026801210A4302600068084071
:105A14000B900B984548026802210A430260006813
:105A240008400A900A98012007900D9003200390E3
:105A34000E90002008900F90052006900007049017
:105A44000DA90591FBF76EFF039B04980599089A2D
:105A540002250D950E930F92FBF764FF039B0498A8
:105A64000599089A04240D940E930F92FBF75AFF9C
:105A7400039A0599079B08980D930E920F902C4852
:105A84000290FBF74FFF0298039B0599089A0D9526
:105A94000E930F92FBF746FF0298039B0599089A11
:105AA4000D940E930F92FBF73DFF039B0498059909
:105AB400089A08240D940E930F92FBF733FF039B6F
:105AC40004980599089A10240D940E930F92FBF7ED
:105AD40029FF069B079A089916480990164C0460FA
:105AE40043608160C1608023036113024361D20279
:105AF40082612022C2610162FBF7B6FA002801D05C
:105B040007F029FC12980B490165129888620C2051
:105B140001900022114607F0D6FE019806F008FF16
:105B240013B030BD00240140401002403410024044
:0C5B340000040050680E00200800024031
:105B400030B58DB00C900BA8099001700AAC089488
:105B50002220019020700520000707900121069166
:105B6000C90305910022029207F031FF0C980A2127
:105B7000039100910323049321462246FDF702F985
:105B80000599069A079807F022FF029A0798059947
:105B9000A37807252B400B9D2B4363704223237072
:105BA00007F015FF03990C98009102232146224625
:105BB000FDF7E8F80599069A079807F008FF019B9A
:105BC000029A07980599237007F001FF0399049B37
:105BD000089A0C9800911146FDF7D4F80599069A99
:105BE000079807F0F4FE089909988A780178084622
:105BF0001040884203D0034805F0AAFCFEE70DB030
:085C000030BDC0461BE60008A0
:105C080000B581B0009000983121C9004058009932
:105C180088670098CE21405A00997C2288520098C3
:105C2800CC21405A00997E2288520098D4214058AD
:105C38000099802288500348002102F025F901B01C
:085C480000BDC046A0000020D1
:105C500000B585B004900498D4214058049A84215A
:105C6000505004984058049980228958401A039053
:105C70000A480068029002997D20C00048430399B9
:105C800005F072FB0190019804998822885004481D
:105C9000002102F0FDF805B000BDC046D40F002081
:045CA000A000002040
:105CA40000B585B00F490191CC200A5A8C200A52C4
:105CB400085E7E22895E401A04900B4800680390B7
:105CC40003997D20C0004843049905F04BFB01462D
:105CD40001980291029990228150002102F0D6F895
:0C5CE40005B000BDA0000020DC0F002077
:105CF00000B58DB00C90424805F02AFC0C989C2110
:105D00004058002803D14A4805F022FC75E00C9861
:105D10009C210291405805F089FA00220992394BE2
:105D2000039305F0F5F8384B01931A685B6805F0AA
:105D3000EFF8099A0B910A900A980B99334B089344
:105D400007F02DFB05F0E2F9014601980C9A942327
:105D50000793D1500C99CE22895A0C9A9823049318
:105D6000D1520C99CC22895A0C9A9A230593D1527C
:105D700043680268264805F0EBFB02990C984058EE
:105D800005F054FA039B099A05F0C2F802460B4647
:105D9000204805F0DDFB04990C98405E05F046FABA
:105DA000099A1D4B069305F0B3F802460B461B48B3
:105DB00005F0CEFB05990C98405E05F037FA069B7E
:105DC000099A05F0A5F802460B46154805F0C0FBF8
:105DD00007990C98405805F029FA089B099A07F092
:105DE000DEFA02460B460F4805F0B2FB0E4805F0FE
:105DF000AFFB09990D4802F04BF80DB000BDC0464D
:105E000097E1000800408F401006002080842E415A
:105E100043E400089DDF000800005940ACDF0008A3
:105E200003E2000837E600080DE20008A0000020A9
:045E3000A9E10008DC
:105E340000B58FB04A4805F089FB4A480A90CE2144
:105E44000191425AA0214252405E05F0EDF9002230
:105E54000992454B079305F059F802460B4643480F
:105E640005F074FB0A990198085E9822895E401A2D
:105E74000B900B9805F0D8F9079B099A05F046F8A2
:105E840002460B463A4805F061FB3A48016842680D
:105E94000D920C9143680268374805F057FB0A9845
:105EA4009C210291405805F0BFF9099A334B0393A2
:105EB40005F02CF802460B46314805F047FB0299E1
:105EC4000A98405805F0B0F9039B099A05F01EF8AA
:105ED4000C9A0D9B05F01AF8099A0D910C900C98E8
:105EE4000D99284B089305F009F80D910C900C9826
:105EF40004900D9805900B9805F096F902460498C5
:105F04000B46059905F002F8099A0D910C900C982E
:105F14000D991D4B069307F040FA05F0F5F802467B
:105F24000A98A4214250405805F07EF9069B099A2C
:105F340004F0ECFF079B099A07F02FFA089B099AD3
:105F440004F0F8FE02460B46104805F0FFFA10482C
:105F540005F0FCFA09990A9801F098FF0FB000BD0A
:105F6400B7DF0008A000002000005940CEDF000881
:105F740023E2000800060020DDDF000800408F4017
:105F840031E200080000F03F65CDCD4110E000088B
:045F94004BE60008D0
:105F980000B58DB00AA90020059008810B90472113
:105FA8000A912A49099108700520000702900122E8
:105FB80001921103039107F006FD96200890FAF765
:105FC8006DF9059A224800902021069107F0FBFC04
:105FD8000898FAF763F90098019A069907F0F3FC14
:105FE8000898FAF75BF902980399059A07F0EBFC11
:105FF800059A07200490022107F063FC049806F034
:1060080095FC1448079000F027F80898FAF746F925
:1060180006990798FFF790FD0599079800F060F832
:106028000699079800F0C0F80798342100F020F985
:1060380000F066F900F072FA0898FAF72FF9099952
:106048000320087007F0EDFE0DB000BDBE1400205F
:0860580000040050A00D00201F
:1060600010B58AB0099008AC079400220292A27081
:106070001B48208005200007069001210591C903D7
:10608000049107F0A4FC09980A21039100910223CE
:1060900021462246FCF776FE0499059A069807F0F9
:1060A00096FC029A069804992623237007F08FFC29
:1060B0000399079A0998009103231146FCF762FEA1
:1060C0000499059A069807F082FC079880780A28B8
:1060D00003D0044805F03CFAFEE70AB010BDC04604
:0860E000460A000060E400081C
:1060E80030B58DB00C900BA8099001700AAC0894DB
:1060F80023200190207005200007079001210691B8
:10610800C90305910022029207F05DFC0C980A2150
:10611800039100910323049321462246FCF72EFEA7
:106128000599069A079807F04EFC029A0798059970
:10613800A378EF252B400B9D2B43637043232370DB
:1061480007F041FC03990C9800910223214622464E
:10615800FCF714FE0599069A079807F034FC019B92
:10616800029A07980599237007F02DFC0399049B60
:10617800089A0C9800911146FCF700FE0599069ABA
:10618800079807F020FC089909988A78017808464A
:106198001040884203D0034805F0D6F9FEE70DB059
:0861A80030BDC0463BE20008D7
:1061B00030B58DB00C900BA8099001700AAC089412
:1061C00023200190207005200007079001210691EF
:1061D000C90305910022029207F0F9FB0C980A21ED
:1061E000039100910323049321462246FCF7CAFD44
:1061F0000599069A079807F0EAFB029A079805990D
:10620000A3789F252B400B9D2B4363704323237062
:1062100007F0DDFB03990C980091022321462246EA
:10622000FCF7B0FD0599069A079807F0D0FB019B93
:10623000029A07980599237007F0C9FB0399049BFC
:10624000089A0C9800911146FCF79CFD0599069A56
:10625000079807F0BCFB089909988A7801780846E6
:106260001040884203D0034805F072F9FEE70DB0F4
:0862700030BDC04667E60008DE
:1062780010B58CB00B900AA80890017009AC07946F
:10628800512020700A98607000220292A2700520A6
:106298000007069001210591C903049107F093FBBB
:1062A8000B980A2103910091022321462246FCF70C
:1062B80065FD0499059A069807F085FB029A0698E9
:1062C80004993123237007F07EFB0399079A0B98F2
:1062D800009103231146FCF751FD0499059A06988D
:1062E80007F071FB0798089980780978884202D0EE
:1062F800024805F029F90CB010BDC04633E000088B
:1063080000B5A3B005202290002021901F901F986F
:10631800042834DC1EA90E9100228A707C4808806B
:106328001DA812908270028005200007119001219B
:106338001091C9030F9107F046FB0E99129A0A2093
:10634800009074480323FCF719FD0F99109A1198CF
:1063580007F039FB12980078FF280CD11DA8407867
:106368001EA90978884206D11DA8807820A908703E
:106378000120219003E01F98401C1F90C7E7219837
:10638800002809D1052000070121C90207F02FFBC9
:10639800C820F9F783FFF5E720986021084320A972
:1063A800087000201C901B901B98042830DC1AA948
:1063B8000991452008702098487019A80D9000226E
:1063C8000280052000070C9001210B91C9030A9156
:1063D80007F0F9FA09990D9A0A2000904D4802230E
:1063E800FCF7CCFC0A990B9A0C9807F0ECFA0D987C
:1063F8000078FF2808D119A840781AA90978884296
:1064080002D101201C9003E01B98401C1B90CBE795
:106418001C98002809D1052000070121C90207F0AE
:10642800E6FAFA20F9F73AFFF5E7002018901790F6
:10643800179804285CDC15A9049100200390888033
:10644800334815903448022206F0B3FA039A0499A7
:10645800887013A80890828013920520000707907F
:1064680001210691C903059107F0ADFA0499089A2C
:106478000A20009027480623FCF780FC0599069A15
:10648800079807F0A0FA08980078FF282BD113A8DE
:10649800407815A90978884225D113A8807815A9CC
:1064A800497888421FD113A8C07815A989788842ED
:1064B80019D113A841790291011D1748012206F04C
:1064C80078FA0146029888420DD113A8007940064F
:1064D800002807D513A800798006002802D50120D6
:1064E800189005E000E0FFE71798401C17909FE719
:1064F800189800280AD1052000070121C90207F0D1
:1065080076FA4B208000F9F7C9FEF4E723B000BD06
:0C65180025EC0000A00D00203C0F00202E
:1065240000B599B005201890002017901690169881
:1065340004283FDC5E4815905E4815A908910222A4
:1065440006F039FA08998870002214920520000791
:106554000B9001210A91C903099107F036FA0899B1
:106564000A200090544814AA0C920423FCF708FC57
:1065740009990A9A0B9807F028FA0C980078FF28D2
:1065840014D114A8407815A9097888420ED114A80A
:10659400807815A94978884208D114A8C07815A92B
:1065A4008978884202D10120179003E01698401C94
:1065B4001690BCE7179800280AD10520000701218E
:1065C400C90207F016FAAF204000F9F769FEF4E7B4
:1065D4000020139012901298042859DC10A90391FA
:1065E400002002908880354810903248022206F03C
:1065F400E2F9029A039988700EA8079082800E929D
:1066040005200007069001210591C903049107F0B4
:10661400DCF90399079A0A20009027480623FCF71F
:10662400AFFB0499059A069807F0CFF9079800780C
:10663400FF2828D10EA8407810A90978884222D1D1
:106644000EA8807810A9497888421CD10EA8C07879
:1066540010A98978884216D10EA841790191011DAB
:106664001448012206F0A7F90146019888420AD18C
:106674000F990DA8017000780006002802D50120AA
:10668400139005E000E0FFE71298401C1290A2E787
:10669400139800280AD1052000070121C90207F038
:1066A400A8F919200001F9F7FBFDF4E719B000BDC2
:1066B400F2EC00003C0F0020A00D002021EC0000B3
:1066C40000B591B00DA903910020029008720E90BC
:1066D40047480D904748022206F06DF9029A039943
:1066E40088700AA8079002720B920A9209920520F8
:1066F4000007069001210591C903049107F065F98B
:106704000399079A0A2000903B480923FCF738FBB9
:106714000499059A069807F058F907980078FF2815
:1067240058D10AA840780DA90978884252D10AA8FC
:1067340080780DA9497888424CD10AA8C0780DA95F
:106744008978884246D10AA8017A0191011D294815
:10675400042206F030F90146019888423AD10B9997
:1067640008A801700078000600282AD508A8007837
:106774004007002825D508A800784006002820D422
:1067840008A80078000700281BD410A90020C870AE
:106794000AA842798A7082794A70C0790870109880
:1067A400C00D002806D01098154940181090109874
:1067B400099005E01098C00D002801D110980990A7
:1067C40007E00E49C1204200885A401C8852FFF756
:1067D400E1FB07E00949C1204200885A401C885265
:1067E400FFF7D8FB099800F00DF811B000BDC046C2
:1067F40012EC00003C0F0020A00D0020A00000209F
:04680400010000FF90
:1068080010B59CB01B908A4800688A49884203D01A
:1068180087490868401C086087480168CA0F8A18B9
:106828005210891A01601B9A016889180160006872
:10683800C10F401840101A901A9980480A903122C6
:10684800D20081500146C83109911A9A836FD21A31
:106858007B4B01931A60C96880228258891A199162
:10686800199988228058484304F0DCFC00220D92D4
:10687800744B059304F048FB04F044FC019A0A9910
:10688800034609981893189B6324A4000B511268B7
:10689800189BD21A6C4B06931A600422805E7E22E3
:1068A800895E401A04F0BEFC02460A9802920A4623
:1068B80002991792169117990491169903919021AC
:1068C800405804F0AFFC024603980B46049906F0C2
:1068D80062FD059B0D9A04F017FB04F013FC0146BA
:1068E8000698159100681599411A58480160006882
:1068F80004F098FC0D9A564B06F04DFD0D9A554B39
:1069080006F049FD0D9A544B04F0FEFA02460A9827
:106918000B4652494B600A604A6808920968079119
:106928009421405804F07EFC0D9A4D4B04F0ECFA8B
:10693800024607980B46089906F02DFD024609986D
:106948000C460A99474B0C935C601A600622805EDD
:106958009822895E401A04F065FC02460A980B9258
:106968000A460B9913921291A421405804F05AFC3C
:106978000D9A3D4B04F0C8FA119110901298139992
:10698800109A119B06F007FD0D9A384B04F0D0F9C8
:106998000A460C990F920E90086849680E9A0F9B48
:1069A80006F0F9FC0D9A0B4631494B6008600868FF
:1069B8004968304B04F066FB002808D12C49086868
:1069C800496800222C4B04F07DFB002806D01B49A7
:1069D800192000010858E42288500BE0244908686F
:1069E80049680022174B06F0D6FC04F08BFB1349CC
:1069F800E42288500E480068152813DB0F49C83177
:106A0800C869096A884203DD0C49C831C869086247
:106A18000A49C831C869496A884203DA0749C8314E
:106A2800C869486215490120086000201CB010BDE3
:106A380020100020FFFFFF7F24100020A00000206E
:106A4800D40F002000408F40DC0F0020D80F00201A
:106A58000000084000004940000060411006002086
:106A680080842E410006002065CDCD410000F03F16
:106A78000806002000206140002061C0B40F0020FB
:106A88000649C86D4042E12213014343D817052245
:106A980092018B50891848607047C046A0000020BA
:106AA80000B585B00D480190C06DE1210A010023B1
:106AB8000093194604F03CFC009B0A460199039296
:106AC8000290F8200858F8314968054A04F030FC6B
:106AD800029A039B04F090FC05B000BDA0000020C2
:046AE800A086010083
:106AEC0000B58DB000200B9031480A9031482D2113
:106AFC00C9004058002806D52E482D21C900405801
:106B0C004042059001E0002005900599C8170891B6
:106B1C000990002007900690264843218900405890
:106B2C00002815DC08980999214A04920023039344
:106B3C0004F0FCFB039B1F4AD26D04F05BFC034684
:106B4C0003980A460499C91A90410691079016E0D9
:106B5C0008980999164A02920023019304F0E6FB67
:106B6C00144A43239B00D258D31704F043FC03462A
:106B7C0001980A460299C91A904106910790079804
:106B8C00069A00210C4BD21A884104DB0020079096
:106B9C000748069008E00799069A0020524288415F
:106BAC0002DB00200790069006980DB000BDC04691
:0C6BBC00A0860100A0000020A1860100BE
:106BC80010B5A8B0002316932793269325932493F2
:106BD80023932293219320931F931E931D931C9319
:106BE8001B931A93EE48C06DE1210A01194604F07F
:106BF8009FFB19911890EB484168006808430028EA
:106C080009D1FE484B2189004158FE484843FC49B8
:106C180000224A600860FC48416800680843002870
:106C280009D1F648132109014158F6484843F64965
:106C380000224A600860F148E421405800281ED428
:106C4800EE4813905221405A04F0ECFA0022EF4B20
:106C580004F05AF90246139814920A4614991F929E
:106C68001E91C8301590C06904F0DCFA1E9A1F9B6B
:106C780006F091FB04F046FA1599886259E0DF495D
:106C88001291C86D6822895A04F092FB0146129845
:106C98001791E421405817994942884245DAD74864
:106CA8000E90C8301190C06904F0BCFA2591249068
:106CB80024980C9025980D90179804F0B3FA024682
:106CC8000C980B460D9904F01FF902460E980F9286
:106CD8000A460F992792269127990122D2075140F7
:106CE80027915021405A04F09DFA00221092C74B78
:106CF80004F00AF9109A2391229022982399C44B00
:106D080004F016F802460B462799269803F0B2FEBF
:106D18002191209024982599209A219B06F03BFBED
:106D280004F0F0F91199886203E0B449C831C869E0
:106D38008862B2487021425EC830816A891A8162CD
:106D4800C069002823D5AD480B90C8300A90C069A7
:106D58004442E317AA4948680A68121958410A6068
:106D6800486008684968A74A002304F05DFB0B994E
:106D780002460A984266426E7D20C0005043C96DA3
:106D880004F016FB0B994F229200885213E09B489F
:106D9800C8300990C469E3179B4948680A68121902
:106DA80058410A60486008684968964A002304F018
:106DB8003BFB0999886691490791C83108918C6A0B
:106DC800E317486B0A6B121958410A6348638C6AC7
:106DD800E317C86F8A6F121958418A67C867886FA6
:106DE800C96FE1221201002304F006FB079A01464D
:106DF80008982D23DB00D150416B036B1998189A22
:106E0800D21A884106DA1998189A7C49F823CA5088
:106E1800F8314860794905208201881840688A5805
:106E28000021521E884106DB74490520820100209A
:106E380088508918486071480690C16D5422805A5C
:106E4800484304F02BFA0022704B04F05DF804F07C
:106E580073F90A4606991B921A90D82008585822A6
:106E6800895A88420DDD6548E4214258D0171B999C
:106E78001A9BD21A884104DA66490888401C08809F
:106E880002E064490020088000216248405E5B49B6
:106E98005622895A88420DDD1898199A5749C831DF
:106EA8004A6308630020C867886703F08BFA5A4969
:106EB8000120086051490491C8310591086B496B5C
:106EC800E1221201002304F097FA0499024605987A
:106ED800C26200690322D201895A884247DA4748C8
:106EE800D82140584D49884241DB4D480188491C0A
:106EF800018000880A2839DB47480068012835D115
:106F080047490A2008803D4809214901405800099D
:106F1800E12826D339480921490140584149884286
:106F28001FD836482D21C9004058002805D43348B9
:106F38002D21C9004058039005E030482D21C90093
:106F480040584042039003982C49029143229200F2
:106F5800885003F0ADF802982F4A0021116000F024
:106F680093FF2649492082000020885002E02C49DE
:106F78000020088021486421405A0190042836D80E
:106F88000198810001A040588746C046B16F0008AB
:106F9800BF6F0008CD6F0008DB6F0008E96F0008BD
:106FA800A000002028060020FFF77AFD13490122DF
:106FB8001202885020E0FFF795FD104901221202C5
:106FC800885019E003F0DAF80C49012212028850BF
:106FD80012E003F00BF909490122120288500BE074
:106FE80003F072F9054901221202885004E00349AE
:106FF800012002020020885028B010BDA000002007
:107008002806002080EE3600300600200000594097
:107018000000F0BF2C100020B00F0020E903000092
:087028002A10002080FC0A0080
:1070300000B587B00690314800683149884203D0D6
:107040002E490868401C08602E4801680A0A891AFF
:107050000160069A0168891801600068000A0590BD
:1070600005982949C83104914A8800230393194699
:1070700004F062F9039B062204F05EF904F020F9A3
:10708000039A224B03F044FF04F040F8049908618E
:107090001A4800681E49884213DB1B49C831086939
:1070A0004969884203DD1849C831086948611649B1
:1070B000C83108698969884203DA1349C831086907
:1070C0008861069810490291CA228A5A00230193C6
:1070D000194604F031F9019B062204F02DF904F061
:1070E000EFF8019A094B03F013FF04F00FF802992F
:1070F00065229200885007B000BDC04618100020DD
:10710000FFFFFF7F1C100020A00000200000244192
:04711000010A000070
:1071140000B583B00948026801210A43026000688F
:10712400084002900298092001900121002206F0F3
:10713400CAFB019805F0FCFB03B000BD3810024007
:1071440000B583B001901E48007880021D494018A4
:107154006946012200F03EF8002803D002A903206A
:10716400087029E00198002802D00098019908705D
:1071740068460078FF2806D1154804F0E7F902A90B
:107184000020087018E068460078392806D10F48B6
:1071940004F0DCF902A9012008700DE068460078CB
:1071A400382806D1084804F0D1F902A90220087051
:1071B40002E002A90320087002A8007803B000BD11
:1071C400E075FF1F00F8FF0783E600085DE2000892
:0471D40052E000087D
:1071D80086B00490039102920498029940181149CC
:1071E800097889020122D2068918884203D905A99B
:1071F8000120087011E00020009000980299884250
:1072080008D20498009A805C039988540098401C1E
:107218000090F2E705A90020087005A8007806B0DC
:087228007047C046E075FF1F2E
:10723000F0B587B006908E4804F08AF98D48059025
:1072400005994B20000288610599002000908883F1
:1072500005990122CA8305990A84059948850599EB
:1072600088850599C88505990886059948860599F0
:1072700088860599C886059988630599C863059924
:10728000086405994864059B7B4999640599C8641D
:107290000599086505994865059B78499965059B99
:1072A000802463211953059B822469211953059B6E
:1072B000842473491951059B882472491951059BEF
:1072C0008C240A211953059B8E2402211953059CF5
:1072D00090256D4B6353059C92256C4B6353059B26
:1072E00094241A55059A9623D152059BAF229201F8
:1072F00098241A53059B9A24654A1A53059B9C248B
:10730000644A1A53059B9E24634A1A53059BA02482
:10731000624A1A53059BA2247D2201921A53059AB0
:10732000A4235F4DD552059AA6235E4CD452059AEC
:10733000A8265D4B9353059EAA275C4AF253059EEF
:10734000AC27F553059DAE26AC53059CB025635381
:10735000059BB2241A53059BB42432221A53059B71
:10736000B624534A1A53059BB824524A1A53059B14
:10737000BA2407221A53059ABC23D050059AC02379
:10738000D050059AC423D050059AC823D050059BED
:10739000CC245A221A53059AD023D050059A50660D
:1073A0001066059BC2439A66059BDA66059B5A6781
:1073B000414A1A67059AC943D16740499167059ABE
:1073C0009168491C9160059AD82191800599C880DF
:1073D000059939200870FAF791F80198C000FAF77A
:1073E00023F837480068C007002804D034490868EB
:1073F0000122904308603348022101603249097834
:107400004908491E81600121C16004A9FAF7F6F814
:10741000002800D0FEE72C48007880022B49401855
:107420000390002002900398274909788902284A8E
:107430008918884214D203990298C3000D4AD018C3
:10744000D25843680120F9F7A3FF002806D103981A
:10745000083003900298401C029000E0FEE7E2E74B
:10746000FAF76EF8069800F035F807B0F0BDC046A0
:107470008BE200085804002090D0030040420F0027
:10748000A086010080482800B0360000302C0000A3
:10749000E02E000060EA0000C0DA000083FF000078
:1074A0004C1D0000581B000054F2000048F400007E
:1074B00038FF00001027000000D68AEA007884C94F
:1074C000142002409C0F0020E075FF1F00F8FF070A
:0474D000D4F8FF07E6
:1074D400F0B58BB00990CB4800788002CA494018B7
:1074E400CA49D822FFF776FE002803D00AA9012052
:1074F400087082E1C5480890089880690999086174
:107504000898808B099988820898C08B0999C88249
:107514000898008C099908830898408C09998883F5
:107524000898808C0999C8830898C08C09990884A4
:107534000898008D099948840898408D09997C22FF
:1075440088520898808D09997E2288520898C08DA7
:1075540009999827C8530898008E09999A26885340
:107564000898408E09998C22039288520898808E3C
:107574000999A02408530898C08E0999A822069254
:1075840088520898806B0999802200928850089844
:10759400C06B09998422029288500898006C09995A
:1075A4008822019288500898406C0999902204928C
:1075B40088500898806C09999C2548510898C06C9B
:1075C4000999A423C8500898006D0999AC22079220
:1075D40088500898406D099988670898806D099AC1
:1075E40094210591505000990898405A09995222C3
:1075F400885208988221405A099950228852019A47
:107604000299089840580999C865039908988058C0
:10761400099A10660898405A099954228852089881
:107624008E21405A099A5621505204990898405A7A
:1076340009995822885208989221405A099A5A2145
:10764400505205990898405C099964228852089818
:107654009621405A099968228852069A07990898EF
:10766400C05B099FB8860898805B099EF0860898DD
:10767400405B099D288708989E25405B099D688783
:107684000898005B099CA0870898A224005B099CC9
:10769400E0870898C05A099B402418530898A623E9
:1076A400C05A099B422418530898805A099A4423C3
:1076B400D0520898AA22805A099A4623D052089890
:1076C400405A0999482288520898AE21405A09998B
:1076D4004A2288520898B021405A09994C2288526B
:1076E4000898B221405A09994E2288520898B42128
:1076F400405A09996A2288520898B621405A099931
:107704006C2288520898B821405A09996E228852EE
:107714000898BA21405A0999702288520898BC21C5
:10772400405809994B22920088500898C02140582B
:1077340009991322120188500898C42140580999C4
:107744004D22920088500898C82140580999272250
:10775400D20088500898CC21405A09997222885244
:107764000898D021405809992522D20088500899B8
:10777400486E0A6E099B1946F831F8241A5148607C
:107784000898806E09994322920088500898C06E28
:1077940009991122120188500899486F0A6F099BB0
:1077A40005218C0119191A5148600899C86F8A6F0C
:1077B400099B2921CC0019191A5148600898C068FE
:1077C4000999486008988088D82803D00AA901201C
:1077D400087012E00898C088002803D00AA9012084
:1077E40008700AE008980078392803D00AA9012013
:1077F400087002E00AA9002008700AA800780BB0FB
:10780400F0BDC046E075FF1F00F8FF0758040020D4
:1078140000B5B3B031903091F84803F097FEF848C2
:1078240000788002F7494018F749D022FFF7D2FCCC
:10783400002803D032A90120087003E3F2482F90F6
:10784400F2482E902F98406D2E9948652F98408DC0
:107854002E9948852F98808D2E9988852F98806B36
:107864002E9988632F98C06B2E99C8632F98006C4B
:107874002E9908642F98408E2E9948862F98406C34
:107884002E9948642F98806D2E9988652F98C08D05
:107894002E99C8852F98008E2E9908862F98806C73
:1078A4002E9988642F98808E2E9988862F98C06C84
:1078B4002E99C8642F98C08E2E99C8862F98006D73
:1078C4002E9908653098012803D14B2000022A9094
:1078D40002E02F9880692A902A982E99886130981E
:1078E400012802D10020299002E02F98808B299052
:1078F40029982E9988833098012802D10120289054
:1079040002E02F98C08B289028982E99C88330982D
:10791400012802D10120279002E02F98008C2790A3
:1079240027982E9908843098012802D100202690A7
:1079340002E02F98408C269026982E9948843098FF
:10794400012802D10020259002E02F98808C2590F8
:1079540025982E9988843098012802D100202490FB
:1079640002E02F98C08C249024982E99C8843098D3
:10797400012802D10020239002E02F98008D23904B
:1079840023982E9908853098012802D163202290EB
:1079940003E02F987821405A229022982E99802231
:1079A40088523098012802D19948219002E02F98FA
:1079B400C06F219021982E998422885030980128F4
:1079C40002D19448209003E02F98802140582090C1
:1079D40020982E99882288503098012802D10A20B4
:1079E4001F9003E02F988421405A1F901F982E99CE
:1079F4008C2288523098012802D169201E9003E01D
:107A04002F987A21405A1E901E982E9982228852CD
:107A14003098012802D102201D9003E02F9886217E
:107A2400405A1D901D982E998E2288523098012814
:107A340002D179481C9003E02F988821405A1C9069
:107A44001C982E99902288523098012802D17348AC
:107A54001B9003E02F988A21405A1B901B982E9963
:107A6400922288523098012802D101201A9003E012
:107A74002F988C21405C1A901A982E99942288543D
:107A84003098012802D10220199003E02F988E210A
:107A9400405A199019982E999622885230980128A4
:107AA40003D1AF208001189003E02F989021405A11
:107AB400189018982E99982288523098012802D14B
:107AC400E548179003E02F989221405A1790179891
:107AD4002E999A2288523098012802D1DF481690B4
:107AE40003E02F989421405A169016982E999C22C0
:107AF40088523098012802D1D948159003E02F9874
:107B04009621405A159015982E999E2288523098A5
:107B1400012803D17C20C043149003E02F989821BE
:107B2400405E149014982E99A0228852309801280F
:107B340002D17D20139003E02F989A21405E139088
:107B440013982E99A22288523098012802D1C54850
:107B5400129003E02F989C21405E129012982E9967
:107B6400A42288523098012802D1BF48119003E022
:107B74002F989E21405E119011982E99A62288522A
:107B84003098012802D1B948109003E02F989E2123
:107B9400405E109010982E99A8228852309801289F
:107BA40002D1B3480F9003E02F98A221405E0F90BA
:107BB4000F982E99AA2288523098012802D1A948F8
:107BC4000E9003E02F98A421405E0E900E982E99FB
:107BD400AC2288523098012802D1A3480D9003E0CA
:107BE4002F98A621405E0D900D982E99AE228852B2
:107BF4003098012814D19D480C9015E0CBE600087C
:107C0400E075FF1F00F8FF0730050020580400202E
:107C1400A086010080482800B0360000302C000007
:107C24002F98A821405E0C900C982E99B02288526F
:107C34003098012802D18E480B9003E02F98AA2196
:107C4400405E0B900B982E99B222885230980128EE
:107C540002D132200A9003E02F98AC21405E0A90B2
:107C64000A982E99B42288523098012803D1C7204B
:107C7400C043099003E02F98AE21405E0990099813
:107C84002E99B62288523098012802D1794808905A
:107C940003E02F98B021405A089008982E99B822F2
:107CA40088523098012802D10720079003E02F98CA
:107CB400B221405E079007982E99BA2288523098D4
:107CC400012802D10020069003E02F98B4214058E7
:107CD400069006982E99BC2288503098012802D12B
:107CE4000020059003E02F98B8214058059005988E
:107CF4002E99C02288503098012802D15A2004902D
:107D040003E02F98C421405A049004982E99CC2261
:107D140088523098012802D10020039003E02F9864
:107D2400C8214058039003982E99D02288502E9948
:107D34000020486608662E9AC14391662E9AD16641
:107D44002E9A51674C4911672E9A0221C943D16773
:107D54004A4991672E99C42288502E99C822885086
:107D64002F9A9168491C91602E9A91602E9AD8217D
:107D740091802E99C8802E99392008703098012856
:107D840002D10020029002E02F98007C0290029819
:107D94002E9908743098012802D10020019002E045
:107DA4002F98C068019001982E99C860F9F7A4FB38
:107DB4007D20C000F9F736FB31480068C007002871
:107DC40004D02F4908680122904308602D480221FD
:107DD40001601E4909784908491E81600121C1607A
:107DE4002DA9F9F709FC002800D0FEE71748007810
:107DF4008002174940182C9000202B902C9813498E
:107E040009788902204A8918884214D22C992B981F
:107E1400C300104AD018D25843680120F9F7B6FAC3
:107E2400002806D12C9808302C902B98401C2B90BD
:107E340000E0FEE7E2E7F9F781FB3198FFF748FB42
:107E440032A9087032A8007833B000BDE075FF1F76
:107E540000F8FF0758040020E02E000060EA00004C
:107E6400C0DA00004C1D0000581B000054F2FFFF54
:107E740048F4FFFF1027000000D68AEA007884C97E
:0C7E8400142002409C0F0020D4F8FF07DF
:107E9000F0B58FB00E900DA808900170E44803F083
:107EA00057FBE4480C900E9800690C9988610E9875
:107EB000808A0C9988830E98C08A0C99C8830E9882
:107EC000008B0C9908840E98808B0C9948840E982E
:107ED000C08B0C9988840E98008C0C99C8840E98DD
:107EE000408C0C9908850E987E21405A0C99888503
:107EF0000E987C21405A0C9948850E98982106913D
:107F0000405A0C99C8850E989A210791405A0C99AD
:107F100008860E988C210391405A0C9948860E9839
:107F2000A026805B0C9988860E98A824005B0C998B
:107F3000C8860E98802280580C9988630E988421F8
:107F4000019140580C99C8630E98882102914058BD
:107F50000C9908640E989021049140580C9948643B
:107F60000E989C27C0590C9988640E98A4254059F6
:107F70000C99C8640E98AC23C0580C9908650E98EB
:107F8000806F0C9948650E989421059140580C9982
:107F900088650E985221405A0C9988520E985021AB
:107FA000405A0C9982228852019A0E98C06D0C9901
:107FB0008850029A0E98006E0C998850039A0E9879
:107FC0005421405A0C9988520E985621405A0C99C7
:107FD0008E228852049A0E985821405A0C99885241
:107FE0000E985A21405A0C9992228852059A0E985E
:107FF0006421405A0C9988540E986821415A0C9A71
:108000009620115206980E99898E0C9A1152079853
:108010000E99C98E0C9A115208980E99098F0C9AD4
:10802000D1530E99498F0C9A9E27D1530E99898F5F
:108030000C9A91530E99C98F0C9AA22691530E99BE
:108040004022895A0C9A51530E994222895A0C9A0D
:10805000A62551530E994422895A0C9A11530E9910
:108060004622895A0C9AAA2411530E994822895AF9
:108070000C9AD1520E994A22895A0C9AAE23D152A7
:108080000E994C22895A0C9AB023D1520E994E2245
:10809000895A0C9AB223D1520E996A22895A0C9AA3
:1080A000B423D1520E996C22895A0C9AB623D1521C
:1080B0000E996E22895A0C9AB823D1520E997022C9
:1080C000895A0C9ABA23D1520E994B2292008958A0
:1080D0000C9ABC23D1500E991322120189580C9A84
:1080E000C023D1500E994D22920089580C9AC42376
:1080F000D1500E992722D20089580C9AC823D1500A
:108100000E997222895A0C9ACC23D1520E992522AB
:10811000D20089580C9AD023D1500E990A46F832D1
:10812000F823C95853680C9A536611660E99432276
:10813000920089580C9A91660E9911221201895861
:108140000C9AD1660E9905229301CA18C958536832
:108150000C9A536711670E992922D300CA18C9587F
:1081600053680C9AD36791670C9A9168491C916087
:108170000C9AD82191800C9A0021D1800C9A392137
:1081800011700078002806D02B4803F0E1F90E9812
:1081900040680C99C860F9F7B1F97D20C000F9F783
:1081A00043F926480068C007002804D0234908681E
:1081B0000122904308602248022101602149097888
:1081C0004908491E81600121C1600BA9F9F716FA1F
:1081D000002800D0FEE71B48007880021A494018AA
:1081E0000A90002009900A98164909788902174ACE
:1081F0008918884214D20A990998C3000D4AD018E8
:10820000D25843680120F9F7C3F8002806D10A982C
:1082100008300A900998401C099000E0FEE7E2E768
:10822000F9F78EF90E98FFF755F90FB0F0BDC0467B
:10823000A1E200085804002085E400081420024050
:108240009C0F0020E075FF1F00F8FF07D4F8FF0720
:1082500000B587B016484F218900405A002803DC3A
:1082600006A9154808801EE01148C8300190C06E6C
:1082700003F018F80246019802920391006F03F090
:1082800011F8024602980B46039902F041FE05914F
:108290000490049805990022064B05F080F802F03E
:1082A00035FF06A90880002106A8405E07B000BD82
:0C82B000A000002000005940FFFF00006B
:1082BC0010B594B090492520C00008588F4A126818
:1082CC00801ACD22520088521F2012901298012839
:1082DC0011DB12988A4982008818001F00688850A8
:1082EC001298884982008818001F006888501298DC
:1082FC00401E1290EAE78048C830C169804A11607C
:10830C0000698049086080491191002010900F91FC
:10831C000E90C1430D910C910B910A9112901298F1
:10832C001F2853DC1298810075484058C1174840EB
:10833C00401A0F99884209DA129881007048405807
:10834C00C1174840401A0F9012980D901298810056
:10835C006B484058C1174840401A0E99884209DBB7
:10836C001298810066484058C1174840401A0E9038
:10837C0012980C901298810062484058C1174840DE
:10838C00401A1199884209DA129881005D484058C8
:10839C00C1174840401A119012980B901298810006
:1083AC0058484058C1174840401A1099884209DD76
:1083BC001298810053484058C1174840401A1090F9
:1083CC0012980A901298401C1290A8E70E980F99D8
:1083DC00401AC1174840401A099010981199401A38
:1083EC00C1174840401A08904349C86D6822895A01
:1083FC0002F0DCFF07900798142102F0AFFF079002
:10840C001920069009980799884203DA13A9414864
:10841C0008806BE008980699884203DA13A93C4857
:10842C00088063E00020C1430591049103911290F0
:10843C0012981E2816DC1298314982008818406860
:10844C008958401AC1174840401A0490049805995D
:10845C00884203DD04980590129803901298401CF2
:10846C001290E5E7039810283DD1089802F0D8FE49
:10847C0000900191099802F0D3FE024600980B4639
:10848C00019902F03FFD00220292204B04F081FF83
:10849C0002F036FE02460298174947239B00CA5247
:1084AC002522D2008958154A1160129012981F2863
:1084BC0019DC12998A00124880581F22511A8B001D
:1084CC000D49C831CB18F0241851129B9C000D4853
:1084DC000059D21A9200891817221201885012984A
:1084EC00401C1290E2E713A900200880002113A879
:1084FC00405E14B010BDC046A00000200C1000203F
:10850C00200D0020200C0020FFFFFF7F00408F403B
:08851C00FEFF0000FFFF00005C
:1085240010B594B091492520C0000858904A1268AB
:10853400801ACD22520088521F20129012980128CE
:1085440011DB12988B4982008818001F006888503C
:108554001298894982008818001F00688850129870
:10856400401E1290EAE78148192109014158814AC5
:108574001160D4214058804908608049119100203D
:1085840010900F910E90C1430D910C910B910A9193
:10859400129012981F2853DC129881007548405895
:1085A400C1174840401A0F99884209DA129881008D
:1085B40070484058C1174840401A0F9012980D90C7
:1085C400129881006B484058C1174840401A0E99D0
:1085D400884209DB1298810066484058C117484018
:1085E400401A0E9012980C901298810062484058DC
:1085F400C1174840401A1199884209DA129881003B
:108604005D484058C1174840401A119012980B9089
:108614001298810058484058C1174840401A109990
:10862400884209DD1298810053484058C1174840D8
:10863400401A109012980A901298401C1290A8E7C1
:108644000E980F99401AC1174840401A0990109883
:108654001199401AC1174840401A08904349C86DFF
:108664006822895A02F0A6FE07900798C117890F5D
:108674004018801007906420069009980799884252
:1086840003DA13A9404808806BE0089806998842E9
:1086940003DA13A93B48088063E00020C143059135
:1086A40004910391129012981E2816DC12983149F5
:1086B4008200881840688958401AC1174840401AF7
:1086C400049004980599884203DD04980590129853
:1086D40003901298401C1290E5E7039810283DD1AE
:1086E400089802F0A1FD00900191099802F09CFD08
:1086F400024600980B46019902F008FC00220292FF
:108704001F4B04F04AFE02F0FFFC02460298174990
:108714008F235B00CA522522D2008958144A116063
:10872400129012981F2819DC12998A001148805857
:108734001F22511A8B000D49C831CB18140118514E
:10874400129B9C000C480059D21A920089182722C7
:10875400120188501298401C1290E2E713A90020DD
:108764000880002113A8405E14B010BDA0000020B2
:1087740008100020A00C0020A00B0020FFFFFF7FAA
:0C87840000408F40FEFF0000FFFF0000DF
:1087900000B589B0089007911C4800681C498842C0
:1087A00003D01A490868401C086008980799401AC5
:1087B00002F03CFD0591049005980190049800900A
:1087C00014480390CA21405A02F030FD0246009836
:1087D0000B46019904F0E3FD002202920E4B02F0D9
:1087E00097FB029A05910490049805990B4B02F0AF
:1087F0008FFB0B4A0B4B02F08BFB02F087FC0399BB
:1088000019221201885009B000BDC0460410002092
:10881000FFFFFF7FA0000020ECFF23410000444049
:08882000FCA9F1D24D62403FBA
:1088280030B58FB000200E900D900C900B900A90F0
:108838003648026802210A4302600068084009902D
:1088480009983248026804210A4302600068084017
:10885800089008982D48026820210A4302600068A1
:108868000840079007982948026801210A430260D6
:108878000068084006900698052000070190F92135
:108888004D0100220392294605F09DF8039A012024
:10889800029004021E480490214605F094F80299BB
:1088A80004984A020A92212212040B920C910AA9F6
:1088B8000591F9F735F80198029B039A05990A95ED
:1088C8000B930C920D92F9F72BF80298039A0599DD
:1088D80040230A930B920C900E48F9F721F8029B5B
:1088E800039A049805990A940B930C920D92F9F740
:1088F80017F8029B039A0498059920240A940B936D
:108908000C930D92F9F70CF80FB030BD34100240FB
:088918000004005000080050AB
:1089200081B00146684601800088012149028842E1
:1089300002D102490120086001B07047B40F002045
:1089400030B5A5B000201390249023902290209061
:108950001F901E901B901A9019A9087018A90870F2
:1089600000F048FA0028FFD1F7F732FC00F07AFA5D
:10897000204802F0EDFDFCF7C3F9FCF733FAFCF7F1
:1089800069F9FFF751FFFEF7C5FB01F065F8FCF749
:108990006BFF00F0BFFE00F0C7FA01F02DF901F007
:1089A00073FAFEF771F816A81190FEF7CBFB119938
:1089B000024615A802700378FC4A53800978D181D9
:1089C0000078129003281FD81298810001A0405807
:1089D0008746C046E5890008ED890008F989000846
:1089E000038A0008F148FEF723FC0DE0EF48FEF78C
:1089F00071FD09E069E00008EC480021FEF70AFF7C
:108A000002E0EA48FEF714FCE94802F0A1FDE7485D
:108A1000FEF760FDE748402104F089F800280FD1F7
:108A20003220F7F73FFCE348402104F080F80028AB
:108A300006D1E14802F08CFDDC480121FEF7EAFE98
:108A4000DA480169828AC38ADC480090DC4804F075
:108A5000C1FBDC481090F8F717F91098DA490822A2
:108A6000F7F75AFE6420F7F71DFCFDF795FAD74893
:108A700002F06EFD00F0C8FB002014901498CB4962
:108A8000098B884218DA052000070D900122D102D7
:108A90000E9104F09CFFAF2040000F90F7F702FC0E
:108AA0000D980E99002204F092FF0F98F7F7FAFB49
:108AB0001498401C1490E1E7C5480068012827D1AC
:108AC000C34900200B900860BF480A90806800F0FE
:108AD000F3FD0A98006800F09DFF0A984068FEF7D1
:108AE000A7FA0A99C8680969FFF752FEAF4AC83267
:108AF0000C921069C117D269D31702F01DFC0B9BB1
:108B00007D22D20002F07CFC0C990864FFF70AFD7C
:108B1000B0480068012806D105F08FF9FFF7CEFBB9
:108B2000AC4900200860F7F7B7FB22902298239900
:108B3000401A219022982390219920984018209043
:108B400021991F9840181F901A98012805DB219839
:108B5000002802D01A98401E1A909F4801680A689F
:108B60000F210A4019A90A7000684068179018A8D8
:108B700000780978884269D0199818A908708B493B
:108B80002520C2008858401C88501B9800280BD113
:108B90000520000701210991890204F02CFF0998A2
:108BA00001028E4804F027FFFEF70EF801F07CF971
:108BB00000F034FB00F058FC00F0E2F900F012FE87
:108BC0007A490891672292008852FFF741FB089981
:108BD0008B22520088527C480490C06900F0E0FE6D
:108BE000049808994069CA2203928A5A002306937E
:108BF000194602F0A1FB069B0B22059202F09CFB9A
:108C000002F05EFB069A764B079302F081F902F0C0
:108C10007DFA039A069B08990446049815252D01B0
:108C20004C5380698A5A194602F086FB059A069BC6
:108C300002F082FB02F044FB069A079B02F068F9FF
:108C400002F064FA0899A922520088525748408BD2
:108C5000002873D05A482621405C00286ED1534822
:108C6000408B029001282CD0029802282ED0029826
:108C700003282FD00298042831D00298062837D034
:108C80000298072836D00298082837D00298092879
:108C900038D002980A2838D002980B2839D0029888
:108CA0005049884238D002984F49884238D00298BB
:108CB000FD218900884237D002984C49884212D061
:108CC00035E03A480021FFF7E3F833E03748FEF794
:108CD000AFFA2FE035480121FEF79CFD2AE033482A
:108CE000FEF7F8FB26E031480121FFF7D1F821E03B
:108CF00000F064F92D48FCF787FF1BE02B48FCF7D8
:108D0000A7FF17E0FCF7CEFF14E02848FCF7F0FFC0
:108D100010E0FDF78FF80DE0002000F05DF909E0AC
:108D2000012000F059F905E000F00AFA02E03048AD
:108D300002F00EFC1D4900204883FFE71D4840213A
:108D400003F0F5FE00281BD11A98002818D10A203C
:108D5000F7F7A8FA1748402103F0E9FE00280FD1E1
:108D60007D2080001A901B98002807D101221B92B9
:108D700005200007910204F02AFE01E000201B906C
:108D80000F4805F010F800280FD00D48FCF7CAFB7B
:108D9000022806D11B98002802D1094804F093FA52
:108DA00003E0064984222220885085E6A0000020A6
:108DB000EBE6000800080050FBE60008140B00205A
:108DC00038060020040E0020600F0020B7E20008E3
:108DD000B80F0020B40F0020100F00200004005036
:108DE00000002441F2030000F3030000D20400005D
:048DF00092E4000801
:108DF40000B589B000200090089007900690059077
:108E040004900390029002A8F8F74AFD009801A983
:108E140008700698AA2806D1104802F097FB01A909
:108E24000020087012E00698BB2806D10A4802F018
:108E34008DFB01A90120087008E00698CC2805D113
:108E4400044802F083FB01A90220087001A80078FD
:108E540009B000BD5BE700083FE7000823E700080E
:108E640000B59BB00EA80290342103F019FB00203A
:108E740000900D900C900B900A9009900890079028
:108E84000690059004900390012001908002F8F769
:108E9400D1FEF8F7BBFE2149086818221043086088
:108EA400F8F7BEFE009A0199029806230E931091DA
:108EB4000B021193129240231393022315931693DA
:108EC4001792082218924A04199249071A91F8F73E
:108ED400EBFE002801D004F03EFA07200A9002219C
:108EE4000B9100200C900D900AA8F9F7C3F9002803
:108EF40001D004F030FA0A480390002004900120C5
:108F0400810708910002099003A8F9F763FB002880
:108F140001D004F020FA1BB000BDC0465C10024032
:048F24000140020006
:108F280000B583B011480268012109030A430260B1
:108F380000680840029002980D4801900D490160B0
:108F4800012101714171072282601022C260FF2253
:108F580002610022426182610162F8F721F800286B
:108F680001D004F0F6F903B000BDC0463810024045
:088F78003C0F00200030024014
:108F800000B581B00A482521C9004058094902F0BE
:108F900013FA0090009808490968884206D00098A2
:108FA0000549086002480021FEF772FF01B000BDCC
:0C8FB000A000002080510100E40F002010
:108FBC00BFF34F8F034904480860BFF34F8F00BFC6
:0C8FCC00FDE7C0460CED00E00400FA05D3
:108FD80000B58BB009A9019108700020089007908E
:108FE8000690059004900390029002A8F8F756FCAA
:108FF80001980078C00700283AD04A4802F0A4FA3D
:109008000698AA2830D102200290BB200690F8F7D3
:1090180071FA002802D0424802F096FAF8F7AAFA44
:10902800002802D03D4802F08FFA404802F08CFA3E
:1090380002A8F8F76BFB002808D03E4802F084FA33
:10904800F8F7BAFA0AA90020087055E0F8F7B4FA58
:109058002E4802F079FAF8F76FFA2D4802F074FA00
:10906800334802F071FA02E02F4802F06DFA40E04E
:109078000698BB283DD102200290AA200690F8F756
:1090880039FA002806D0264802F05EFA0AA900201C
:10909800087031E01A4802F057FAF8F76BFA00281E
:1090A80006D01E4802F050FA0AA90020087023E0F2
:1090B800144802F049FA02A8F8F728FB002808D05B
:1090C800F8F77AFA144802F03FFA0AA90020087063
:1090D80012E00D4802F038FAF8F76EFA0B4802F081
:1090E80033FAF8F729FA0A4802F02EFA094802F08A
:1090F8002BFA0AA9012008700AA800780BB000BD55
:109108009EE00008F9E200080FE50008D5E4000831
:109118008FE0000831E300080FE3000878E000085A
:109128000FE70008A3E40008DBE20008C4E4000835
:08913800EEE40008C5E20008A6
:1091400000B589B000200790069005900490039028
:109150000290019001A8F8F7A5FB0620019001906C
:10916000BB2005900720000606900520000607900A
:10917000F8F7C4F9002802D0174802F0E9F9F8F727
:10918000FDF9002802D0154802F0E2F9144802F077
:10919000DFF901A8F8F7BEFA002808D0144802F059
:1091A000D7F9F8F70DFA08A9002008700FE0F8F7D2
:1091B00007FA0C4802F0CCF9F8F7C2F90A4802F0B5
:1091C000C7F90A4802F0C4F908A90120087008A8E4
:1091D000007809B000BDC0460FE7000878E000083D
:1091E000C4E40008D5E400088FE00008EEE40008BD
:0491F000C5E20008CC
:1091F40081B0009002490120086001B07047C04668
:04920400B80F00207F
:109208000249C8310248C88788877047A0000020F3
:04921800FFFF000054
:10921C0080B589487421405A002800D0E6E0874880
:10922C000088002804D08449832042008448885256
:10923C00814883214900405E002807D07E48832165
:10924C004900405E401C002800D088E07A49D820B4
:10925C000858898E88420EDA7E4802F073F97648F7
:10926C0083214A0001218152052000074902002276
:10927C0004F0A7FB73E07049E42008583C228A5E96
:10928C007D21C900514388420FDA714802F05AF926
:10929C0069498320420002208852052000070121E1
:1092AC004902002204F08DFB59E06349CE20085E90
:1092BC004822895E88420FDD644802F043F95E491A
:1092CC008320420003208852052000070121490217
:1092DC00002204F076FB42E05749CC20085E48227D
:1092EC00895E88420FDD574802F02CF952498320E1
:1092FC004200042088520520000701214902002267
:10930C0004F05FFB2BE04C49CE20085E4C22895EBA
:10931C0088420EDA4C4802F015F947498320420086
:10932C0005208852000701214902002204F049FB64
:10933C0015E04149CC20085E4C22895E88420EDA49
:10934C00404802F0FFF83C49832042000620885236
:10935C000520000701214902002204F032FB3648A7
:10936C0083214900405E00283FD03349D82008585B
:10937C00C98E884239DD3049E42008583C228A5E87
:10938C007D21C900514388422FDD2B49CE20085E38
:10939C004A22895E884228DA2749CC20085E4A2274
:1093AC00895E884221DA2449CE20085E4E22895EED
:1093BC0088421ADD2049CC20085E4E22895E884204
:1093CC0013DD1D4883214900405E02280DD0224840
:1093DC0002F0B8F81849832042000020885205207A
:1093EC0000070122510204F0ECFA1FE0124874212C
:1093FC00405A012806D1052000070122510204F031
:10940C00E0FA13E00C487421405A022807D10520D9
:10941C00000701214902002204F0D3FA06E00520DE
:10942C00000701214902002204F0CBFA0248742102
:10943C00405A0249088080BDA0000020281000205E
:10944C00FFFF000075E3000877E70008B1E00008B3
:0C945C002CE5000853E30008D4E00008F1
:1094680080B589487621405A002800D0E6E0874830
:109478000088002804D0844941208200844888520A
:10948800814841218900405E002807D07E4841215B
:109498008900405E401C002800D088E07A49D82026
:1094A8000858098F88420EDD7F4802F04DF876484B
:1094B80041218A000121815205200007090200226A
:1094C80004F081FA73E07049E42008583E228A5E6D
:1094D8007D21C900514388420FDD724802F034F8FB
:1094E8006949412082000220885205200007012195
:1094F8000902002204F067FA59E06349CE20085EA9
:109508004022895E88420FDD654802F01DF85E49F9
:10951800412082000320885205200007012109020A
:10952800002204F050FA42E05749CC20085E40225D
:10953800895E88420FDD594802F006F852494120F9
:109548008200042088520520000701210902002218
:1095580004F039FA2BE04C49CE20085E4422895E9B
:1095680088420EDA4C4801F0EFFF4749412082005B
:1095780005208852000701210902002204F023FA7D
:1095880015E04149CC20085E4422895E88420EDA03
:10959800404801F0D9FF3C4941208200062088520A
:1095A8000520000701210902002204F00CFA3648C0
:1095B80041218900405E00283FD03349D82008580F
:1095C800498F884239DA3049E42008583E228A5EB9
:1095D8007D21C900514388422FDA2B49CE20085EED
:1095E8004222895E884228DA2749CC20085E422236
:1095F800895E884221DA2449CE20085E4622895EA7
:1096080088421ADD2049CC20085E4622895E8842BD
:1096180013DD1D4841218900405E02280DD02348F2
:1096280001F092FF1849412082000020885205204D
:1096380000070122110204F0C6F91FE01248762142
:10964800405A012806D1052000070122110204F022
:10965800BAF913E00C487621405A022807D10520B0
:10966800000701210902002204F0ADF906E00520F7
:10967800000701210902002204F0A5F90248762119
:10968800405A0249088080BDA00000209E000020AA
:10969800FFFF0000B9E300089BE7000897E3000814
:1096A800E3E0000866E5000845E5000806E1000873
:1096B80000B583B00290104801688A09891A0160D0
:1096C800029A01688918016000688009019001996F
:1096D8000A4848430A4901F06BFE01460948C82276
:1096E8008152C83000900199074801F061FE009945
:1096F800488003B000BDC046F80F0020E880000095
:0C970800FFFF0000A0000020D08A2F7599
:1097140000B589B000210191089107910691059146
:10972400049103911C4802901C4A026081607F22CC
:10973400C260FF22026141618161C161012292071D
:1097440002624162F9F748F8002801D003F003FEF1
:1097540004A90220087000204870887005900790C2
:1097640008900D480122F9F723F9002801D003F0ED
:10977400F2FD03A901220A700420487016208870A3
:109784001820C8700448F9F7ADF9002801D003F097
:10979400E2FD09B000BDC046100F002000280040C3
:1097A40082B00190019800680A4988420FD10A48A2
:1097B4000268012189020A4302600068084000909F
:1097C4000098064908680122D2031043086002B0D9
:1097D4007047C046002800403C1002405C10024024
:1097E40000B591B05D480F905D480E905D480D90B6
:1097F40000200C905C48049058210391405A01F0D9
:1098040013FD5A4A5A4B03F0C8FD01F07DFC03993D
:10981400024604980B92405A01F006FD554A564BF5
:1098240003F0BBFD01F070FC014604980A91534912
:109834000968CF2252008152D821405809900998D2
:109844000B99884208DD4E49002008604B490860A6
:1098540010A9514808807BE009980A99884208DADF
:109864004749002008604549086010A94A48088013
:109874006EE043480068002802D109984049086016
:109884003F480090006801F0CFFC00220192354B64
:10989400029301F04FFA01F037FC01460098089159
:1098A400006801F0C1FC019A029B01F027FB01F062
:1098B4002BFC079009980899884208DD304900205C
:1098C40008602E49086010A93248088040E00998D1
:1098D4000799884208DA2A49002008602749086065
:1098E40010A92C48088033E024480168491C016011
:1098F40000682449884205D31B49E42008582322E0
:10990400D200885218482521C90040581E4901F048
:1099140051FD069006981D490968884215D006989D
:109924001A4908601A4801688A09891A01600E49AF
:109934002322D2008B5E0268D2180260006880097C
:10994400059005988D225200885210A900200880A5
:10995400002110A8405E11B000BDC04651B89E3F22
:10996400B81E85EB00002440A00000207B14AE4705
:10997400E17AF03F0AD7A3703D0AEF3FF00F0020D1
:10998400E80F0020312A000080510100EC0F002074
:0C999400F40F0020FEFF0000FFFF0000A9
:1099A00000B583B00290029917484843C117090CCB
:1099B0004018001401900198144940180190019931
:1099C00064204843019001980A2101F0CDFC104920
:1099D000C831C8800620085E0822895E884204DDFE
:1099E0000B49C831C88808810BE00949C8310620F5
:1099F000085E0A22895E884203DA0549C831C888B0
:109A0000488103B000BDC046E40C0000A8FDFFFF84
:049A1000A000002092
:109A140000B585B004900498C1170C4AC83202926C
:109A240052880023019301F085FC019B062201F07A
:109A340081FC01F043FC019A054B01F067FA01F047
:109A4400B7FB0299C86005B000BDC046A000002065
:049A540000002441A9
:109A580000B581B01048009010490160412189008B
:109A680041600021816007221302C3600161012364
:109A780043619B0483611023C36101624162816277
:109A8800C26201634163F9F7D7F8002801D003F0F7
:109A980060FC01B000BDC046A00D002000300140B0
:109AA80000B591B0109000200F900E900D900C9082
:109AB8000B90109800681E49884236D11D480268EC
:109AC800012109030A430260006808400A900A98C5
:109AD8001948026801210A43026000680840099099
:109AE8000998E0200B9002200C90002001900D9026
:109AF8000E900F900520000702900BA9F7F710FFB2
:109B08000199029808910791069105910491012203
:109B18000392D30304930592069104A9F7F700FF73
:109B28000298039A202103F04EFF11B000BDC046F1
:0C9B380000300140401002403410024098
:109B440082B00A48026801210A43026000680840A2
:109B54000190019806480268012109070A4302603E
:109B6400006808400090009802B07047401002401E
:049B74003C1002405F
:109B780000B581B0F6F780FB0D480168491C01600B
:109B88000C4900910068C0087D280FD3F6F780FBC8
:109B9800094988420AD30949C831C86D401CC865BB
:109BA800886D401C886502490020086001B000BD2E
:109BB800E00F0020204E0000214E0000A0000020F1
:109BC80080B50248F7F740FB80BDC046680E00200C
:109BD80080B50248FBF728FB80BDC046140B002067
:109BE80080B50248F9F760FE80BDC046C40E00206B
:109BF80030B518490122500208800B46C8330020AE
:109C0800D86598654524A500134C4C53C5435D643D
:109C18009D644725AD004C538F256D004C5323257B
:109C2800ED004C538D256D004C5302240C814A8164
:109C380005248C81D4071C62084C5C62D2031A810B
:109C4800074A5A81074C5C619A61C12252008852C6
:109C580030BDC046A0000020FFFF0000FFFFFF7FCF
:089C6800FF7F00000080FFFFF8
:109C700000B587B05448006838210840009020287B
:109C800000D982E00098810001A040588746C04674
:109C90008B9D00088B9D00088B9D00088B9D000804
:109CA0008B9D00088B9D00088B9D00088B9D0008F4
:109CB000159D00088B9D00088B9D00088B9D00085A
:109CC0008B9D00088B9D00088B9D00088B9D0008D4
:109CD000319D00088B9D00088B9D00088B9D00081E
:109CE0008B9D00088B9D00088B9D00088B9D0008B4
:109CF0001D9D00088B9D00088B9D00088B9D000812
:109D00008B9D00088B9D00088B9D00088B9D000893
:109D1000279D000830492F48086045E02E497D20E6
:109D20000002086040E02C490120C00308603BE0CD
:109D30002648016803221140039100687021084001
:109D40000009401C02900398032805D1029921487C
:109D500001F032FB059004E002991D4801F02CFB54
:109D60000590059A194801687F231B021940090ACA
:109D7000514305910068400F401C049005980499D8
:109D800001F01AFB144908600EE01448006807212E
:109D9000C9020840C10A01208840019001990C487D
:109DA00001F00AFB0C490860074800680F2109020E
:109DB000084081090A4840580690069A06490868F2
:109DC000D040086007B000BD081002400C100240EF
:109DD0000024F40000127A009800002000100240D5
:049DE00004C50008AE
:109DE40010B58EB00D9000200C900B900A90099045
:109DF40008900D9800681F49884238D11E480268AF
:109E0400012189030A43026000680840079007980B
:109E14001A48026802210A4302600068084006905A
:109E240006984020089002200190099001200A9091
:109E3400002004900B900C901148029008A9039103
:109E4400F7F770FD019B02980399049A8024089403
:109E540009930A920B920C92F7F764FD049A1B2063
:109E64000590114603F02FFD059802F061FD0EB038
:109E740010BDC0460038014040100240341002407A
:049E84000004005086
:109E88000649086E4042E12213014343D8172922AC
:109E9800D2008B50891848607047C046A000002047
:109EA800F0B595B07E48416800680843002809D19C
:109EB8007C484D21890041587B4848437849002215
:109EC8004A6008607948416800680843002809D159
:109ED80074482721C90041587348484373490022F0
:109EE8004A6008606F48E4214058002815D46D483E
:109EF80009907221415A1491E42141581498484319
:109F0800642101F02DFA09995F229200885070208F
:109F18000B5E8858C01A885005E06249F02008583E
:109F28005F22920088505F4D08955F208000295875
:109F3800C81712911390D8202958C817109111905A
:109F480012981399109A119B01F0F2F97D22D20010
:109F58000023079301F050FA079B0F910E90286E8B
:109F68000D930C900C980D99E122120101F0E0F983
:109F78000B910A900F9C0E9E17200201A9184868A1
:109F8800AB589B196041AB5048600F9F0E9829232E
:109F9800DE00AC196368AD592D1808987B418551CE
:109FA8006360496883580B980A9AD21A884107DA7D
:109FB8000B980A9B3B49172212018B50891848605D
:109FC80038492920C200881840688A580021521E42
:109FD800884106DB33492920C200002088508918AF
:109FE8004860304906912920C20088588918496874
:109FF800E122120104920023059301F0FDF9049A6D
:10A00800059B06995B24A4000851172004010859F0
:10A018000919496801F0F0F9014606982F22D20083
:10A0280081502121C9004058002823D51D4803909C
:10A03800C8300290006C4442E317194948680A681E
:10A04800121958410A60486008684968164A00238E
:10A0580001F0EAF9039902460298C266426E7D2031
:10A06800C0005043C96D01F0A3F903994F22920033
:10A07800885213E00B48C8300190046CE3170B4971
:10A0880048680A68121958410A60486008684968AF
:10A09800054A002301F0C8F90199086715B0F0BD19
:10A0A80018060020A000002080EE360020060020C0
:10A0B80000B581B00D485B2189004058002805D4BF
:10A0C8000A485B2189004058009005E007485B2159
:10A0D800890040584042009000980449112212011A
:10A0E800885000F005F801B000BDC046A00000206F
:10A0F80000B587B0002005907D20C00004901D4861
:10A10800432189004058002805D51A494520820076
:10A11800194888522BE017494320800008580390BB
:10A128000398C96D884206D31249452082007D20D4
:10A13800C00088521BE00F48C06D002805D10D49AA
:10A14800452082000C48885211E003987D21CA00FE
:10A1580000230193194601F0EBF8019B054A02928E
:10A16800D26D01F061F9029945229200885207B038
:0CA1780000BDC046A0000020FFFF00005A
:10A1840000B589B01848006E002300930793069029
:10A1940006980799E122120101F0CCF802460098D2
:10A1A40001920A460199059204910390029005993F
:10A1B40004980843002810D00B491720020188583E
:10A1C40089184968094A002301F0B4F8049A059BE8
:10A1D40001F014F90391029002E000200390029030
:10A1E400029809B000BDC046A0000020A08601006E
:10A1F40000B58DB000200B9031480A9031485B21A6
:10A2040089004058002806D52E485B218900405813
:10A214004042059001E0002005900599C817089177
:10A224000990002007900690264811210901405802
:10A23400002815DC08980999214A04920023039305
:10A2440001F078F8039B1F4A126E01F0D7F8034619
:10A2540003980A460499C91A90410691079016E09A
:10A2640008980999164A02920023019301F062F8B2
:10A27400144A11231B01D258D31701F0BFF8034627
:10A2840001980A460299C91A9041069107900798C5
:10A29400069A00210C4BD21A884104DB0020079057
:10A2A4000748069008E00799069A00205242884120
:10A2B40002DB00200790069006980DB000BDC04652
:0CA2C400A0860100A0000020A18601007F
:10A2D00000B58FB000200D9039490C910B90394892
:10A2E000112109014058002809DC3649C86D2D228A
:10A2F000D200895840180021099108900AE031499C
:10A300004320800008582D22D20089584118C817D0
:10A31000089109902B490846C83002900069032231
:10A32000D201895A4018C10F41184810C917079126
:10A33000069008980999069A079B00F0FDFF7D2278
:10A34000D200002301F05CF80246029803920A460C
:10A35000039905920491806C01280EDB04980599FD
:10A36000174A002300F0E8FF164A11231B01D258B8
:10A37000D31701F045F80B900CE004980599104AAA
:10A380000023019300F0D8FF019B0E4A126E01F0EA
:10A3900037F80B900B9AD01700210B4BD21A88413B
:10A3A00002DB07480B9007E00B9AD11700205242BE
:10A3B000884101DB00200B900B980FB000BDC04618
:0CA3C000A0860100A0000020A186010082
:10A3CC0010B586B013480190006E002300930593DE
:10A3DC00049004980599E122120100F0A7FF0246AF
:10A3EC0000980B46019903930292039A029C17233F
:10A3FC001B01CC50CB185A602922D20088508A18E5
:10A40C0050605B229200885009225201885006B09D
:08A41C0010BDC046A0000020A5
:10A42400C20F490089184000034A40428A4101D3BF
:0CA4340000207047012070470000E0FF8E
:10A440000122D2079143034A4A4010434142484106
:08A450007047C0460000F07FD8
:10A45800074A0A40531E9A41C00F49000818054987
:10A46800884201D3002000E0012010407047C04618
:08A478000000F07F0000E0FF8E
:10A4800030B50E4B5D1C0C0D2C4010D0AC420ED0E4
:10A49000A2189A4205DD0120C007014009480918A9
:10A4A00009E0002A04DD064B19401205114330BDB6
:10A4B0000120C0070140002030BDC046FE0700005B
:08A4C000FFFF0F800000F07F98
:10A4C80010B54B005B0D084CA34201D0002B02D104
:10A4D8000023136010BD054C1B191360044A11407A
:10A4E800044A891810BDC046FF07000002FCFFFFA0
:08A4F800FFFF0F800000E03FB0
:10A50000F0B587B00E4604460021C843574F069069
:10A51000401C0590384601914841590004914D0D69
:10A52000534900D18CE0E50F710002914919039164
:10A53000650006994D1B03998F4100D282E0D10F2F
:10A54000049D69185500059F7D1B88417AD3012120
:10A55000C807304004904748354605400340101B6B
:10A560001846A84171D2039109050298470D05913B
:10A5700003D0481E06400E430DE08D420AD20398D8
:10A58000C004E10F6E00761864007F1E85423546D8
:10A59000F7D300E02E461D0D3748054004D005993D
:10A5A000481E03400B430FE0059883420CD20398EA
:10A5B000C00406901946D30F4800C31852006D1E00
:10A5C000069881421946F6D3AF4212DDA01A3146F1
:10A5D000994104D454405E40264302D113E0204602
:10A5E0003146C40F49000E1944007F1EAF42EDDC16
:10A5F0002F462046841A35469D41059906D4504081
:10A600005E40064304D1019C049916E00446354699
:10A610000D420AD10398C004E10F6A00511864008A
:10A620007F1E05420D46F7D000E02946002F15DDBC
:10A63000781E049A891800050918204607B0F0BD55
:10A64000019CFAE7019C0A49F7E762405D40154327
:10A6500000D00496002DD7D10024D5E70398C21B63
:10A66000204600F049FE04460020E2E7FFFFDFFF3E
:0CA670000000F87FFFFFFF7FFF070000E5
:10A67C00F0B583B00D46044628494A1C280D1040FD
:10A68C00421E8A4240D22749884205D20024002D1E
:10A69C00264635DA264E33E03331884201D92E4630
:10A6AC002EE01F49461820462946324600F00EFE81
:10A6BC001D4A114001434A424A410020002D01DA53
:10A6CC00014600E0012111430291184901903246E4
:10A6DC0000F01CFE074632460E462E402740019BDA
:10A6EC00D843401C1049594100F000FE029A38181A
:10A6FC007141002A00D10E46002A00D107463C4683
:10A70C002046314603B0F0BD002802D10121C90713
:10A71C000D402E460028F3D10024F1E7FE0700007F
:10A72C0001FCFFFFFF030000FFFF0F000000F0FF24
:04A73C000000F0BF6A
:10A74000F0B587B00A0D521E484B9A4214D206AAA1
:10A75000FFF7BAFE06460F464948301A474881417E
:10A76000069C3046394618DA0022474B00F0E4FADE
:10A7700006460F46641E14E0C30F4A00D318440077
:10A7800064423B4C9C416AD3520D6CD000290A466E
:10A7900000DA394A002963DA66E00022394B00F01A
:10A7A000CBFA059403900D460024E243049430460E
:10A7B0003946FFF765FE354B002200F0BDFA024630
:10A7C0000B460398294600F0A3FB03900F46024670
:10A7D0000B4602F0E4FD04460D462D4E02213046A4
:10A7E00022462B4603F04FFB2A4A2B4B00F0A4FADB
:10A7F0000290019110360321304622462B4603F089
:10A800006AFB02460B460298019900F081FB224642
:10A810002B4602F0C4FD039C22463B4602F0BFFDDE
:10A8200022463B4600F088FA06460F46059800F09F
:10A83000FDFC04460D46194A194B02F0B0FD3246A4
:10A840003B4600F079FA06460F46164B204629464D
:10A85000049A02F0A4FD32463B4600F06DFA0A4627
:10A86000114607B0F0BD034A0020F9E7FE070000DB
:10A870000000E0FF0000F0FF0000F87F9EA0E63F30
:10A88000CE3B7F660000F0BF0000E0BF0000E03F6D
:10A89000C00000089AB5B312FF0750C0A80C615C55
:08A8A00010D02BBF0030E63F91
:10A8A800F0B585B00C4607465948411C220D0A40B0
:10A8B800511E814200D38EE05948C01B5748A04121
:10A8C80000DAA2E000205849C91B5649A1410146B7
:10A8D8007FD30120C007214681435648381A54487F
:10A8E800814174D3544A554B3846214602F053FDF2
:10A8F8000122D2072240524BD31800252A4604953C
:10A9080000F016FA00F0FEFB039000F08BFC0290BA
:10A918000E464C4B002202F03EFD3A46234600F01C
:10A9280007FA04460F46484A484B0298314602F057
:10A9380032FD22463B4600F0FBF906460D4602462C
:10A948000B4602F028FD0F46414A424B044602904E
:10A9580002F021FD404A414B00F0EAF922463B460D
:10A9680002F019FD3E4B049C224600F0E1F9324604
:10A978002B4602F010FD05460E46204630492A4671
:10A98800334600F0B9FA01900091364A364B029CE2
:10A998002046394602F0FFFC344A354B00F0C8F92E
:10A9A80022463B4602F0F7FC019A009B00F0C0F9F2
:10A9B80002460B462846314600F0A6FA049A204B78
:10A9C80000F0B6F9039A521CFFF756FD01E017494B
:10A9D800002005B0F0BDF80F610008187900494261
:10A9E8000C49814121460ED30120C00781430A4802
:10A9F8004840384300D075E7002C214600DA002192
:10AA0800002C00DA00273846E3E70349E0E7C046B0
:10AA1800FE0700000000E0FF0000F07F422E8640A5
:10AA2800EF39FAFE2B2386C0D2BC7ADD0000F03F56
:10AA3800A19CC73B2342920C3CF92F9E2C15F73F53
:10AA48000000E03F0030E6BFA80C615C10D02B3F4F
:10AA58001CDC586FA452F13EE0F6B36FE4707C3F03
:10AA68000000D03F0938DE6F993F403FB351427133
:04AA78008E71AC3FF0
:10AA7C00F0B585B016460024E7438B4D7A1C2A4668
:10AA8C0062414A4002436FD001955A00550D00D1E6
:10AA9C0008E100940290874C601C039104930D0D07
:10AAAC0005406D1EA54273D21D461C0D0440824B01
:10AABC00E4185B1C9C426BD337463046294600F0A9
:10AACC001FFB064600F0ACFB2A46029D7840514025
:10AADC000143039C30D101200290C00786422BD049
:10AAEC00002E0096714B41D0F0174640361A0027C5
:10AAFC0001970393012E019A00D02A460497012E48
:10AB0C006A4B00D023462F462846214602F041FCD2
:10AB1C00224605460C46304602990840634B00D04D
:10AB2C00134642423A400498039902F032FC07461D
:10AB3C000B467608DDD11AE0002228462146134642
:10AB4C0000F0BEFA002802D0604900241DE001206C
:10AB5C00C007844328462146FFF7ECFD3A46049B88
:10AB6C0002F017FCFFF79AFE04460EE000270020C7
:10AB7C004E493A461D4600F0C5F904460098002897
:10AB8C0000D42946002800D43C46204605B0F0BD30
:10AB9C000298C30F4C00E3184400641E484C5C41FF
:10ABAC00E2D20125F30FD21873005B1B434B9A4181
:10ABBC0010D23F4A114210D0424B0C465C40044329
:10ABCC0026D00C4654400443049827D100283CDA84
:10ABDC002146DAE734460499D7E737463046049CD9
:10ABEC00214600F08DFA064600F01AFB4C403B461D
:10ABFC004340234327D1049900291C46194600DA07
:10AC0C002B49F007C1D0E807039E06407118BCE73A
:10AC1C000094049800281ADA009819E0584006436A
:10AC2C0002982CD1284A4A400243009C1F49ACD0C0
:10AC3C00EA07039B93430022391A01989841144662
:10AC4C002ED31B4A2CE0049A3FE711469DE7104691
:10AC5C0003903046049F394600F052FA044600F047
:10AC6C00DFFA794070400843039802D1E807039952
:10AC7C000818E10700D00390009C039985E7EB07C7
:10AC8C000C469C430023391A0198A0411C461946D6
:10AC9C0000D37AE70C48039E46400298304301D01B
:10ACAC00114672E7014970E7FFFFEF3F0000F03FEC
:10ACBC000000F07FFE07000001F8FFFF0000E0FF3E
:10ACCC00FFFF1F000000F0FF0000F0BF0000F87F46
:10ACDC00F0B581B000280090124D13D00146C0177A
:10ACEC0041400F1A0026104CF80707D00CCC304608
:10ACFC002946083C02F04DFB06460D4608347F08F9
:10AD0C00F2D100E000260020064932462B4600F026
:10AD1C00F9F8009A002A00D43046002A00D42946BB
:0CAD2C0001B0F0BD0000F03FE80000089E
:10AD3800F0B40125ED070F005F405AD48B4200D1D3
:10AD4800824205D950404240504059404B405940FA
:10AD58004E18760DDF187F0D3BD0741C640529D082
:10AD6800F41B352C26D80E0DDB022B43DB0AC90257
:10AD78002943C9121700202C1ED2E741E240574050
:10AD8800E3415A40A340E3405A4000248018594107
:10AD98000AD3B21C520521D0C207012F6241170005
:10ADA8004008CB0718434908013636054208AF4129
:10ADB80060417141F0BC7047203C06D01F00E7415C
:10ADC800E3405F400024012A6741C0186141EBD38A
:10ADD800DFE7002EEED129400020EBE701363105F0
:10ADE8000020E7E7E742E5D10020C143090DC90487
:10ADF800E0E76B400E00871A9E4104D26E40C01BEC
:10AE0800B141D21973414E18DF18AC0AE642E9D2B3
:10AE1800760D7F0D31D0F41B362CCBD8B4460E0DF1
:10AE2800DB022B43DB0AC9022943C90A012C32D8A9
:10AE380004D1D4075208DF073A435B08EF0A64429B
:10AE4800904199411ED0002239424DD124194041E8
:10AE580049410124394204D1013400184941394299
:10AE6800FAD06246A24204D9361B013E360589193A
:10AE7800A0E7F10AC90700209CE736429AD10020D2
:10AE8800002197E70200224394D0B842DED20100A5
:10AE980020002024E3D1202C13DD203CE2411700C0
:10AEA800A240E2405740E3415A40A340E3405A40A1
:10AEB800012FBF410137174300227C42984191413D
:10AEC8000CE01700E741E2405740E3415A40A340F5
:10AED800E3405A407C429041994100220F0303D23B
:10AEE800013E241940414941013E36054708AC411D
:08AEF80050417141F0BC7047AC
:10AF0000F0B40125ED076B40004C20473FAD000831
:10AF1000F0B40125ED070C005C402C40A446AE0ABD
:10AF20004C18DF18F4423DD2F74245D2640D4CD0A4
:10AF30007F0D3CD0E41BC9022943CF0ADB022B431F
:10AF4000DB0A0600B61A9F4104D2013CB6197F41C4
:10AF5000B6185F416812800D241838DD001884424D
:10AF600025D8E80C0021B6197F41B61A9F4103D3BA
:10AF700040414941F7D304E0B6185F410018494108
:10AF8000F1D32405B6197F41B61A9F4105D3374343
:10AF9000C20717430022012F50416141624611430D
:10AFA000F0BC70470CD100280AD1F74208D200202B
:10AFB000C143490D0905F1E7002A01D1F74206D046
:10AFC0000020C143090DC904EAE77F0DF8D0002035
:04AFD0006146E5E70A
:10AFD40030B401256D054C00E54215D85C00E5420E
:10AFE40012D80C001C436400044314430FD005D250
:10AFF40082428B418041013030BC7047904299417C
:10B004008041013030BC7047002030BC70470120C3
:04B0140030BC704795
:10B0180070B4012676054C005D00E6420CD8EE427D
:10B028000AD825430543154303D0994204D19042D9
:10B0380002D1012070BC7047002070BC7047C04628
:10B0480030B401256D054C00E54215D85C00E54299
:10B0580012D80C001C436400044314430FD005D2DB
:10B06800904299418041013030BC704782428B4107
:10B078008041013030BC7047002030BC704701204F
:04B0880030BC704721
:10B08C0030B401256D054C00E54215D85C00E54255
:10B09C0012D80C001C436400044314430CD005D29A
:10B0AC0082428B418041404230BC70479042994172
:10B0BC008041404230BC7047002030BC7047C046D5
:10B0CC0030B401256D054C00E54215D85C00E54215
:10B0DC0012D80C001C436400044314430CD005D25A
:10B0EC00904299418041404230BC704782428B4132
:10B0FC008041404230BC7047002030BC7047C04695
:10B10C00F4464A1805D200F051F801D5C017400892
:10B11C00604701235B05D34206D200F047F801D506
:10B12C000120C0074042604701D10042F5D0D01742
:04B13C004008704710
:10B140004A00520D01239B02D21A01321DD45242F1
:10B150003F321DDD8C46C902430D1943C002012355
:10B16000DB071943202A02D308000021203AD141ED
:10B17000D04048409140D140484063461B4203D5EF
:10B18000002340428B411900704700200021704786
:10B19000002801D0012211434B0001225205D34265
:10B1A00000D959080020C90FC90701D4C04341087C
:04B1B0007047C046DE
:10B1B4004A0010D2520D03231B02FF33D21A0AD4C1
:10B1C40052421F3209D4400DC90208430123DB0750
:10B1D4001843D040704700207047D0177047C046CE
:10B1E4004B001BD25A0D01239B02D21A013215D4F3
:10B1F40052423F3215DBC902430D1943C0020123F9
:10B20400DB071943202A02D308000021203AD14148
:10B21400D04048409140D140484070470020002130
:08B224007047D01701007047CC
:10B22C00054B004206D5404200B5984708BC0122A8
:0CB23C00D207114318470000A5B200081B
:10B248000B00034329D0CA0FD200043212023D3248
:10B25800094203D5002349424042994102D10100E5
:10B268000020203A0B0C04D1103A0904030C1943AE
:10B278000004094203D4013A00184941FBD5844629
:10B28800C00A4B051843C90A120563465B055B41B2
:0CB2980002D3012B0023584151417047A4
:10B2A40042221201033A010007D002D4013A0018E5
:0CB2B400FCD51205C30A4005991870472C
:10B2C0000B00034305D0042212023D320942014B18
:08B2D0001847704765B2000841
:10B2D800202A07D203009040914052422032D340A6
:10B2E80019437047203A0100914000207047C0463A
:10B2F800202A07D2D0400B00D1405242203293403E
:10B3080018437047203A0800D04000217047C046D3
:10B31800202A07D2D0400B001141524220329340DC
:10B3280018437047203A08001041C9177047C046B3
:10B3380030B5514343435C18010C130C0D005D43B9
:10B34800641992B2514380B242430D0C0904521859
:10B3580065415843010C00048018694130BDC0465E
:10B36800CA1751408B1A17D0C1174A409446484013
:10B37800411A48081A0000E052008242FCD9002015
:10B3880000E05208914200D3891A40419A42F8D10C
:10B3980062465040801A704710B500F095F810BD0D
:10B3A80007B5FFF7DDFF0EBC4243891A00BDC04652
:10B3B8000A0015D00300400800E052008242FCD980
:10B3C800002000E052089B1A06D340418A42F9D176
:10B3D800704752089B18F8D200188A42F9D1704772
:08B3E80010B500F071F810BD72
:10B3F00038B504004D42FFF7DFFF4543611938BD02
:10B4000070B5CC1760406140001BA141DD176A4058
:10B410006B40521BAB4100F00BF862406340121BC3
:10B42000A3416C4060406140001BA14170BDC0461B
:10B43000002B09D1002907D110B51100FFF7D8FF63
:10B440000A000021002310BD70B400240125ED077F
:10B45000002B07D1002905D0834203D2130000221C
:10B460002C0000250026A419994200D1904212D93F
:10B4700092185B4103D2EE076D086408F3E7DE071C
:10B480005B08520892190126F6079B1903E0DE07B4
:10B490005B0852089219801A994103D364416D41A7
:10B4A000F5D30FE024196D410AD2DE075B0852087C
:10B4B000921980185941F5D364416D41E7D301E0F9
:10B4C0008018594102000B002000290070BC704711
:08B4D000002000217047C04676
:10B4D800F0B503AF93B06E46F51D2135F41D393430
:10B4E80074613362F261F160306102F032FDB06084
:10B4F800C21D07218A436946B1616946881A70608E
:10B508008546F41D1D3400212422204600F0CAFF80
:10B518000B487169F2680A6048600A482860306917
:10B528002862B06868617068E8602046F169326A2C
:10B5380000F01EF8B1698D46FE1F053EB546F0BD08
:08B548004BDF0008FFFFFF7F4D
:10B5500083B010B581B0044603A80EC0054800684A
:10B5600003AA0092214602F020F801B010BC02BCF0
:08B5700003B008478C00002025
:10B57800F0B59FB012920B460446002020600121CE
:10B588000A020F924A020B928A020192CA020092A0
:10B5980003220D92920205920D034A0307928A0331
:10B5A80003920491C90317910A90C043029016941C
:10B5B80009951978252909D0002901D100F03CFE08
:10B5C8005C1C169801F090FF2346F2E7DB1C0A9FEB
:10B5D8000B9C981E00780246203A102A2CD880210D
:10B5E80092003E461F4602A39A583B463746974666
:10B5F8003DB600085DB600085DB6000857B60008FD
:10B608005DB600085DB600085DB6000851B60008D2
:10B618005DB600085DB6000881B6000855B600089A
:10B628005DB6000849B600085DB600085DB60008BA
:10B638004DB6000840210AE05E28294607D009E0F7
:10B64800102104E0214602E0179900E020210F4371
:10B658005B1CBEE75B1E014630390024092916D859
:10B668000A2161434418303C591C18780246303A84
:10B678000A2A0B46F4D30AE0129901C91291C10FA4
:10B6880009010F43C1174840441A581E0078002684
:10B698002E281CD118782A2805D158789B1C129975
:10B6A80040C912910FE05B1C0146303909290CD8BA
:10B6B8000A2171434618303E591C18780246303A20
:10B6C8000A2A0B46F4D3002E01D40F990F43E11731
:10B6D8006B2808DC4C2803D068283CD06A280AD19B
:10B6E8000220074305E06C2830D07A2801D074285E
:10B6F80001D118785B1C8C43462811931BDD014649
:10B708006339152937D8C0467944097949008F44E7
:10B71800710B4D1BD70A0B0A0A0A0A8194610A0A9F
:10B728008F0A560A0A3A44E70C94039C27430021DF
:10B73800089139468EE0442815DD452834D046283E
:10B7480000D036E7079807430098BAE018786C28C5
:10B758002ED1022003E0187868282CD1082007434E
:10B7680058789B1CC7E7252800D08EE2252116981B
:10B7780001F0BAFE7AE2472800D19FE0582800D0AD
:10B7880017E707990F430C94D34A782800D1203241
:10B79800039C0F990F42394601D0D04B19403B0604
:10B7A800DB171340089355E007980743019888E092
:10B7B8005B1C049A01E05B1C042217439BE70C9472
:10B7C8000F990F4201D0C5490F403946039C00220A
:10B7D80008923FE00C9438060F990F430E97C01754
:10B7E800232101400891129820C8129000240820B3
:10B7F8000690D3E1129E3578621E169C2046394683
:10B80800159201F0C3FE2046294601F06DFE361D53
:10B818001296C2E01298006839071699096800D58F
:10B8280037E2BA07016000D434E20021416031E216
:10B838001596129901C912918EE00C940F990F4236
:10B84800394601D0A54A11403A06D2173023134091
:10B858000893039C02220A40214205D1002A129A29
:10B8680008D1131D00240BE0002A129B13D104CB2E
:10B87800D41715E0D21D07239A435468134608339A
:10B88800129315684A0713D408220A4000D0EDB273
:10B89800002A0ED102E1DB1D0722934314CB0033AB
:10B8A80012934B0707D40B0700D5E3E01546E4E0F5
:10B8B800ADB20024F2E015B21204DDE007980743A8
:10B8C800059807430F98074201D0304600E006204C
:10B8D8000C943946059A1140891A4A424A4100286F
:10B8E80000D002461592129CE41D07208443266866
:10B8F800656830462946FEF79FFD083412940028F3
:10B90800304629460ED000221346FFF7DBFB3A46A5
:10B9180007990A4000280C9C0FD0002A704819D0BB
:10B92800704817E0FEF77AFD00280C9C37D007987E
:10B9380007426D480ED06D480CE0002A6C4900D0D3
:10B948006C49002A01D06B4800E06948401CBA06DF
:10B9580000D5084668490F400028684E00D00646C2
:10B968000F980742304602D100F016FD02E0159903
:10B9780000F04AFD054659480740621B16983946AB
:10B98800159201F003FE002D07D0169C3178204651
:10B9980001F0AAFD761C6D1EF8D1F8065DE130466F
:10B9A8002946FEF755FD002800D10646002800D19B
:10B9B800002513963046294602F05FFA0446012016
:10B9C800002C089001D0C00745401EAA30461095AB
:10B9D8002946FEF775FD1E980D9948430A21FFF781
:10B9E800BFFC06461E90002C01D0602007430022B1
:10B9F800139C2046294614921346FFF709FB00289A
:10BA080018D1701CFFF766F922462B46FFF75AFB40
:10BA180000281E9806D0411C1E91801CF2E71E9833
:10BA2800401E1E90FFF756F922462B46FFF72AFBC9
:10BA38000028F4D13D4605980540089883021E98D1
:10BA48009D42159E00D113E105998D4207D186428A
:10BA580000DC0DE10421C943884200DC08E10199BA
:10BA68000F42109D0E9300D180E20E2800DCD0E139
:10BA7800149E7BE255B21206D417002C05D48A0610
:10BA88000AD44A060AD5202207E000226D42A241C4
:10BA98002D230893144601E02B2208920F9A114295
:10BAA80001D00E4A11400A460F990E920A42049993
:10BAB80000D03146069100276E2838DD6F380928F6
:10BAC80000D98AE07844007940008744196786865F
:10BAD800868636868667C04658300000FFFDFFFF21
:10BAE80084E500087FE50008E3E70008DFE70008D1
:10BAF8008EE5000889E50008FFFEFFFF15E1000854
:10BB08002846204369D0E808610740180146072005
:10BB18002840303018AAD055C808E40862078018B1
:10BB28000A4622437F1C002A0D46EFD155E05828CB
:10BB380034D0642801D069284FD1284620434CD0FE
:10BB480011461798014010912A461098002808D0ED
:10BB580038460D990840032803D118A82C21C1554F
:10BB68007F1C002510462146159414460A222B46B0
:10BB7800FFF75AFC149013910A222B46FFF7D8FBC3
:10BB8800201A3021014318A8C1557F1C0920001B29
:10BB980015988541149D139CD6D31EE02846204352
:10BBA8001AD007980E990142C04800D0C048290908
:10BBB8002207891800270A460F212940415C18AB43
:10BBC800D955110924092307C918134623437F1C93
:10BBD800002B1546EFD100E00027089DFF2D01D866
:10BBE800029801E0B348FF300B9C0C9B0699CE1BD2
:10BBF800F1178E43B9195A1A002D00D012180E9950
:10BC0800214203D1169801F0C1FC00221592290A9D
:10BC1800169C03D0204601F067FC01E0002D03D0FC
:10BC28002046294601F060FC20460E99159A01F03D
:10BC3800ADFC30212046324602F075F9012F0ADBAF
:10BC48007D1C18A84019801E0178204601F04CFC84
:10BC58006D1E012DF5D80E98C006099D119B00D4C4
:10BC6800A7E420211698159A02F05DF9119BA0E42B
:10BC78000F9934318842109C06950FD113982146AC
:10BC88008D4A8E4BFFF740F90FE0002800D090E472
:10BC9800E2E201701298001D12908AE44042FFF718
:10BCA80019F8139A234601F076FB04460E46002243
:10BCB8001346FFF7ADF9002839D120463146FEF783
:10BCC800BBFB00282046314600D01CE60E97002218
:10BCD8007B4BFFF7B5F900281E9F0FD000222046A6
:10BCE8003146774BFFF710F904460E460022744B95
:10BCF800FFF7A6F97F1C0028F0D11E9700222046E6
:10BD08003146704BFFF7DEF9002811D0002220469B
:10BD180031466B4B01F03FFB04460E460022694B4F
:10BD2800FFF7D0F97F1E0028F0D11E9700E00E978C
:10BD3800059806998142159801D0014600E0411EF8
:10BD4800029D0028149100D1002113914842FEF76A
:10BD5800C1FF2A46FEF790FB22463346FEF7E8FF6E
:10BD680006460D4600220692554C2346FFF768F911
:10BD780000280AD01E98401C1E90002230462946F2
:10BD88002346FFF7C1F806460D46109615951398F9
:10BD9800002866D000990B4680330E9A13408B42D8
:10BDA80061D1102800DB10200546FEF793FF3246CC
:10BDB800159B01F0F0FAFFF711FA0C4601462143F2
:10BDC800069914914FD0214606463F4A3F4BFFF74C
:10BDD800AFFA4A08C3079A184008C90708183C4927
:10BDE800081A3C48904114953DD330460A22002356
:10BDF8002146FFF719FB0C4607460A220023FFF7E6
:10BE080013FB1498401E14902DD01A433846EDD0D9
:10BE180029E0C143711810290E4600DB10263A06A6
:10BE280000D5A3E0002900D1A0E03046FEF752FF7C
:10BE3800139A2B4601F0AFFA00242246264BFEF750
:10BE480077FFFEF717FC22461D4BFEF755FB2246EF
:10BE58002346FFF7DDF8002800D184E0761EE4D100
:10BE680082E00698149080210E9806460140149AA4
:10BE780011430C98801A002901D1401F00E0801F4F
:10BE8800139009981E9C064201D1089D46E00321A3
:10BE98002046FFF785FA881C0125C04678440079BA
:10BEA800400087441B2A381B2A00C046CFE70008F9
:10BEB800BFE70008FFFEFFFFA0C8EB85F3CCE17FDA
:10BEC800000024400000F03FCDCCCCCCCCCCCCCC76
:10BED80099999999999999190000E03F641E1E94BF
:10BEE800002210981599DF4B01F055FA1090159122
:10BEF8001398401E139002250DE0A41E1E940022E4
:10BF080010981599D84B01F046FA1090159113988E
:10BF1800801E13900325149AD01782437006800F51
:10BF2800149202D01398401E1390204601F0F7FF98
:10BF3800632802DD1398401E13900898C002374604
:10BF4800874310981599FFF749F906460C46FFF7FD
:10BF5800B3F902460B4610981599FEF7CDFF1090DD
:10BF68001591139A76E034461E9826461038149692
:10BF78007142884200DC0846FEF7ACFE029AFEF7E2
:10BF88007BFA139A2B46FEF7D3FE05460C461E98FD
:10BF9800401CFEF79FFE2A462346FFF717F80028A5
:10BFA8001E9800D0401C002814D4112818D301462C
:10BFB80010391E911021081AFEF78CFE2A462346D6
:10BFC80001F0E9F9FFF70AF906460C46002015903A
:10BFD800109018E01095159400261E96344612E02D
:10BFE80000201E9028462146FFF7F8F806461594CB
:10BFF8000C46FFF761F902460B4628461599FEF7ED
:10C008007BFF1090159138460E998843974908315F
:10C0180000250A4608326D1C0B684968F31A234646
:10C028008B411146F6D280213940149A11434B1E98
:10C038000A469A41002901D00021C9437B069B0F7B
:10C0480000D0D1431E9A891A0C9A149BD21A5118FF
:10C058004A1B0746D017114681430B9810300E979C
:10C0680007420AD1012A08DB0F462021169801F061
:10C078003BFA7F1EF9D10E9A01E03A460F4640205E
:10C088001040910603D4002809D0202104E000289C
:10C0980001D02D2100E02B21169801F025FA0E98E9
:10C0A800C00607D4002F05D03021169801F01CFADD
:10C0B8007F1EF9D16D1EE8006C4A111849681258A4
:10C0C800B01A2046884101D2302007E03020B61A45
:10C0D8008C41401CB31A23468B41F8D2C1B2169842
:10C0E80001F002FA002DE5D113970E9E3446009810
:10C0F8000440169F0BD01E98012808DB401E1E9096
:10C108003021384601F0F0F91E980028F6DC80202E
:10C1180030401499084344D02E21384601F0E4F900
:10C12800149D102D00DB1025E8178543002C01D144
:10C13800284601E01E98281A159CFEF7CBFD149A94
:10C14800012A22DB109A234601F025F9FFF746F869
:10C1580004460E462F467F1EF800444A11184968C7
:10C168001258A01A3046884101D2302007E030200A
:10C17800A41A8E41401CA31A33468B41F8D2C1B28F
:10C18800169801F0B1F9002FE5D11499481B169FB4
:10C198000E9E06D06C1A3021384601F0A5F9641CB1
:10C1A800F9D301980642099D139F38D00798064293
:10C1B80001D0452100E06521169E304601F094F932
:10C1C8001E980028304604D42B2101F08DF91E98C2
:10C1D80005E02D2101F088F91E9840421E90642840
:10C1E8000DDB6421FFF7E4F801463031304601F0F9
:10C1F8007BF91E986421FFF7D3F808461E910A219F
:10C20800FFF7AEF801463031304601F06DF91E985F
:10C218000A21FFF7C5F83031304601F065F9002FE3
:10C22800119B01D1FFF7C5F9169C2021204601F08A
:10C238005BF97F1EF9D119E5169CE068002805D046
:10C2480006CC083C914201D20A9A4254204601F099
:10C2580090F920681FB0F0BD169801F08AF902988D
:10C26800F8E7C046000024400000594030010008AB
:10C2780009490968091A4A1E9141084A1268121A9E
:10C28800531E9A410A4006490968081A411E884106
:10C29800104040427047C0468C00002090000020AB
:04C2A80094000020DE
:10C2AC000F480321016141610E4A82610E49C1614F
:10C2BC00012189020162002181624162C162026630
:10C2CC000A4A4266102282660167C1664167084AC3
:10C2DC000F234B40D35C4354491C1029F8D17047B1
:10C2EC006C0A0020A4E500082E100020AE140020DB
:04C2FC0093E50008BE
:10C30000F0B581B00D461821414316484618F06A31
:10C31000183602281ED0144601280ED00027002807
:10C320001DD1304601F053F9A04218D330462946BA
:10C33000224601F057F9274611E0304601F047F94F
:10C340000746A04200D32746304629463A4601F028
:10C3500049F904E03046294601F061F907463846BC
:08C3600001B0F0BD6C0A0020E1
:10C36800F0B581B014460D4606460A480078002804
:10C3780001D1FFF797FFEFF31087012181F31088B0
:10C38800304629462246FFF7B7FF87F3108801B0E9
:08C39800F0BDC0466C0A002054
:10C3A000F0B581B00178002925D003220146009222
:10C3B00091430D680023DC438607F60EB440E44346
:10C3C0002C43114D6719A743104A174206D14C68F8
:10C3D00067191646A643091D3E42F8D022060FD023
:10C3E0002204120E09D02202120E08D0220E009B47
:10C3F00006D0042304E0002004E0012300E002232F
:10C40000C918081A01B0F0BDFFFEFEFE80808080D2
:10C41000F0B581B00022002934D00378002B31D050
:10C4200003270246BA430024E5438607F60EB540CB
:10C43000EE431568354306463E40711804290CD377
:10C440000097134EAF19114BAB433B4204D1091F68
:10C450005568121D0329F5D8009F2B060DD02B041B
:10C460001B0E07D02B021B0E06D02B0E00D004276C
:10C470003C4602E0012400E002248C4200D30C463A
:10C48000101A0219104601B0F0BDC04680808080AD
:04C49000FFFEFEFEAF
:10C49400002A03D0013A8B5C8354FBD17047C04619
:10C4A40000220B0011001A00002A02D0013A815424
:04C4B400FCD1704700
:10C4B80002480068002800D101487047CC0F0020CE
:04C4C80074000020DC
:10C4CC007F2805D8034A125C0348405C1040704733
:0CC4DC0000207047E7E700080EE60008AB
:10C4E8007F2805D8034A125C0348405C1040704717
:0CC4F80000207047E7E700080EE600088F
:10C504000000000000000000000000000000000027
:10C514000000000000000000000000000000000017
:10C5240001000000020000000300000004000000FD
:10C5340006000000070000000800000009000000D9
:10C5440000000000000000000000000000000000E7
:10C5540001000000020000000300000004000000CD
:0CC5640015E4000890C5000870C5000830
:10C57000CDC400086FDF0008ABD60008E9C400088E
:10C580007BDF0008B9D600085FDF00087DD6000811
:10C5900017E400080DE600080DE600080DE60008A7
:10C5A0000DE600080DE600080DE600080DE600089F
:10C5B0000DE600080DE60008FFFFFFFFFFFFFFFF8D
:10C5C000FFFFFFFFFFFF0000DBE30008BFE50008FF
:10C5D0001CE10008DCE5000873E10008ADE5000897
:08C5E000B6E500087AE100084D
:10C5E800034C206804348047FBE7FCF7A5F9FEE715
:04C5F80068E80008E7
:10C5FC000448054988438546044880470448054952
:10C60C000160EBE7008000200700000065D3000804
:08C61C0008ED00E00000000839
:10C62400FEE7FEE7FEE7FEE7FEE7FEE7FEE7FEE7DE
:10C63400FEE7FEE7FEE7FEE7FEE7FEE7FEE7FEE7CE
:10C64400FEE7FEE7FEE7FEE7FEE7FEE7FEE7FEE7BE
:10C65400FEE7FEE7FEE7FEE7FEE7FEE7FEE7FEE7AE
:0CC66400FEE7FEE7FEE7FEE7FEE7FEE76C
:04C67000719C0008B1
:10C6740087B006900591049203A9002008701F203A
:10C6840002900299481E029000200029019009D0CE
:10C69400059802991F221140C840012108404142D7
:10C6A400484101900198C007002800D0E9E70498A8
:10C6B400009018284CD80098810001A04058874663
:10C6C40053C7000855C7000855C7000855C70008D8
:10C6D40055C7000855C7000855C7000855C70008C6
:10C6E40045C7000855C7000855C7000855C70008C6
:10C6F40055C7000855C7000855C7000855C70008A6
:10C7040037C7000855C7000855C7000855C70008B3
:10C7140055C7000855C7000855C7000855C7000885
:10C7240029C700080298072802D303A9012008702A
:10C7340011E00298082802D303A9012008700AE036
:10C744000298102802D303A90120087003E002E034
:10C7540003A90120087003A8007800280DD10598CA
:10C76400069909684861069800688068182188431A
:10C774000499084306990968886003A8007807B0FB
:02C784007047FC
:10C7860081B000900098806804210840800801B0BC
:02C796007047EA
:10C7980084B00390029100200190029800900C2828
:10C7A80032D80098810001A040588746E9C70008A0
:10C7B80011C8000811C8000811C80008F3C700080C
:10C7C80011C8000811C8000811C80008FDC70008F2
:10C7D80011C8000811C8000811C8000807C80008D7
:10C7E80003980068406B01900EE003980068806B26
:10C7F800019009E003980068C06B019004E0039879
:0EC808000068006C0190FFE7019804B07047D3
:10C8160083B002900191009202984069019A042126
:10C826000A400721914088430099914008430299A4
:06C83600486103B07047E9
:10C83C0081B000900098C0680321890208404142F1
:06C84C00484101B07047F5
:10C8520000B583B002900298806A0190019801F0BD
:06C8620001F803B000BD67
:10C8680000B583B002900298806A01900199886DA2
:10C878004022104388650199C86D04221043C86599
:0AC88800019800F0E8FF03B000BDC6
:10C8920083B00290019100920298806A019A1F214E
:10C8A2000A400F2319469140884300999B0619407C
:0EC8B200890E914008430299886203B07047D6
:10C8C00081B000900098006807218905084001B0F8
:02C8D0007047AF
:10C8D20081B000900098806802210840400801B0B1
:02C8E20070479D
:10C8E40081B00090009880680121C907084317218E
:0AC8F40088430099886001B0704786
:10C8FE0081B000900098B42140587F21084001B0CB
:02C90E00704770
:10C9100081B000900098006903218907084001B0A8
:02C9200070475E
:10C9220081B00090009800680F218904084001B08E
:02C9320070474C
:10C9340000B581B001466846017000214056F4F705
:06C94400DFFA01B000BDA6
:10C94A0000B581B001466846017000214056F4F7EF
:06C95A00E8FA01B000BD87
:10C9600085B00490039102920020019001980299F1
:10C97000490888420ED2039801998A008118805A8A
:10C980000004498840180499096808600198401C0F
:10C990000190EBE702A80078C007002808D00498AF
:10C9A00000680090039801998900405A0099088016
:0AC9B00004980068006805B07047A5
:10C9BA0000B587B00690059104920020029006996E
:10C9CA000220487706980168886801221043886027
:10C9DA000698006A019001281BD0019802281FD0EE
:10C9EA000198032823D100200390039804998842D0
:10C9FA000AD205980399890040580699096808607F
:10CA0A000398401C0390F0E70698006800680290BB
:10CA1A000DE006980599049A00F06CFF029006E072
:10CA2A0006980599049AFFF796FF0290FFE7069980
:0ACA3A0001204877029807B000BD04
:10CA440000B587B0059004910392029301A90020D8
:10CA5400087005982421405C012803D106A902200E
:10CA640008705EE005992422012088540598252148
:10CA7400405C012848D10599252202208854059953
:10CA84000020C86305980168086801229043086083
:10CA940005980499039A029BF4F7A0FB0598006B90
:10CAA400002806D00598016808680E221043086023
:10CAB4000BE0059801680868042290430860059813
:10CAC400016808680A22104308600598406C0068F1
:10CAD400C003002806D50598416C0868012212029B
:10CAE400104308600598006D002806D00598016D74
:10CAF400086801221202104308600598016808685A
:10CB040001221043086009E005998020C863059953
:10CB140024220020885401A901200870019806A944
:0ACB2400087006A8007807B000BDF5
:10CB2E0084B0009101460098039102A908800398F1
:10CB3E0000690988084203D001A90120087002E0AB
:0ECB4E0001A90020087001A8007804B070470B
:0ACB5C0081B06946088001B07047FF
:10CB660000B585B00390029101920398029B01994A
:10CB760000910321C9020022F6F7A1FA002808D085
:10CB86000399086E20221043086604A90320087042
:10CB960029E00398029B0199009180210022F6F773
:10CBA60022FB002808D00399086E2022104308664D
:10CBB60004A90320087016E00398029B01990091CE
:10CBC600032149020022F6F77AFA002808D00399D1
:10CBD600086E20221043086604A90320087002E0AC
:0ECBE60004A90020087004A8007805B000BD66
:10CBF40084B0039002910192029A1F210A400120FD
:10CC040090400090009B039A106A98431062019A26
:10CC14000298084082400399086A1043086204B0ED
:02CC2400704757
:10CC260000B583B001900198002803D102A9012024
:10CC360008703EE001983D21405C002806D101992C
:10CC46003C2200208854019800F000FF01993D2203
:10CC560002208854019901C9F6F749FB0199482237
:10CC66000120885401993E220120885401993F22CF
:10CC76008854019940228854019941228854019987
:10CC86004222885401994322885401994422012062
:10CC9600885401994522885401994622885401995D
:10CCA6004722885401993D220120885402A9002078
:0ACCB600087002A8007803B000BD6A
:10CCC00000B585B00390029101926946002008707A
:10CCD00003983C21405C012803D104A9022008707C
:10CCE00075E003993C22012088540198002815D151
:10CCF00003980068029B19685A68DB68F6F7DCFE47
:10CD00000398016888690C229043886102988268C0
:10CD10000398016888691043886151E001980428EC
:10CD200017D103980068029B19685A68DB6800F005
:10CD300052F803980168886903229202904388613F
:10CD4000029880680202039801688869104388612C
:10CD500036E00198082815D103980068029B1968ED
:10CD60005A68DB6800F08DFE03980168C8690C22E0
:10CD70009043C8610298826803980168C8691043AB
:10CD8000C8611DE001980C2817D103980068029B28
:10CD900019685A68DB6800F055F803980168C8699B
:10CDA000032292029043C8610298806802020398AD
:10CDB0000168C8691043C86102E069460120087033
:10CDC00003993C2200208854009804A9087004A804
:06CDD000007805B000BD73
:10CDD60086B005900491039202930598006A00902C
:10CDE6000599086A102290430862059880690190A7
:10CDF60001980321090288430190039801020198D2
:10CE06000843019001980F21090388430190029875
:10CE1600000381B20198084301900099A020814344
:10CE26000091049909010140009808430090019877
:0ECE36000599886100980599086206B070475A
:10CE440086B005900491039202930598006A0090BD
:10CE54000599086A01221203904308620598C06983
:10CE6400019001980321090288430190039801026B
:10CE740001980843019001980F2109038843019008
:10CE84000298000381B2019808430190009905209B
:10CE94004003814300910499090301400098084329
:10CEA400009001980599C86100980599086206B038
:02CEB4007047C5
:10CEB60081B0009000982821405CC00700280AD065
:10CEC6000098006840680121490488430099CA6AAD
:10CED60010430968486000982821405C80070028B4
:10CEE6000AD5009800684068012109048843009922
:10CEF6000A6B10430968486000982821405C400787
:10CF060000280AD5009800684068012189048843F2
:10CF160000994A6B10430968486000982821405CD4
:10CF2600000700280AD50098006840680121C90357
:10CF3600884300998A6B1043096848600098282145
:10CF4600405CC00600280AD5009800688068012168
:10CF5600090388430099CA6B1043096888600098E2
:10CF66002821405C800600280AD500980068806861
:10CF760001214903884300990A6C104309688860B7
:10CF860000982821405C4006002819D500980068C2
:10CF96004068012109058843009A536C18431268BA
:10CFA60050600098406C88420AD10098006840683A
:10CFB60003214905884300998A6C10430968486033
:10CFC60000982821405C000600280AD500980068D1
:10CFD60040680121C90488430099CA6C1043096856
:06CFE600486001B0704735
:10CFEC0082B00190019880214058212835D10198B8
:10CFFC006A21405A694608806846008800282CD06F
:10D00C0001985621405A00280DD101980168886872
:10D01C000122D2059043886001980168086840227B
:10D02C001043086019E001980068C06900060028E8
:10D03C000ED50199086D0078096888620199086D10
:10D04C00401C086501995622885A401E8852FFE7F9
:0ED05C000098401E69460880CEE702B070477B
:10D06A0081B0009000988021405821281FD1009853
:10D07A005621405A00280CD100980168086880227D
:10D08A0090430860009801680868402210430860CD
:10D09A000DE00099086D0078096888620099086DAA
:10D0AA00401C086500995622885A401E885201B0D1
:02D0BA007047BD
:10D0BC0000B585B0049004986021405A02A90880FC
:10D0CC00049884214058222831D104980068406A81
:10D0DC0001A908800498806D03900198029908407A
:10D0EC00039908800499886D801C8865049A5E21D8
:10D0FC00505A401E50520498405A002816D1049899
:10D10C00016808680922520190430860049801687C
:10D11C0088680122904388600499842220208850DA
:10D12C0004990020C866049800F081FD05E004987D
:0ED13C000168886908221043886105B000BDB3
:10D14A0000B583B0029002986021405A01A9088074
:10D15A0002988421405822282FD102980068406AF8
:10D16A00694608800098019908400299896D0870FB
:10D17A000299886D401C8865029A5E21505A401EA9
:10D18A0050520298405A002816D10298016808683D
:10D19A0009225201904308600298016888680122B6
:10D1AA0090438860029984222020885002990020A6
:10D1BA00C866029800F03CFD05E00298016888699B
:0AD1CA0008221043886103B000BD85
:10D1D40030B587B00A9C06900591049203A8038099
:10D1E4000088002803D003A80088032802D303A9D9
:10D1F4000120088003A800880930029004980028C0
:10D2040002D00498012802D10298401C029006988A
:10D214000A99059A049B03AC2488029D0195009405
:10D22400F7F7ECFE0699002048770699888406995A
:10D234000884069926228854069908770699C88393
:0AD2440006992222885407B030BD7D
:10D24E0000B581B0009000980168086840229043B4
:10D25E0008600099802220208850009900200867DD
:0AD26E00009800F0DFFC01B000BDE5
:10D2780000B581B00090009926220C208854009AAD
:10D288001068FF21283151188B239B00D25AF7F7D9
:06D29800EDF901B000BD3C
:10D29E0081B0009000998B2082000020885001B050
:02D2AE007047C7
:10D2B00081B0009000994520C2000020885000995C
:06D2C000087501B0704783
:10D2C60000B585B0049000200390049827300290A2
:10D2D6000498FFF7E1FF02980078049AFF212831AD
:10D2E600019150540398401C0390049840180299E9
:10D2F600039A0B7800F05CFD01990390049840189E
:10D30600039900F02BFD0390039804998B22920059
:10D3160088500498FFF7ADFF0498FFF7C6FF05B0E5
:02D3260000BD48
:10D3280084B0039002910192009302988030029099
:10D3380002980399009A88540098401C009001981C
:10D348000399009A88540098401C0090009804B0F3
:02D3580070471C
:02D35A0070471A
:02D35C00704718
:02D35E00FEE7E8
:02D36000704714
:02D36200704712
:02D36400704710
:10D3660008D1002806D1F54204D801D3002A01D1FC
:10D376006D0D09D10020C143090DC904F0BDF9D1D5
:10D386001242F7D1640DF5D00020C1434905490882
:10D39600A6E000206146F0BDF0B50127FF070E00AC
:10D3A6005E403E40B446BE0A4C18DD18F442D7D261
:10D3B600F542E4D2640DECD06D0DEAD06419C902D1
:10D3C6003943460DC0023143DB023B43DB0A10B44E
:10D3D6008E4685B297B26F43140C6C433E0CA4196B
:10D3E600260C2404BFB227439CB26C43A419190C23
:10D3F6006943250CA4B249190D04090C6419000CE3
:10D4060095B245433E0C76193743BFB2360C150C20
:10D416004543AD19A6B2240CAD192E0437432E0C84
:10D4260036199DB24543AD19ACB22E0C89191D0CA7
:10D4360045436D182E04290C3443704680B295B2CC
:10D4460045433E0C76193743BFB2360C150C45439F
:10D45600AD19A6B2AD19240C2E0437432E0C36197D
:10D466009DB24543AD19ACB22E0C89191D0C45432E
:10D476006D182E043443290C75462D0C90B2684362
:10D486003E0C80190604BFB23E43070CA0B23F18FB
:10D49600120C6A43D019020C80B2240CA4189AB25A
:10D4A6006A43121914042043120C89181B0C6B438F
:10D4B600C91810BC01273D05294203D1B6194041C0
:10D4C6004941013CFF077D0D013D641B0BDB6D00EF
:10D4D600AC4209DA240500254208BE416841614193
:0AD4E60066463143F0BD54E74EE7FF
:10D4F00030B581B0044668460170206900280FD01D
:10D500000CCC083C9A4233D26269531C636181544B
:10D51000A069616981422BD1204600F02EF827E0F6
:10D52000E068002809D00CCC083C9A4220D2551C57
:10D530009D4200D1002181541AE0A068002808D043
:10D540000CCC083C9A4213D2551C9D420DD0C9B256
:10D550000CE0236A002B0BD003CC083C884207D296
:10D56000694601222046984702E00021920081503E
:0AD570002068401C206001B030BDAF
:10D57A0010B54269002A07D00446036A002B01D07D
:0AD58A00216998470020606110BD80
:10D5940080B5CB0606D4890501D5302100E02021D1
:06D5A40000F0C3FC80BD95
:10D5AA0070B514460D460646FEF781FF0146304621
:0AD5BA002A462346FDF78BFF70BDE3
:0AD5C40080B50068FEF7CEFE80BDC2
:10D5CE00C2680169914201D9D04302E0D243891861
:06D5DE0080680818704788
:10D5E400F0B581B0154604464068A268E668801923
:10D5F400971BBD4204D22A46FEF74AFF751909E07B
:10D604000E463A46FEF744FFF119ED1B60682A46C0
:0AD61400FEF73EFFE56001B0F0BD37
:10D61E00F0B583B016460D46C76800210190029101
:10D62E000269F943BA4202D95418816802E05218CD
:10D63E00816854184268C91B8C4200D30C46B44210
:10D64E0000D33446D01929462246FEF71CFFE719AF
:10D65E00019881688F4200D100270299C760361B5E
:0ED66E002D196118002EDAD1084603B0F0BD68
:10D67C0010B50446002000290DD0002A0BD00978E3
:10D68C0048B2002808D4002C00D021600021196079
:0ED69C005960411E884110BD0120C04310BDE1
:0ED6AA00014641391A2901D220210843704758
:0ED6B800014641391A2901D22021084370474A
:10D6C60081B0009000988068012109070840000F8A
:04D6D60001B07047E8
:10D6DA0081B00090009880680121084001B070472D
:10D6EA0082B001900091019840690099042211408A
:0CD6FA0007228A401040C84002B0704770
:10D7060000B585B0039003980068FFF7DFF8019035
:10D7160003980068FFF7DEFF002842D00198002832
:10D726003FD103980068806805210840012808D188
:10D7360003980068F3F76BF8039801680320086004
:10D746000CE00399886D102210438865039AD16D09
:10D7560001200143D16504A9087025E0F2F799FD7F
:10D766000290039800688068C007002819D0F2F775
:10D7760090FD0299401A032812D303980068806826
:10D78600C00700280CD00399886D102210438865C5
:10D79600039AD16D01200143D16504A9087003E005
:10D7A600DFE704A90020087004A8007805B000BDD2
:10D7B60000B583B002900298806A01900198806D4E
:10D7C6005021084238D10199886D01225202104336
:10D7D600886501980068FFF72EF8002828D0019880
:10D7E600807E002824D10198006800680007002880
:10D7F6001ED501980068FEF7C3FF00280ED10198D8
:10D80600016848680C22904348600198806D0121A8
:10D816000843090288430199886509E00199886DE2
:10D826002022104388650199C86D01221043C865FE
:10D836000198FBF7DCFC0DE00198806DC00600281E
:10D8460003D5019800F008F804E00198006D416BDB
:08D856000298884703B000BDF1
:08D85E0081B0009001B0704799
:08D8660081B0009001B0704791
:10D86E0082B00190009101980068072189058843D4
:0CD87E00009908430199086002B070474F
:10D88A0081B00090009880680121084001B070477B
:10D89A0081B0009000988068C00F401E4142484104
:04D8AA0001B0704712
:10D8AE0082B0019000910198B42280587F21884364
:0CD8BE00009908430199885002B070479F
:10D8CA0000B583B0034602A80370019100920021BB
:0CD8DA0040560199F3F7D1FA03B000BDED
:10D8E60000B581B000900098F3F735FB01B000BD9C
:08D8F60081B0009001B0704701
:10D8FE0086B005900491039200200290029803993D
:10D90E008908884214D2049802998A008118805C92
:10D91E0000064A78120480188A7812028018C97894
:10D92E0040180599096808600298401C0290E5E7C6
:10D93E0003A80078800700283DD0039803210840F3
:10D94E00012806D1049802998900405C059909685E
:10D95E00087003980321084002280FD104980299F9
:10D96E008A008118805C00024978401801A908805D
:10D97E00059800680090019800990880039803218B
:10D98E000840032817D1049802998A008118805CF8
:10D99E0000024978401801A9088005980068009097
:10D9AE0001980099088004990298800040188078A8
:10D9BE0005990968087005980068006806B07047F8
:10D9CE0083B0029001A8018068460270007800289A
:10D9DE0004D001A800880299886103E001A800889C
:08D9EE000299886203B0704742
:10D9F60083B0029001A80180029949690091009ABA
:10DA06000188104608400004914340180299886135
:04DA160003B07047A2
:10DA1A0083B002A908700020019002986946087034
:10DA2A00684600780A2807D30198401C019000989C
:10DA3A000A3869460870F3E701980007000E69463C
:08DA4A000978084303B070479E
:08DA520081B0009001B07047A3
:08DA5A0081B0009001B070479B
:08DA620081B0009001B0704793
:08DA6A0081B0009001B070478B
:08DA720081B0009001B0704783
:08DA7A0081B0009001B070477B
:10DA820086B005900491039202930598006A009073
:10DA92000599086A01221202904308620598C0693A
:10DAA200019001980321884301900399019808434A
:10DAB20001900198F0218843019002980001C1B2BF
:10DAC200019808430190009905204002814300918A
:10DAD20004990902014000980843009001980599B1
:0CDAE200C86100980599086206B0704702
:10DAEE0086B004900391029201A900200870049858
:10DAFE003C21405C012803D105A9022008703BE0BF
:10DB0E0004993C220120885402980090002806D0E7
:10DB1E00009804280ED00098082817D022E0049808
:10DB2E000068806E0F2188430399084304990968A1
:10DB3E0088661AE004980068806E0F2109028843F7
:10DB4E00039908430499096888660EE004980068F2
:10DB5E00806E0F21090488430399084304990968CC
:10DB6E00886602E001A90120087004993C22002079
:10DB7E008854019805A9087005A8007806B070476A
:08DB8E0081B0009001B0704766
:08DB960081B0009001B070475E
:08DB9E0081B0009001B0704756
:10DBA60010B586B0089C0490039102A802700193F8
:10DBB60004980068C06903990840401A41424841E8
:10DBC60002A9097888422AD10898401C002825D045
:10DBD600F2F75FFB0199401A0899884202D8089823
:10DBE60000281BD10498016808680D225201904351
:10DBF6000860049801688868012290438860049947
:10DC060080222020885004998422885004997C22FE
:10DC16000020885405A90320087003E0C8E705A979
:0CDC26000020087005A8007806B010BDB2
:08DC320081B0009001B07047C1
:08DC3A0081B0009001B07047B9
:10DC420083B0019001987C21405C012803D102A994
:10DC52000220087026E001997C2201208854019953
:10DC62008022242088500198006800680090019862
:10DC7200036818680121884318600098490788439F
:10DC8200009001990020486600980199096808608F
:10DC920001992020885001997C220020885402A9F1
:0CDCA2000020087002A8007803B0704752
:10DCAE0081B00090009880214058212820D1009802
:10DCBE005621405A00280CD100980168086880222D
:10DCCE00904308600098016808684022104308607D
:10DCDE000DE00099086D0078096888620099086D5A
:10DCEE00401C086500995622885A401E88520BE047
:10DCFE0000980168086880229043086000980168C7
:0CDD0E00086840221043086001B0704714
:10DD1A0000B585B00490039104980399891EF7F71A
:10DD2A00C2FB014601A80180049A03998A18511E70
:10DD3A0009780902921E12788A1869460A800088B0
:10DD4A000988884202D10398029002E00020C04369
:08DD5A000290029805B000BD23
:10DD620000B585B00490039104980399F7F79FFBDF
:10DD7200014602A80180029901AA11704078694601
:10DD8200087001980499039A88540398401C0390E0
:10DD920000980499039A88540398401C03900398AE
:04DDA20005B000BD0B
:10DDA60081B000900098007D0121084001B07047C5
:10DDB60010B588B007900691059204A803700698DE
:10DDC6004078039003980190032806D0019806280E
:10DDD6000CD00198102812D01AE007980699059AD7
:10DDE60004AB1B78F7F7D7FB029018E00798069963
:10DDF600059A04AB1B78F7F746FC02900FE00798EC
:10DE06000699059A04AB1B78F7F79FFC029006E08B
:10DE160007980399059B0122FFF783FA029002985F
:04DE260008B010BD73
:10DE2A0080B50520000701221103FFF7CBFD80BD55
:08DE3A0080B5F8F742FC80BD41
:0CDE420080B501204002F3F7BEFE80BD59
:10DE4E00F0B581B01E4615460C4607461846FEF73D
:10DE5E000CFA0146002000290AD46543A54207D3D7
:10DE6E00304639462A46FFF7A6FB2146FDF79DFAB6
:04DE7E0001B0F0BD42
:04DE8200C80F70470E
:10DE8600F0B581B01C4615460091CA0017183E46EB
:10DE9600103EB068F1682A46FFF77EFA0CCEFCF712
:10DEA60048FF009A032A0DDB183F561E2A462346D2
:10DEB600FFF772FA0CCF083FFCF73BFF761E083FD0
:10DEC600012EF3D82A462346FFF766FA01B0F0BDC5
:10DED600F0B581B01D4616460346C800022916DB7A
:10DEE60000931F18083F4C1C304629460CCF083FAC
:10DEF600FCF71FFF32462B46FFF74EFA641E083F1B
:10DF0600022CF3D8009B083306460D4600E01B188A
:10DF1600083B0CCB30462946FCF70BFF01B0F0BDA1
:08DF2600C1174840401A704782
:10DF2E0070B5012A09DB0C460546561C28462146CB
:0CDF3E00FFF7D7FA761E012EF8D870BD50
:10DF4A0010B50C46436A01212046FFF77BFF10BD3E
:04DF5A0040207047AC
:10DF5E00024601207F2901D9C043704711707047D6
:0CDF6E00014661391A2900D220387047A2
:0CDF7A00014661391A2900D22038704796
:10DF86004552524F52205452494D4D494E47205604
:07DF9600414C5545530A0000
:0FDF9D0049205265666572656E7A3D25660A00F9
:0BDFAC00547368756E743D25660A0012
:10DFB7002D2D2D204761696E2044726966742043B8
:07DFC700414C202D2D2D001F
:0FDFCE0041637475616C20543D256620430A0041
:10DFDD0041637574616C20493D2566204128776940
:10DFED0074686F7574206761696E2074656D70203B
:10DFFD00647269667420636F7272656374696F6EA3
:03E00D00290A00DD
:10E010004B6F7272656B74757266616B746F723D73
:10E020002566205B2031202F2043656C7369757352
:03E030005D0A0086
:10E033004552524F52204144535F313236305F498B
:0FE043006E7075744D757853656C6563740A0063
:10E0520046697273742073746172742064657465A6
:07E0620063746564210A00EC
:0FE069004953454E534F523A20496E69740A008D
:10E07800466C617368206F6220756E6C6F636B20ED
:07E088006572726F720A005D
:0FE08F00466C61736820206C6F636B65640A00D8
:10E09E002E2E2E466C61736820756E6C6F636B65E9
:03E0AE00640A0001
:10E0B1004F5554505554535F4C56505F5348554E2D
:10E0C100545F4F56455254454D5045524154555257
:03E0D100450A00FD
:0FE0D4004F5554505554204C5650204F4B0A0076
:10E0E3004F5554505554535F4F56505F5348554EF8
:10E0F300545F4F56455254454D5045524154555225
:03E10300450A00CA
:0FE106004F5554505554204F5650204F4B0A0040
:07E11500286E756C6C2900F7
:10E11C004A616E75617279004665627275617279D9
:10E12C00004D6172636800417072696C004D6179D9
:10E13C00004A756E65004A756C7900417567757398
:10E14C00740053657074656D626572004F63746F13
:10E15C00626572004E6F76656D6265720044656330
:07E16C00656D6265720000A1
:07E17300414D00504D00007A
:0FE17A0025612025622025652025542025590088
:0EE1890075617274206572726F72200A0D004B
:10E197002D2D2D204761696E202043414C202D2DC8
:02E1A7002D0049
:10E1A9004144535F313236305F426174746572792C
:10E1B90043757272656E744761696E43616C696219
:10E1C900726174696F6E53746172743A2045525268
:10E1D9004F5220494E2043414C4942524154494FE4
:10E1E9004E2C204E4F205245464552454E43452020
:0AE1F90043555252454E54210A00CE
:0AE2030054736869703D25660A0037
:10E20D002D2D2D204761696E202043414C20454E18
:06E21D0044452D2D2D00EB
:0EE2230064656C746120543D256620430A003A
:0AE2310052656620493D25660A008B
:10E23B004552524F52204144535F313236305F5377
:10E24B006574436F6E76657273696F6E4D6F64653F
:02E25B000A00B7
:10E25D004E6F726D616C2073746172742077697486
:10E26D00686F757420454550524F4D206368616E3F
:0EE27D006765732064657465637465640A00E8
:10E28B00454550524F4D2046554C4C20524553540A
:06E29B004F5245210A006C
:10E2A100454550524F4D2053544F524520434F4EF8
:06E2B100464947210A0066
:0EE2B7004144533132363020496E69740A00FA
:10E2C5002E2E2E456E61626C65206C6F636B20652A
:06E2D50072726F720A0074
:10E2DB002E2E2E466C617368206C6F636B20616C05
:0EE2EB007265616479206163746976650A006A
:10E2F9002E2E2E466C617368206F6220756E6C6FCE
:06E30900636B65640A006D
:10E30F00466C617368204F7074696F6E62797465C3
:10E31F002070726F6772616D6D206661696C6564E4
:02E32F000A00E2
:10E331002E2E2E44697361626C65206C6F636B20B5
:10E3410070726F636573732066696E697368656463
:02E351000A00C0
:10E353004F5554505554535F4C56505F424154549B
:10E363004552595F554E444552564F4C54414745CB
:02E373000A009E
:10E375004F5554505554535F4C56505F4348495080
:10E385005F4F56455254454D50455241545552459F
:02E395000A007C
:10E397004F5554505554535F4F56505F434849505B
:10E3A7005F4F56455254454D50455241545552457D
:02E3B7000A005A
:10E3B9004F5554505554535F4F56505F4348495039
:10E3C9005F554E444554454D50455241545552456B
:02E3D9000A0038
:10E3DB0053756E646179004D6F6E6461790054758D
:10E3EB006573646179005765646E65736461790068
:10E3FB00546875727364617900467269646179005F
:0AE40B0053617475726461790000BA
:02E415004300C2
:02E417002E00D5
:10E4190056616C7565206E6F742076616C69640A4B
:01E4290000F2
:10E42A004672657175656E6379204D6561737572A3
:09E43A006564203D2025640A0000
:10E44300492028776974686F757420636F6D7065F0
:0DE453006E736174696F6E293D25660A00C5
:10E460004552524F52204144535F313236305F5350
:10E470006574496E7465726E616C5265666572652D
:05E480006E63650A0057
:0DE4850057726974696E6720534E210A00BA
:10E49200554E4B4E4F574E20434F4D4D414E440A21
:01E4A2000079
:10E4A300537461727420656E61626C65207265617C
:10E4B300646F75742070726F74656374696F6E0A2C
:01E4C3000058
:10E4C4002E2E2E466C61736820756E6C6F636B0A1A
:01E4D4000047
:10E4D500466C617368204F7074696F6E62797465FC
:09E4E500206C6F636B65640A0092
:10E4EE002E2E2E456E61626C65206C6F636B2070F4
:10E4FE00726F636573732066696E69736865640A0B
:01E50E00000C
:10E50F00466C617368204F7074696F6E62797465C1
:0DE51F002070726F6772616D6D65640A0097
:10E52C004F5554505554535F4C56505F4F564552AF
:09E53C0043555252454E540A00A9
:10E545004F5554505554535F4F56505F42415454A4
:10E555004552595F4F564552564F4C544147450A0F
:01E5650000B5
:10E566004F5554505554535F4F56505F4F56455272
:09E5760043555252454E540A006F
:05E57F002D494E46008D
:05E584002D696E660028
:05E589002B494E460085
:05E58E002B696E660020
:10E5930000000000000054545220524547474553A1
:01E5A3000077
:09E5A4005465726D696E616C0032
:09E5AD00256D2F25642F2579004E
:09E5B60025483A254D3A25530091
:10E5BF0053756E004D6F6E0054756500576564009E
:0DE5CF0054687500467269005361740000C5
:10E5DC004A616E00466562004D61720041707200C6
:10E5EC004D6179004A756E004A756C004175670083
:10E5FC00536570004F6374004E6F76004465630082
:01E60C00000D
:01E60D00000C
:0DE60E000007032004170201085710408088
:10E61B004552524F52204144535F313236305F5393
:0CE62B00657444617461526174650A00FA
:10E637004B6F7272656B74757266616B746F723D46
:04E6470025660A003A
:10E64B002D2D2D204761696E20447269667420431D
:0CE65B00414C20454E4445202D2D2D0043
:10E667004552524F52204144535F313236305F5347
:0CE67700657443686F704D6F64650A00A5
:10E68300454550524F4D20776173206368616E6733
:10E69300656421205765206E65656420746F207062
:10E6A300726573657276652063616C696272617409
:10E6B300696F6E20616E642073657474696E67732D
:08E6C3002064617461210A006A
:10E6CB00454550524F4D20464143544F52592052CD
:10E6DB004553544F52452F555044415445210A0040
:10E6EB007265616420636F6E6669672E2E2E0A0059
:10E6FB00666163746F727920726573746F72652EC5
:04E70B002E2E0A00A4
:10E70F00466C61736820756E6C6F636B20657272F7
:04E71F006F720A000B
:10E7230050524F54454354494F4E3A204F425F5243
:0CE7330044505F4C4556454C5F300A00D6
:10E73F0050524F54454354494F4E3A204F425F5227
:0CE74F0044505F4C4556454C5F310A00B9
:10E75B0050524F54454354494F4E3A204F425F520B
:0CE76B0044505F4C4556454C5F320A009C
:10E777004F5554505554535F4C56505F5348554E60
:10E78700545F554E44455254454D5045524154559A
:04E7970052450A00DD
:10E79B004F5554505554535F4F56505F5348554E39
:10E7AB00545F554E44455254454D50455241545576
:04E7BB0052450A00B9
:10E7BF0030313233343536373839414243444546A8
:10E7CF0030313233343536373839616263646566D8
:04E7DF004E414E0059
:04E7E3006E616E00F5
:10E7E70020202020202020202068282828282020BA
:10E7F7002020202020202020202020202020202012
:10E8070048101010101010101010101010101010C9
:10E817008484848484848484848410101010101069
:10E8270010818181818181010101010101010101C2
:10E837000101010101010101010101101010101076
:10E847001082828282828202020202020202020293
:10E85700020202020202020202020210101010203B
:10E8680029E900089D000020221400003BE9000867
:10E878000000002088E800089D000000F3C500089B
:10E8880088B00590049103A90020087005980290AB
:10E898000498019015490868012292041043086001
:10E8A800EFF3108006900698009072B603A80078DF
:10E8B8003F280ED801980068029908600198001D49
:10E8C80001900298001D02900398401C03A908704B
:10E8D800ECE707480068C003002800D5F9E700986E
:10E8E8000790079880F3108808B0704714200240FA
:10E8F8001020024064C5000864C5000864C500080B
:10E9080064C5000864C5000804000000C00F0020AA
:10E91800C40F0020C80F00200024F40001000000EC
:10E92800206861680834002200E042540139FCD5AF
:02E93800704726
:10E93A0020686168A2680C3401E08B5C8354013A58
:04E94A00FBD5704742
:020000040801F1
:04C7FC00B83E7CA324
:040000050800C5FD2D
:00000001FF
